:020000040000FA
:10000000000204000000000024A7000024A7000054
:1000100024A7000024A7000024A7000024A70000B4
:1000200024A7000024A7000024A7000024A70000A4
:1000300024A7000024A7000024A7000024A7000094
:1000400024A7000024A7000024A7000024A7000084
:1000500024A70000587A00007E7A000024A7000040
:1000600024A7000024A7000024A7000024A7000064
:1000700024A7000024A7000024A7000024A7000054
:1000800024A7000024A7000024A7000024A7000044
:1000900024A7000024A7000024A7000024A7000034
:1000A00024A7000024A7000024A7000024A7000024
:1000B00024A7000024A7000024A7000024A7000014
:1000C00024A7000024A7000024A7000024A7000004
:1000D00024A7000024A7000024A7000024A70000F4
:1000E00024A7000024A7000024A7000024A70000E4
:1000F00024A7000024A7000024A7000024A70000D4
:1001000024A7000024A7000024A7000024A70000C3
:1001100024A7000024A7000024A7000024A70000B3
:1001200024A7000024A7000024A7000024A70000A3
:1001300024A7000024A7000024A7000024A7000093
:1001400024A7000024A7000024A7000024A7000083
:1001500024A7000024A7000024A7000024A7000073
:1001600024A7000024A7000024A7000024A7000063
:1001700024A7000024A7000024A7000024A7000053
:1001800024A7000024A7000024A7000024A7000043
:1001900024A7000024A7000024A7000024A7000033
:1001A00024A7000024A7000024A7000024A7000023
:1001B00024A7000024A7000024A7000024A7000013
:1001C00024A7000024A7000024A7000024A7000003
:1001D00024A7000024A7000024A7000024A70000F3
:1001E00024A7000024A7000024A7000024A70000E3
:1001F00024A7000024A7000024A7000024A70000D3
:10020000FFFFFF00FFFFFF0024A7000024A700005E
:1002100024A7000024A7000024A7000024A70000B2
:1002200024A7000024A7000024A7000024A70000A2
:1002300024A7000024A7000024A7000024A7000092
:1002400024A7000024A7000024A7000024A7000082
:1002500024A70000587A00007E7A000024A700003E
:1002600024A7000024A7000024A7000024A7000062
:1002700024A7000024A7000024A7000024A7000052
:1002800024A7000024A7000024A7000024A7000042
:1002900024A7000024A7000024A7000024A7000032
:1002A00024A7000024A7000024A7000024A7000022
:1002B00024A7000024A7000024A7000024A7000012
:1002C00024A7000024A7000024A7000024A7000002
:1002D00024A7000024A7000024A7000024A70000F2
:1002E00024A7000024A7000024A7000024A70000E2
:1002F00024A7000024A7000024A7000024A70000D2
:1003000024A7000024A7000024A7000024A70000C1
:1003100024A7000024A7000024A7000024A70000B1
:1003200024A7000024A7000024A7000024A70000A1
:1003300024A7000024A7000024A7000024A7000091
:1003400024A7000024A7000024A7000024A7000081
:1003500024A7000024A7000024A7000024A7000071
:1003600024A7000024A7000024A7000024A7000061
:1003700024A7000024A7000024A7000024A7000051
:1003800024A7000024A7000024A7000024A7000041
:1003900024A7000024A7000024A7000024A7000031
:1003A00024A7000024A7000024A7000024A7000021
:1003B00024A7000024A7000024A7000024A7000011
:1003C00024A7000024A7000024A7000024A7000001
:1003D00024A7000024A7000024A7000024A70000F1
:1003E00024A7000024A7000024A7000024A70000E1
:1003F00024A7000024A7000024A7000024A70000D1
:10040000AF242200007F22000001880000000000CD
:100410000C000700608B290001002000110007007C
:10042000000020000000E000020032000000020096
:10043000000000008CA50200000000000040DA006F
:100440000000FE004440A900603320000000E000EE
:100450000300320000002000A00188004440A800F2
:100460000000060091018800800078000000EB0089
:1004700015003700E280400032A0B4009101BA00BC
:10048000E280400032A0B4009102BA00E280400055
:1004900032A0B4000002EB00472BDE00F507B200EB
:1004A000602CE10004003A000059EB008301E900F0
:1004B000FDFF3E00040037006128E100010032002A
:1004C0000082EB00040007001101BA000200E00006
:1004D000E8FF3A00000006003159BA008301E90044
:1004E0000C0032002159BA008301E90008003200F3
:1004F0000400E00003003A00E280400032A0B400B3
:10050000F5FF370011D9BA008301E900FAFF3A007C
:100510008100E800E180400032A0B4000000060045
:1005200000000000000000000000000000000000CB
:1005300000000000000000000000000000000000BB
:1005400000000000000000000000000000000000AB
:10055000000000000000000000000000000000009B
:1007D000889FBE008A9FBE00010578000100E000EE
:1007E0000400350008003C000000E000200032005A
:1007F0000500370060001000E080180002003B0098
:1008000001F02C001A0037000004BE006011B8008F
:100810006B0920000982CF00020039000882CF0056
:100820000441B000694252000E00320008003B0053
:1008300082817100610164008904D1000884D300C1
:100840008B05E8000442E800F9FF3A000500370094
:100850000804440089844C008B05E9000442E90047
:10086000FBFF3A002C0107000AF0A70001F0A000EE
:100870004F05BE004F04BE0000000600F4FF2F002D
:100880004B0137001400200049013700889FBE004B
:100890008A9FBE008C1F780060010700670133004B
:1008A00003866C006450E1002E0032006420E100F9
:1008B000330032006150E1002F0032006120E1007E
:1008C0003100320085855500EB07B000090020009B
:1008D00008042000050037000804440089844C0007
:1008E0000A0031000603430087834B0000015300D8
:1008F00081815B00F8FF33000203BE000800A00006
:100900000804440089844C00F6FF3900C639DD0034
:100910008301730001003200130020008904D1001C
:100920000884D3000998A300050032000800A7003E
:100930000300A0008904D1000884D3008B05E800DF
:100940008904D1000884D3000001EB000281D200A9
:10095000F100070001F0A1000CF0A70001F0A000D9
:100960003F0137006420E100410132000801BE0070
:100970000200BE00F7FF37006120E1003C013200B9
:100980006000B800F3FF37000000200001F82700E6
:10099000F0FF370003F0A200889FBE008A9FBE00D0
:1009A0008C1F78001D010700240133006450E10012
:1009B0004F0032006420E1005200320003826C00DC
:1009C00007003B000905D0000306D000820F540049
:1009D0000C065D0002003900020032008901780037
:1009E000030678008582550004003D000003FD00E9
:1009F0008103FD008502EA008B854200840F7200AE
:100A000002003B0060001000E08018006011B80098
:100A10000005EB007A28E1000A00390006007800A2
:100A2000C75DDD00F707B200878075002D00370035
:100A3000828171000A017800610560008180D10027
:100A40000080D3008502E900F9FF3B000604400066
:100A50008784480002003B0060041400E0841C000E
:100A60000988A300070032008A8171008281710029
:100A7000610164008904D1000884D3008B05E8007B
:100A8000170037000978A30013003A000B00E000BC
:100A9000130034008B05E9000804440089844C00ED
:100AA0000A4474000978A3000D003A000B00E0002E
:100AB000070034008B05E9000804440089844C00D9
:100AC00001003A000B0020000978A300F7FF320074
:100AD0000001EB0002003700828171000A017800FA
:100AE0008D0007000CF0A70001F0A000DC0037002B
:100AF0006420E10002003A00838F6C00DC003300C8
:100B00000801BE000200BE00D5003700889FBE006D
:100B10008A9FBE008C1F7800C0000700C70033000A
:100B200003866C006450E100240032006420E10080
:100B3000270032006150E100220032006120E10014
:100B4000210032008B854200EB07B1000134B80070
:100B5000003AB8000804420089844A00013AB8000B
:100B60000030B8008880400009014A0004003300CA
:100B70000000400081804800020149008B05E90027
:100B8000C909DD008301700001003200130020005C
:100B9000C814DE004814DD004709DE001200B20070
:100BA000C808DE00088470005B00070001F0A100A7
:100BB0000CF0A70001F0A000A90037006120E100BF
:100BC000AB0032000801BE000200BE00F7FF370094
:100BD0006150E100FCFF3A00A50037000001BE00B3
:100BE000A60007000470A70003F0A10003F8A3000B
:100BF00013003A006509B100100032000900350009
:100C00006928E1000200350001002800000005000D
:100C100000004000818048008502E900FCFF3A00A6
:100C200000000600F88F4200050035008100D10069
:100C30000080D3008502E800FCFF3A0000000600B7
:100C40008000EB00000005006022B80006022000D2
:100C50000000D0008180D2000482D2008582D200C0
:100C60000000A0000202520083825A0003003100FB
:100C70000202420083824A000000A1000603E9004C
:100C8000F3FF3A0000000600EFFF07000400BE007B
:100C9000000006000001BE00780007000470A700F5
:100CA00003F0A1006509B100160032000D00350007
:100CB0006828E10006003500F0FF2F00F1FF270053
:100CC0000300E00013003B000100280000000500C5
:100CD00000004000818048008502E900FCFF3A00E6
:100CE00008003700F88F420002003C008000EB0053
:100CF000000005008100D1000080D3008502E800DB
:100D0000FCFF3A000300E00002003B00600010001E
:100D1000E08018000000060081002000618055007E
:100D20000B003D000B00200061FE2F000100E100E0
:100D30001D00340082817100610164008904D100CA
:100D40000884D3000000E800FAFF3A007100200098
:100D500061006400030070000200600009003200BE
:100D600061044400E0844C000988A50005003200BD
:100D70008B05E8006808E10002003A008904D10010
:100D80000884D300F20F20000258E10005003D0066
:100D9000C75DDD00F907B2008980750008007800A2
:100DA000000006000BF827008B007800000005000B
:100DB000889FBE008A9FBE00841F7800170007002E
:100DC0004F00780011003300F0FF2F00838F6C007C
:100DD00006003B00040565000A00A7000800370074
:100DE00009F0A6001000200008003700820F540010
:100DF000838F5C00030039001000200001003E00DA
:100E00000000200009F0A7000000EA004F05BE0026
:100E10004F04BE000000E000000006000004BE0019
:100E2000160007000003BE000405BE000200BE005D
:100E300012000700844F7500000006000200BE008B
:100E40006450E100050036006420E1000200360035
:100E50000968A30001003A000800BE000160A0007C
:100E60004F0678004F05BE004F04BE00000006008C
:100E7000F0FF2F00F1FF2700F9FF3700C70ADE005F
:100E8000F107B200F50FB20008003200E1CF4200D6
:100E9000020032000170A00024000500810F7000E4
:100EA000010032000408050044000500810F7000B5
:100EB00002003A00140005008502E900000040002D
:100EC00081C04800FCFF3B000170A0002400050029
:100ED000005E0000BCE20000613F0000DD83000016
:100EE000C29C00007E200000A3FD00001F41000006
:100EF0009DC30000217F0000FCA20000401E0000F6
:100F00005F010000E3BD00003E60000082DC0000E5
:100F1000237D00009FC10000421C0000FEA00000D5
:100F2000E1BF00005D03000080DE00003C620000C5
:100F3000BEE00000025C0000DF810000633D0000B5
:100F40007C220000C09E00001D430000A1FF0000A5
:100F500046180000FAA40000277900009BC5000095
:100F600084DA000038660000E5BB00005907000085
:100F7000DB85000067390000BAE400000658000075
:100F800019470000A5FB000078260000C49A000065
:100F9000653B0000D9870000045A0000B8E6000055
:100FA000A7F900001B450000C69800007A24000045
:100FB000F8A60000441A000099C70000257B000035
:100FC0003A64000086D800005B050000E7B9000025
:100FD0008CD20000306E0000EDB30000510F000015
:100FE0004E100000F2AC00002F71000093CD000005
:100FF000114F0000ADF30000702E0000CC920000F5
:10100000D38D00006F310000B2EC00000E500000E4
:10101000AFF10000134D0000CE900000722C0000D4
:101020006D330000D18F00000C520000B0EE0000C4
:10103000326C00008ED00000530D0000EFB10000B4
:10104000F0AE00004C12000091CF00002D730000A4
:10105000CA94000076280000ABF500001749000094
:1010600008560000B4EA000069370000D58B000084
:1010700057090000EBB50000366800008AD4000074
:1010800095CB000029770000F4AA00004816000064
:10109000E9B70000550B000088D60000346A000054
:1010A0002B75000097C900004A140000F6A8000044
:1010B000742A0000C8960000154B0000A9F7000034
:1010C000B6E800000A540000D78900006B35000024
:1010D0003E2000000008000020080000001B000067
:1010E0005B440000001B00005B00000044000000A7
:1010F0001B5B0000430000001B5B0000324B000044
:101100000D00000043000000001B00005B320000E7
:101110004400000057610000726E0000696E00001C
:10112000673A0000206E00006F200000766F00001C
:101130006C74000061670000652000006F6E0000A5
:1011400020560000707500006C6C00007570000087
:1011500020700000696E0000002000003D200000AB
:10116000005600005245000047200000746F000048
:101170006F2000006C6F0000772C000020690000D9
:101180007320000074680000657200006520000094
:1011900061200000736800006F720000743F00005F
:1011A000002E0000203C0000003E0000002E000049
:1011B000200000000D0A000028000000293E000069
:1011C00020000000427500007320000050690000FC
:1011D000726100007465000020760000330000009A
:1011E00046690000726D00007761000072650000C2
:1011F00020760000352E0000392000002872000003
:1012000035330000392900002000000020280000AC
:1012100032340000464A00003634000047410000E6
:101220003030000032200000004100003300000098
:101230004234000000420000350000004238000047
:10124000005500004E4B000000290000004900003E
:10125000090000004F0900000048000009000000DC
:101260004C090000004500006E740000657200002B
:10127000207200006177000020760000616C0000A1
:1012800075650000206600006F72000020420000BB
:1012900052470000000000004C45000054000000D0
:1012A0004946000000540000484500004E00000080
:1012B000454C000053450000004700004F5400001B
:1012C0004F000000474F000053550000420000004F
:1012D0005245000054550000524E000000520000DC
:1012E000454D000000500000524900004E540000DF
:1012F000004900004E500000555400000046000018
:101300004F520000005400004F0000004E45000006
:101310005854000000520000454100004400000005
:1013200044410000544100000053000054410000BB
:10133000525400005200000053540000415200007B
:1013400054000000535400004F50000052000000B1
:10135000535400004F50000000530000454E000061
:10136000440000005245000043450000495600007B
:1013700045000000434C00004B00000044410000C9
:101380005400000042490000545200004541000052
:1013900044000000414400004300000041550000AB
:1013A00058500000494E0000005000005355000006
:1013B00000500000554C00004C550000500000004B
:1013C000444500004C410000590000004155000018
:1013D0005800000046520000455100000044000043
:1013E00055540000590000004D41000043520000D8
:1013F0004F000000454E0000440000000052000075
:10140000554E0000004C00004953000054000000FD
:1014100045580000495400000044000045420000C7
:1014200055470000004E0000455700000000000036
:101430003062000000300000303000002C0000005E
:101440003030000000300000313200003334000042
:1014500035360000373800003941000042430000B3
:10146000444500004630000078000000436F000053
:10147000756C0000646E000027740000206B000093
:10148000656500007020000075700000000000001D
:101490005350000049310000000000000029000006
:1014A000002000005700000020520000004900000A
:1014B00032430000310000003A200000000000002C
:1014C0002E00000031570000303100000000000005
:1014D00008080000080800000800000000000000E4
:1014E000204800007A0000000000000000410000D9
:1014F000525400003100000042420000494F0000F9
:10150000310000005241000057310000000000008F
:10151000314100004C530000000000004F43000028
:101520004431000000000000000000000000000046
:101530002900000000000000000000002800FA0060
:101540000000EB00600F98000000EB00E0678800EF
:101550000000EB00D0678800D0678000200798006B
:101560000000EB00100798000000EB00000F78006F
:101570000000EB00A04088000000EB00F06788004E
:101580000000EB00400798000000EB00000F9800FF
:10159000140037000000EB00600798000B003700D4
:1015A0000E089000EE0090004500DD008100400034
:1015B00000D02000808040000040EB008048780090
:1015C0006E0090000000E800600798006E00900038
:1015D000FF0F5000F2FF34000E0890000000E800FA
:1015E000000F98000E089000E40F5000E9FF34004F
:1015F0000000EB00006D8800A1408000E0022000A8
:101600000088B9006102200080804000E093200043
:1016100000804000A475020000000000D14080005E
:1016200000202000008060000000E0000400320084
:1016300071002000C0592000ACA202000000000090
:1016400080862800A47502000000000032043700E4
:10165000006D80000000E00063003200006D80003B
:101660000000E900006D88000000EB0060079800B2
:101670001E003700D2678000006D8000EE009000F1
:101680004500DD008100400000D0200000804000C7
:1016900090407800A0BF2000000041000148780081
:1016A000006D8000EE0090004500DD0081004000EC
:1016B00000D020000080400010407800007A020036
:1016C00000000000D06780000000E800D0678800BC
:1016D0006E0090000000E80060079800D16780006D
:1016E000F00F200000806000D0678800006D80004F
:1016F000EE0090004500DD008100400000D0200099
:1017000000804000104078000004E000D9FF3A005B
:101710000000EB00006D880033003700C0B52000EA
:1017200010407800644060000004E0002E003200A9
:10173000A1408000E00220000088B900FA004000CB
:10174000E0932000008040001000780000000100BD
:101750000000E00024003200A1408000E0022000F0
:101760000088B9006102200080804000E0932000E2
:1017700000804000A4750200000000008086280060
:10178000A475020000000000E1678000D0678000BF
:10179000808F500014003200E067800060079800DE
:1017A0000D003700EE009000A0BF20000080400038
:1017B00010407800007A020000000000EE00900067
:1017C000F00F200000806000600798006E0090001D
:1017D0000000E80060079800EE009000D0678000ED
:1017E000808F5000EFFF3A00E27902000000000015
:1017F0000004E000C9FF320022C2BF006240600066
:101800000004E0000500320010118000D1FF2F001D
:101810000100600010118800BF033700EE7902005C
:1018200000000000604F98006E4890000080FB00B0
:101830006101B9000217980013179800F007200003
:10184000010020000E1190009E119000800F5100A9
:10185000818F59003C033E000E1090009E109000B6
:10186000006001002D033700E20237003E0137001F
:1018700035033700D8003700F9023700530137002D
:1018800031033700770037002F0337000F0337008D
:101890002D0337002C0337000C033700FE013700FF
:1018A000290337005A013700270337002603370082
:1018B00025033700240337002303370022033700B2
:1018C00021033700200337001F0337001E033700B2
:1018D000020137001C0337001B0337001A033700CF
:1018E00019033700180337001703370016033700B2
:1018F00015033700140337001303370012033700B2
:1019000011033700100337000F0337000E033700B1
:101910000D0337000C0337000B0337000A033700B1
:1019200009033700080337000703370006033700B1
:1019300005033700040337000303370002033700B1
:101940000103370000033700FF023700FE023700B3
:10195000FD023700FC023700FB023700FA023700B5
:10196000F9023700F8023700F7023700F6023700B5
:10197000F5023700F4023700F3023700F2023700B5
:10198000F1023700F0023700EF023700EE023700B5
:10199000ED023700EC023700EB023700EA023700B5
:1019A000E9023700E8023700E7023700E6023700B5
:1019B000E5023700E4023700E3023700E2023700B5
:1019C000E1023700E0023700DF023700DE023700B5
:1019D000DD023700DC023700DB023700DA023700B5
:1019E000D9023700D8023700D7023700D6023700B5
:1019F000D5023700D4023700D3023700D2023700B5
:101A0000D1023700D0023700CF023700CE023700B4
:101A1000CD023700CC023700CB023700CA023700B4
:101A2000C9023700C8023700C7023700C6023700B4
:101A3000C5023700C4023700C3023700C2023700B4
:101A4000C1023700C0023700BF023700BE023700B4
:101A5000BD023700BC023700BB023700BA023700B4
:101A60005D003700E16780002E009000810F50007C
:101A700055003200D16780002E009000810F500089
:101A800010003A00D06780008000E900F00F2000CD
:101A900000806000D0678800D1678000A0BF200070
:101AA000808040000040EB0080487800D1678000D3
:101AB00021079800B0862800A475020000000000ED
:101AC000150337000000EB00000F98002E00900077
:101AD0008000E900F00F20000080600020079800DF
:101AE000F0862800A4750200000000002E0190007E
:101AF00062079800210037006E0190006E00900090
:101B00008000E800A0BF20000080400090407800E6
:101B1000A0BF20000000410001487800EE009000C6
:101B2000A0BF200000804000104078000004E000CA
:101B300007003200EE009000A0BF200000804000AF
:101B400010407800007A0200000000000300370017
:101B500000C2B300007A0200000000000E089000EE
:101B60000000E800000F98006E0090008000E80080
:101B7000F00F20000080600060079800EE009000E9
:101B8000D0678000808F5000DBFF3A00D067800074
:101B90008000E900F00F200000806000D06788001E
:101BA00030872800A4750200000000000E08900095
:101BB0003C7802000000000060872800A475020045
:101BC00000000000D402370070C0B300007A0200A9
:101BD00000000000D0023700D16780002E00900086
:101BE000810F5000390032000000EB00000F980018
:101BF000AE01900063079800210037006E0190004D
:101C00006E0090008000E800A0BF2000008040002F
:101C100090407800A0BF20000000410001487800FB
:101C2000EE009000A0BF200000804000104078002F
:101C30000004E00007003200EE009000A0BF20008A
:101C40000080400010407800007A02000000000090
:101C50000300370000C2B300007A02000000000059
:101C60000E0890000000E800000F98006E00900041
:101C70008000E800F00F20000080600060079800FE
:101C8000EE009000D0678000808F5000DBFF3A00AC
:101C9000D06780008000E900F00F20000080600025
:101CA000D067880030872800A4750200000000007B
:101CB0000E0890003C7802000000000060872800B9
:101CC000A4750200000000009302370070C0B3004A
:101CD000007A0200000000008F023700EE79020057
:101CE00000000000604F9800EE489000B0C5B300BF
:101CF00080CF500088023A00EE7902000000000018
:101D0000604F98006E4890000080FB00700F9800B4
:101D100020042000FE089000808F5000DE0032007A
:101D2000200420007E099000800F510005003C0037
:101D300010042000FE099000808F51003400320012
:101D40007502370030042000FE089000808F50009C
:101D50001E003200400420007E099000800F5100D8
:101D6000010032006C0237004E009000E40F50007A
:101D700005003400CA8F0200000000000000EB00E4
:101D80004007980064023700E16780002E00900051
:101D9000810F5000090032002E0090008000E90001
:101DA000F00F20000080600020079800F0862800D7
:101DB000A4750200000000005702370070C0B30095
:101DC000007A02000000000053023700D167800053
:101DD0002E009000810F5000090032002E0090006C
:101DE0008000E800F00F20000080600020079800CD
:101DF00080872800A475020000000000460237001A
:101E000070C0B300007A02000000000042023700F8
:101E10000000EB00000F7800E06780000000E900A0
:101E200080007800F00F20000080600060079800BC
:101E30008D003700EE009000A0BF20000080400021
:101E4000104078000004E00082003A006E0090002C
:101E50008000E900F00F200080806000A0BF20001B
:101E600000804000104078000004E000790032005B
:101E70001E0FE8001E0090009E0F10007500360037
:101E80001E0090000000E80010079800E167800045
:101E9000D0678000808F5000140032000A003700A5
:101EA000D1678000A0BF2000808040000040EB0090
:101EB00080487800D06780008000E900F00F2000A3
:101EC00000806000D0678800D1678000E0678000F4
:101ED000808F5000F2FF3A00D1678000A0BF200041
:101EE000808040000040EB00804878006E00900049
:101EF0008000E900F00F200000806000000F9800D3
:101F0000110037008E089000A0BF20000080400024
:101F1000104078000004E00006003A000E0890002F
:101F20008000E800F00F200000806000500798005B
:101F3000090037000E0890008000E900F00F200033
:101F400000806000000F98008E089000D06780002D
:101F5000808F5000EBFF3A00C0872800A475020074
:101F600000000000A1408000E00220000088B900CD
:101F70006102200080804000E0932000008040004B
:101F8000A475020000000000D14080000020200065
:101F9000008060000000E0000400320071002000BA
:101FA000C0592000ACA2020000000000808628007A
:101FB000A475020000000000DE019000030F9800ED
:101FC000180037008E089000A0BF2000008040005D
:101FD00010407800007A020000000000D267800004
:101FE0008E089000A0BF2000008040009040780044
:101FF000A0BF20000000410001487800D0678000A9
:102000008000E800F00F200000806000D0678800AA
:102010000E0890008000E800F00F200000806000B3
:10202000000F98008E0890006E009000808F500086
:10203000E4FF3A00D1678000A0BF2000808040000C
:102040000040EB0080487800D067800020079800AF
:10205000090037006E0090008000E900F00F2000BA
:102060000080600060079800EE009000D06780005C
:10207000808F50006FFF3A00EE009000D067800024
:10208000808F5000A4013A0070C0B300007A0200B3
:1020900000000000A00137000000EB00000F7800F6
:1020A000E06780000000E90080007800F00F200069
:1020B00000806000600798008E003700EE009000FE
:1020C000A0BF200000804000104078000004E00025
:1020D00083003A006E0090008000E900F00F2000BD
:1020E00080806000A0BF2000008040001040780089
:1020F0000004E0007A0032001E0FE8001E0090008D
:102100000000E9009E0F500075003A001E0090008C
:102110000000E90010079800E1678000D0678000A8
:10212000808F5000140032000A003700D167800011
:10213000A0BF2000808040000040EB008048780075
:10214000D06780008000E900F00F20000080600070
:10215000D0678800D1678000E0678000808F5000E2
:10216000F2FF3A00D1678000A0BF200080804000CD
:102170000040EB00804878006E0090008000E9008D
:10218000F00F200000806000000F98001100370061
:102190008E089000A0BF2000008040001040780012
:1021A0000004E00006003A000E0890008000E800FD
:1021B000F00F2000008060005007980009003700F1
:1021C0000E0890008000E900F00F20000080600001
:1021D000000F98008E089000D0678000808F50001C
:1021E000EBFF3A00C0872800A47502000000000041
:1021F000A1408000E00220000088B90061022000B8
:1022000080804000E093200000804000A475020020
:1022100000000000D140800000202000008060000D
:102220000000E0000400320071002000C0592000CE
:10223000ACA202000000000080862800A475020005
:1022400000000000DE009000010F98001800370029
:102250008E089000A0BF2000008040001040780051
:10226000007A020000000000D26780008E08900013
:10227000A0BF20000080400090407800A0BF200058
:102280000000410001487800D06780008000E8002D
:10229000F00F200000806000D06788000E089000DA
:1022A0008000E800F00F200000806000000F980020
:1022B0008E0890006E009000808F5000E4FF3A007E
:1022C000D1678000A0BF2000808040000040EB006C
:1022D00080487800D2678000220798000900370004
:1022E0006E0090008000E900F00F20000080600088
:1022F00060079800EE009000D0678000808F50004B
:102300006EFF3A00EE009000D0678000808F500092
:1023100001013A001E009000E10F500031003A0028
:10232000C0872800A475020000000000A1408000C2
:10233000E00220000088B900610220008080400097
:10234000E093200000804000A4750200000000001F
:10235000D140800000202000008060000000E000EC
:102360000400320071002000C0592000ACA202001D
:102370000000000080862800A47502000000000014
:102380000A003700D1678000A0BF20008080400095
:102390000040EB0080487800D06780008000E900B2
:1023A000F00F200000806000D0678800D1678000B7
:1023B000E0678000808F5000F2FF3A00D167800014
:1023C000A0BF2000808040000040EB0080487800E3
:1023D000D3678000230798000000EB0010079800E7
:1023E000CD00370070C0B300007A0200000000008A
:1023F000C9003700E16780002E009000810F500077
:1024000013003200E16780002E00900001005000B0
:1024100080007800F00F200000806000000F98001E
:1024200030872800A4750200000000000E0890000C
:102430003C7802000000000060872800A4750200BC
:1024400000000000E067800020079800B20037001D
:1024500070C0B300007A020000000000AE00370038
:10246000D16780002E009000810F500013003200D1
:10247000D16780002E00900000805000800078001E
:10248000F00F200000806000000F980030872800C7
:10249000A4750200000000000E0890003C780200C5
:1024A0000000000020882800A47502000000000041
:1024B000D1678000210798009700370070C0B300F3
:1024C000007A020000000000930037001000200096
:1024D000600F98000000EB0010079800D1678000A3
:1024E000A0BF2000808040000040EB0080487800C2
:1024F000D06780008000E800F00F200000806000BE
:10250000D0678800D26780002207980040882800A2
:10251000D0750200000000007F0037004E009000E0
:102520000000E800400798004E009000F40F5000B3
:1025300079003A008A7B0200000000000000EB00F6
:102540004007980074003700D06780008000E800E2
:10255000F00F200080806000E0678000808F5000D6
:102560006A0032006E489000FF4F5000670036004E
:10257000EE489000E0C7B30080CF500063003E00FB
:10258000D16780002E009000808F500015003A0027
:102590006E489000007A020000000000D1678000C1
:1025A0006E499000A0BF20000080400002487800E3
:1025B000D06780008000E800F00F200000806000FD
:1025C000D0678800D1678000A0BF200080804000D5
:1025D0000040EB0080487800D36780002307980014
:1025E0004D003700D16780002E0090000080500021
:1025F00080007800F00F200000806000000F98003D
:1026000030872800A4750200000000000E0890002A
:102610003C7802000000000020882800A475020019
:1026200000000000D0678000600798001D003700A0
:102630006E0090000001E800EE009000A0BF2000B6
:102640000080400090407800A0BF200000004100C2
:1026500001487800EE009000A0BF200000804000FC
:10266000104078000004E00009003200EE00900005
:10267000A0BF20000080400010407800007A0200D7
:102680000000000050882800A4750200000000002F
:102690006E0090008000E900F00F200000806000D4
:1026A000600798006E0190002E0090008000E90005
:1026B000F00F200000806000800F5100DCFF3A0026
:1026C0006E489000007A020000000000AE0090000A
:1026D0006E499000A0BF20000080400002487800B2
:1026E0002E0090008000E800F00F200000806000C5
:1026F00020079800D06780008000E800F00F2000DD
:1027000000806000D06788000300370070C0B3000D
:10271000007A0200000000006E0890000000E00057
:10272000CBFB3200D0678000400F9800E06780004C
:10273000300F98000000EB00600F98000000EB00E5
:10274000500F98000000EB00F0678800D140800037
:1027500000202000008060000000E0001105320031
:10276000EE3602000000000051002000305A200028
:1027700036A302000000000010002000500F980057
:1027800008053700E1678000A0BF200000804000FE
:1027900010407800604F98006E4890000080FB0069
:1027A0006101B9002217980033179800E007200054
:1027B000010020002E119000BE119000800F5100EA
:1027C000818F5900CB043E002E109000BE10900067
:1027D00000600100C9043700C6043700C504370093
:1027E000C4043700C3043700C2043700C1043700F3
:1027F000C0043700BF043700BE043700BF043700F1
:10280000BC043700BB043700BC043700B9043700F0
:10281000B8043700B7043700B6043700B5043700F2
:10282000B4043700B3043700B2043700B1043700F2
:10283000B0043700AF043700AE043700AD043700F2
:10284000AC043700AB043700AA043700A9043700F2
:10285000A8043700A904370086043700C6023700F1
:102860002B01370034013700DD013700CB01370081
:10287000A00437009F0237009E0437009D043700F4
:102880009E0437009D043700320437004B043700A4
:10289000160437003F0337003E0337003D0337007F
:1028A0003C0337003B0337003A0337003903370056
:1028B0003803370037033700360337008D043700FD
:1028C0008C043700E6013700C9003700890437005F
:1028D0003F003700460137003801370085043700D4
:1028E00065003700AA0137008204370081043700F1
:1028F000800437007F0437007E0437007D043700F2
:102900007C043700670037007A0437007904370009
:10291000780437008F0037007604370075043700DD
:10292000C4013700730437007204370071043700A4
:10293000450137006F0437006E0437006D0437001F
:10294000F0023700F6033700000337002A0437008F
:102950000D043700670437000B01370027003700EC
:102960003A0037007C013700620437002900370045
:102970002B0037005F043700180037005D04370074
:102980005C043700540037001A0037005904370040
:102990001C0037005D00370056043700790337000C
:1029A000A0013700530437005204370017003700E6
:1029B000570137004F0437004E0437004D043700ED
:1029C000D9023700A5003700E9023700C3003700FD
:1029D0004CA302000000000048043700B7070700BE
:1029E000A04080000000E000440432001C08070002
:1029F000420437006C060700400437005309070003
:102A00003E0437002D0907003C043700A1080700E9
:102A10003A043700D082020000000000370437007B
:102A2000A04080000000E00005003A00D101200035
:102A3000305D200036A30200000000002F043700A4
:102A400038810200000000002C043700C0B52000CF
:102A5000104078000000A1000010A100C1B52000C6
:102A60008048780061012000805A200036A30200CF
:102A70000000000021043700C0B52000104078009D
:102A80000000A0000010A100C1B52000804878001F
:102A900051012000E05B200036A30200000000008E
:102AA00016043700C0B52000104078000030A000A8
:102AB000C1B5200080487800C1012000B07E200010
:102AC000ACA202000000000040882800D07502007F
:102AD0000000000009043700C0B520001040780055
:102AE0000030A100C1B5200080487800B10120006D
:102AF000007D2000ACA202000000000040882800F9
:102B0000D075020000000000FC033700A0408000E8
:102B10000000E00005003A00D1012000305D2000F7
:102B200036A3020000000000F4033700CB62A900C6
:102B3000C962A90051012000005F2000ACA2020080
:102B40000000000040882800D0750200000000004E
:102B5000EA033700A04080000000E00005003A00D2
:102B6000D1012000305D200036A3020000000000EB
:102B7000E2033700C0B520001040780070406000CC
:102B80000004E00004003A002102200050E8200088
:102B900036A3020000000000C962A800CB62A900B1
:102BA0004101200050602000ACA2020000000000A3
:102BB00040882800D07502000000000021E3A80032
:102BC000B0C0B300B09E020000000000800078009A
:102BD000F0042000808F500003003E00A0882800F1
:102BE000D07502000000000021E3A900C3033700F4
:102BF000E06780008000E800F00F200000806000A7
:102C0000E0678800D8050700F00307006007980018
:102C10006E0090009E78020000000000D08A28001C
:102C2000A4750200000000006E0090003C780200D5
:102C300000000000D08A2800A475020000000000F7
:102C40006E0090000476020000000000408828001A
:102C5000D075020000000000A8033700E067800084
:102C60008000E800F00F200000806000E06788002E
:102C7000BD050700D5030700600798006E009000AF
:102C80000080FB0070A002000000000060079800B8
:102C90006E0090009E78020000000000D08A28009C
:102CA000A4750200000000006E0090003C78020055
:102CB00000000000D08A2800A47502000000000077
:102CC0006E0090000476020000000000408828009A
:102CD000D07502000000000088033700A04080008B
:102CE0000000E00005003A0011C0B30010C0B300BE
:102CF000869B02000000000080033700A101200035
:102D00009061200036A30200000000007B03370022
:102D1000510020003063200036A3020000000000B4
:102D200023C2BF00614060000004E000FCFF3200ED
:102D30000000FE0071033700DCA302000000000069
:102D40000000E0006D033200A1002000806320003D
:102D500036A3020000000000400620000EA0020082
:102D600000000000669E02000000000023C2BF00B9
:102D7000614060000004E000FCFF320081BF2A00D7
:102D8000014001005D033700350507000000E80041
:102D9000000F9800020037000E84020000000000BF
:102DA0000E0890000000E900000F98000E08900047
:102DB0000000E000F8FF3A00500337002805070044
:102DC0000000E800000F980002003700EC830200CA
:102DD000000000000E0890000000E900000F9800BD
:102DE0000E0890000000E000F8FF3A0043033700AF
:102DF0001B0507000000E800000F98000B003700DB
:102E00006101200020642000ACA20200000000004C
:102E100030840200000000008E75020000000000F7
:102E200040882800D0750200000000000E089000C5
:102E30000000E900000F98000E0890000000E0007C
:102E4000EFFF3A002D033700A04080000000E000B3
:102E500005003A00D1012000305D200036A30200B9
:102E60000000000025033700C002A900C202A8002C
:102E700021E3A800200020000EA0020000000000B6
:102E8000A0C0B300B09E02000000000080007800E7
:102E9000001B2000808F50000F00360090C0B30050
:102EA000B09E02000000000080007800702B20001F
:102EB000808F50000800360011012000806520003E
:102EC000ACA202000000000040882800D07502007B
:102ED000000000000C003700C002A900C202A900D7
:102EE000108B2800D0750200000000002101200096
:102EF00090662000ACA2020000000000408828007C
:102F0000D07502000000000021E3A900FB02370099
:102F1000A04080000000E00005003A00D101200040
:102F2000305D200036A3020000000000F3023700ED
:102F3000C002A900C202A900210120009066200061
:102F4000ACA202000000000040882800D0750200FA
:102F500000000000E9023700F1002000A039200045
:102F6000ACA2020000000000CA9E020000000000A7
:102F700011002000903A2000ACA2020000000000E6
:102F800040882800D075020000000000DB023700F6
:102F9000DC9E020000000000D8023700B0040700E9
:102FA000000F98006100200070682000ACA20200B1
:102FB000000000000E089000DE7702000000000014
:102FC00021002000D068200036A30200000000008D
:102FD0000E0890003AA0020000000000C70237006F
:102FE0009F040700000F9800610020007068200017
:102FF000ACA20200000000000E089000DE77020084
:10300000000000002100200090EC200036A3020008
:10301000000000000E0890000EA00200000000005A
:10302000B6023700D04080000090A000D040880059
:10303000B2023700A04080000000E00005003A0026
:10304000D1012000305D200036A302000000000006
:10305000AA0237006484020000000000A7023700C3
:1030600010002000F0678800100020006007980022
:1030700010003700E16780006E0090008080400003
:10308000F00F200080806000A0BF20000080400082
:1030900090407800E0C3B30080CF500002003A00B7
:1030A0000000EB00F06788006E0090000000E80070
:1030B00060079800E16780006E009000808040000B
:1030C000F00F200080806000A0BF20000080400042
:1030D000104078000004E000E6FF3A00EE009000A7
:1030E00020022000808F50000200340010002000D9
:1030F000F0678800F06780000000E0007F023A007F
:10310000E06780008000E800F00F20000080600091
:10311000E0678800AD02070060079800E167800063
:10312000F00F200080806000A0BF200000804000E1
:1031300090407800D0C3B30080CF500040003A00E8
:103140006E0090000000E0003A0034006E00900035
:10315000E50F500037003C00E06780008000E80089
:10316000F00F200000806000E06788006E00900093
:103170000000E900600798000000EB00000F9800D5
:103180000B0037006E0090008E0890004500DD00B7
:103190008100400000D02000808040000040EB0013
:1031A000804878000E0890000000E800000F9800AA
:1031B0000E089000FF0F5000F2FF34000000EB00FB
:1031C000000F980013003700EE0190000E0A9000E7
:1031D000E1678000A0BF200000804000104178001F
:1031E0004518DD008400400000D020000080400031
:1031F000024878000E0890000000E800000F9800D8
:10320000E06780008000E800F00F20000080600090
:10321000E0678800E1678000A0BF200000804000D8
:1032200090407800E0C3B30080CF5000E6FF3A0042
:103230003202370010002000F06788002F023700AC
:103240006E0090000000E0001B003A000000EB0060
:10325000000F9800140037000E0890000040E800AE
:103260003C78020000000000108D2800A4750200C8
:10327000000000000E0890004500DD00800078008E
:1032800000D0200000804000A47502000000000073
:10329000508D2800D0750200000000000E0890003C
:1032A0000000E800000F98000E089000E40F5000A6
:1032B000E9FF3400110237006E0090000000E000CA
:1032C000090034006E009000E50F500006003C003D
:1032D00040882800D075020000000000EE00900039
:1032E000016D88000502370010002000F06788009B
:1032F00002023700E06780008000E800F00F200045
:1033000000806000E067880030020700200F98000E
:1033100015040700E1678000F00F20008080600046
:10332000A0BF2000008040009040780090C2B30011
:1033300080CF50000D003A00A1408000E002200044
:103340000088B900FC004000E093200000804000AD
:10335000900078002E0890000100010040882800AD
:10336000D075020000000000E401370010002000CA
:10337000F0678800E101370010002000F067880046
:10338000100020006007980010003700E1678000FF
:103390006E00900080804000F00F20008080600070
:1033A000A0BF2000008040009040780020C2B30001
:1033B00080CF500002003A000000EB00F067880068
:1033C0006E0090000000E80060079800E167800050
:1033D0006E00900080804000F00F20008080600030
:1033E000A0BF200000804000104078000004E000F2
:1033F000E6FF3A00F06780000000E000BF013A00FD
:1034000071002000F0682000ACA202000000000063
:1034100020C2B300007A0200000000002200370042
:10342000E1678000F00F200000806000E067880006
:10343000E1678000A0BF20000080400010407800BD
:10344000007A020000000000E1678000A0BF2000B9
:1034500000804000104078000000FB00200F980022
:10346000C0B5200010407800684060000004E00013
:10347000040032002E08900070A00200000000003E
:10348000200F9800A1408000E00220000088B900D1
:10349000E8004000E09320000080400090007800A9
:1034A0002E08900001000100E06780000000E800A5
:1034B000E0678800E1678000F00F200080806000F6
:1034C000A0BF2000008040009040780020C2B300E0
:1034D00080CF5000D2FF3A00E0678000F10F20005B
:1034E00001006000E067880020C2B300007A02009B
:1034F0000000000040882800D07502000000000095
:103500007E013700A1408000E00220000088B90061
:1035100080007800E09320000080400010007800D8
:103520000000010075013700A1408000E00220008A
:103530000088B9008080E800E0932000008040000F
:1035400010007800000001006C013700A1408000ED
:10355000E00220000088B900E4004000E093200071
:103560000080400010007800000001006301370077
:10357000A1408000E00220000088B900E600400081
:10358000E09320000080400010007800000001005F
:103590005A01370071002000F0682000ACA2020040
:1035A0000000000089010700200F9800E0678000FC
:1035B0000000E900E0678800E1678000F00F20006C
:1035C00000806000E0678800250307000000E80035
:1035D000000F980045030700300798003E00900058
:1035E0000000E0005D0032003E0090008040780066
:1035F000B0B42000014878003E009000E80F500071
:1036000006003400C0B52000104078000050A00033
:10361000C1B520008048780050003700C0B52000B8
:10362000104078000050A100C1B52000804878000B
:103630004A0037002E089000689F0200000000003A
:10364000C0B52000104078000042B2000004E00045
:1036500004003A00B0B4200010407800E84F500059
:1036600009003A00C0B52000104078000042B200C6
:103670000004E0000B003200B0B4200010407800DD
:10368000F04F500007003200B0C3B300007A0200D0
:1036900000000000B0B42000104078003C78020028
:1036A00000000000C0B520001040780068406000B5
:1036B0000004E000040032002E08900070A0020018
:1036C00000000000200F9800A1408000E0022000D0
:1036D0000088B900E8004000E0932000008040002E
:1036E000900078002E08900001000100100F980053
:1036F00000C2B300007A020000000000C0B5200044
:10370000104078000044B2000004E00013003200D2
:103710006100200060692000ACA2020000000000EF
:10372000C0B5200010407800684060000004E00050
:10373000040032001E08900070A00200000000008B
:10374000100F98001E089000689F02000000000003
:1037500000C2B300007A0200000000000E089000D2
:103760000000E900000F98000E0890000000E00043
:10377000B0FF3A0040882800D07502000000000029
:10378000DE0037006100200060692000ACA202006A
:1037900000000000B20207000000E800000F9800DF
:1037A000D2020700300798003E0090000000E000C1
:1037B000440032003E00900080407800B0B4200009
:1037C000014878003E009000E80F500006003400E9
:1037D000C0B52000104078000050A000C1B5200006
:1037E0008048780037003700C0B5200010407800CE
:1037F0000050A100C1B5200080487800310037009A
:10380000A1408000E00220000088B900EA004000EA
:10381000E0932000008040001000780000000100CC
:10382000100F9800C0B5200010407800684060007C
:103830000004E000040032001E08900070A00200A6
:1038400000000000100F98001E089000689F020002
:1038500000000000C0B52000104078000042B20017
:103860000004E00004003A00B0B4200010407800EA
:10387000E84F500009003A00C0B520001040780021
:103880000042B2000004E0000B003200B0B420009F
:1038900010407800F04F500007003200B0C3B30072
:1038A000007A020000000000B0B420001040780050
:1038B0003C7802000000000000C2B300007A020061
:1038C000000000000E0890000000E900000F9800C2
:1038D0000E0890000000E000C9FF3A004088280070
:1038E000D075020000000000840037008100200035
:1038F000C069200036A3020000000000A140800043
:10390000E00220000088B900EC004000E0932000B5
:1039100000804000100078000000010077003700B0
:1039200081002000406A200036A302000000000051
:10393000A1408000E00220000088B900EE004000B5
:10394000E09320000080400010007800000001009B
:103950006A003700E1002000C06A200036A30200A0
:1039600000000000A1408000E00220000088B900B3
:10397000F0004000E093200000804000100078003C
:10398000000001005D003700E1002000A06B200076
:1039900036A3020000000000A1408000E0022000E9
:1039A0000088B900F2004000E09320000080400051
:1039B000100078000000010050003700C100200016
:1039C000B0672000ACA2020000000000A14080000F
:1039D000E00220000088B900F4004000E0932000DD
:1039E0000080400010007800000001008E75020089
:1039F000000000004100370019020700000F980086
:103A0000D1002000806D2000ACA202000000000068
:103A10000E089000689F0200000000000E08900051
:103A20000000E800000F980008003700A140800067
:103A3000E00220000088B900F6004000E09320007A
:103A40000080400010007800000001000E08900087
:103A50000000E900000F98000E0890000000E00050
:103A6000F2FF3A0040882800D075020000000000F4
:103A700022003700FA0107000000E800000F98005C
:103A8000A1002000506E2000ACA202000000000047
:103A90000D003700A1408000E00220000088B9003E
:103AA000F8004000E0932000008040001000780003
:103AB000000001008E7502000000000000C2B3008B
:103AC000007A0200000000000E0890000000E900EB
:103AD000000F98000E0890000000E000EDFF3A0093
:103AE00001012000806C200036A3020000000000CD
:103AF0000200370010002000F0678800E0678000B7
:103B00008000E800F00F200000806000E06788007F
:103B1000F06780000000E0001C003200510120002E
:103B2000F06E2000ACA2020000000000BE08900071
:103B3000E0678000808F500007003100E067800060
:103B4000804078003E08900000C050003C780200A1
:103B50000000000006003700E06780008040780029
:103B60003E08900000C050003C78020000000000B9
:103B70000000EB00F067880010002000500F980054
:103B800040882800D075020000000000E167800036
:103B9000D0678000808F500002003A0010002000A3
:103BA000500F98005E0890000000E000F5FA320027
:103BB0004E089000E06788004E089000D0678800AB
:103BC0000000EB00600F98008BF637000600FA004B
:103BD0000000EB00100798000000EB00000F7800D9
:103BE000E16780001E00900080804000F00F200000
:103BF00080806000A0BF20000080400090407800DE
:103C000000C3B30080CF500043003400E167800060
:103C10001E00900080804000F00F20008080600037
:103C2000A0BF2000008040009040780090C3B30007
:103C300080CF500038003C00E16780001E009000FB
:103C400080804000F00F200080806000A0BF200036
:103C500000804000104078008000FB0000FD2F0035
:103C6000008F40001E0090000000E8001007980040
:103C7000120037001E0078006A00B900000F7800BB
:103C8000E16780001E00900080804000F00F20005F
:103C900080806000A0BF20000080400010407800BD
:103CA0000000FB009E00400000FD2F00008F400040
:103CB0001E0090000000E80010079800E1678000F7
:103CC0001E00900080804000F00F20008080600087
:103CD000A0BF20000080400090407800F0C2B300F8
:103CE00080CF500051013400E16780001E00900039
:103CF00080804000F00F200080806000A0BF200086
:103D0000008040009040780090C3B30080CF500006
:103D1000D8FF340045013700E16780001E009000A5
:103D200080804000F00F200080806000A0BF200055
:103D3000008040009040780000C3B30080CF500066
:103D400035013A001E0090000000E80010079800BE
:103D5000E16780001E00900080804000F00F20008E
:103D600080806000A0BF200000804000904078006C
:103D700020C6B30080CF50000B003200E167800006
:103D80001E00900080804000F00F200080806000C6
:103D9000A0BF2000008040009040780020C4B30005
:103DA00080CF50002D003A001E0090000000E80077
:103DB00010079800120037001E0078000000400035
:103DC000000F7800E16780001E00900080804000B6
:103DD000F00F200080806000A0BF20000080400025
:103DE000104078000000FB009E00400000FD2F0006
:103DF000008F40001E0090000000E80010079800AF
:103E0000E16780001E00900080804000F00F2000DD
:103E100080806000A0BF20000080400090407800BB
:103E200010C3B30080CF5000E3FF3200E167800091
:103E30001E00900080804000F00F20008080600015
:103E4000A0BF2000008040009040780000C3B30075
:103E500080CF5000D8FF3200F4003700E1678000C7
:103E60001E00900080804000F00F200080806000E5
:103E7000A0BF2000008040009040780080C7B300C1
:103E800080CF50000B003200E16780001E009000E0
:103E900080804000F00F200080806000A0BF2000E4
:103EA000008040009040780080C5B30080CF500073
:103EB0008E003A001E0090000000E80010079800F5
:103EC000470037001E0078004400DD00000F780036
:103ED000E16780001E00900080804000F00F20000D
:103EE00080806000A0BF20000080400090407800EB
:103EF000F0C2B30080CF500018003400E1678000AA
:103F00001E00900080804000F00F20008080600044
:103F1000A0BF2000008040009040780090C3B30014
:103F200080CF50000D003C00E16780001E00900033
:103F300080804000F00F200080806000A0BF200043
:103F400000804000104078000000FB009E00400010
:103F500000FD2F00008F40001E003700E167800049
:103F60001E00900080804000F00F20000081600063
:103F7000E16780001E00900080804000F00F20006C
:103F800080806000A0BF200000804000904078004A
:103F900000C2B30080C07000A0BF2000000041003C
:103FA00001487800E16780001E009000808040009A
:103FB000F00F200080806000A0BF20000080400043
:103FC000104078000000FB009E00400090FA2F0097
:103FD000008F40001E0090000000E80010079800CD
:103FE000E16780001E00900080804000F00F2000FC
:103FF00080806000A0BF20000080400090407800DA
:10400000F0C2B30080CF50000B003400E1678000A5
:104010001E00900080804000F00F20008080600033
:10402000A0BF2000008040009040780090C3B30003
:1040300080CF5000A3FF3400E16780001E00900095
:1040400080804000F00F200080806000A0BF200032
:10405000008040009040780000C4B30080CF500042
:104060000B003400E16780001E009000808040005B
:10407000F00F200080806000A0BF20000080400082
:104080009040780060C4B30080CF50008DFF3400B2
:10409000E16780001E00900080804000F00F20004B
:1040A00080806000A0BF2000008040009040780029
:1040B00000C6B30080CF50005C003400E167800090
:1040C0001E00900080804000F00F20008080600083
:1040D000A0BF2000008040009040780060C6B30080
:1040E00080CF500077FF340050003700E167800038
:1040F0001E00900080804000F00F20008080600053
:10410000A0BF20000080400090407800F0C2B300C3
:1041100080CF500045003400E16780001E00900011
:1041200080804000F00F200080806000A0BF200051
:10413000008040009040780090C3B30080CF5000D2
:104140003A003C00E16780001E0090008080400043
:10415000F00F200080806000A0BF200000804000A1
:10416000104078008000FB0000FD2F00008F400011
:10417000120037001E0078006A00B900000F7800B6
:10418000E16780001E00900080804000F00F20005A
:1041900080806000A0BF20000080400010407800B8
:1041A0000000FB009E00400000FD2F00008F40003B
:1041B0001E0090000000E80010079800E1678000F2
:1041C0001E00900080804000F00F20008080600082
:1041D000A0BF20000080400090407800F0C2B300F3
:1041E00080CF500011003400E16780001E00900075
:1041F00080804000F00F200080806000A0BF200081
:10420000008040009040780090C3B30080CF500001
:10421000D8FF34000500370010002000F067880048
:104220000000EB00200798000A003700E1678000DB
:104230001E00900000804000E0678800E167800079
:10424000F00F200000806000E06788001E0078000A
:10425000200798002E0090000080FA000000060061
:104260000400FA00E06780008000E800F00F200002
:1042700080806000A0BF2000008040009040780057
:10428000A0C3B30080CF500013003A00E067800065
:104290000080E800E0678800E1678000F00F200000
:1042A00000806000E067880048FE0700000F78008B
:1042B000E06780000000E900E0678800E1678000B7
:1042C000F00F200000806000E06788001E0078008A
:1042D0001007980002003700100020001007980017
:1042E0001E0090000080FA00000006000400FA00A2
:1042F000E06780008000E800F00F20008080600010
:10430000A0BF20000080400090407800B0C3B30000
:1043100080CF50000F003A00E06780008080E80006
:10432000F00F200000806000E067880027FE070093
:10433000000F7800E06780008000E900F00F2000A7
:1043400000806000E06788001E0078001007980079
:10435000020037000000EB00100798001E009000DC
:104360000080FA00000006000000FA000500370097
:10437000E06780008000E800F00F2000008060000F
:10438000E0678800E1678000A0BF20000080400057
:104390009040780000C2B30080CF5000F4FF32009C
:1043A0000080FA00000006000400FA000000EB00A4
:1043B000000F7800E06780008000E800F00F200028
:1043C00000806000E0678800E7FF0700FFFD07004E
:1043D000000F78001E00E0004D003A000000EB00E6
:1043E00010079800130037001E0090000040E800FE
:1043F0003C78020000000000708D2800A4750200C7
:10440000000000009E009000E00220000088B9003B
:104410006102200080804000E09320000080400086
:10442000D0750200000000001E0090000000E800AF
:10443000100798001E009000E70F5000EAFF3400BC
:10444000710120004070200036A30200000000002F
:104450000000EB00F06788001300200082002000BD
:10446000110020001000200055000700000FE90097
:10447000E0FF2F009E0F1000030032000080EB00D1
:104480009E0F100005003A00E1002000B0712000EE
:1044900036A302000000000042003700A140800067
:1044A000E00220000088B900010220008080400066
:1044B000E093200000804000100078000000010020
:1044C000669E0200000000001E007800A0408800E8
:1044D000A1408000E00220000088B900FE004000FA
:1044E000E0932000008040001000780000000100F0
:1044F0001E00E00001003200C222A800510020008E
:10450000305A200036A302000000000025003700CA
:104510001E0FE900700020009E0F10001D003C00DF
:10452000A1408000E00220000088B90001022000C4
:1045300080804000E0932000008040001000780060
:1045400000000100669E0200000000001E007800CE
:10455000A0408800A1408000E00220000088B9004F
:10456000FE004000E0932000008040001000780032
:10457000000001001E00E00001003200C222A8007D
:1045800051002000305A200036A302000000000035
:1045900004003700510120009072200036A3020071
:1045A00000000000D06780008000E900F00F2000CC
:1045B00000806000E06788000080FA0000000600CC
:1045C0001E00FA00100F9800210F9800320F98007B
:1045D000430F98000000EB00400798000000EB003C
:1045E000200798000000EB00100798000000EB0087
:1045F000000F7800A08D2800A475020000000000C4
:104600001E0890003C78020000000000E08D2800A9
:10461000A47502000000000067003700EE79020078
:1046200000000000204F98002E4890000000FB0082
:10463000600F98006E089000ED0F500029003200C6
:10464000EE089000ED8F500007003C006E099000CE
:10465000E80F51000D0032006E089000EA0F500084
:104660002000320035003700D0022000EE08900014
:10467000808F50001E003200800720006E099000DD
:10468000800F5100270032002C0037004E009000B0
:104690000000E000070032004E0090000000E9003A
:1046A00040079800B0862800A475020000000000B2
:1046B000410037001E00E000060032000000EB0061
:1046C000000F7800B0862800A475020000000000EA
:1046D0003900370070C0B300007A0200000000000B
:1046E0003500370010002000200798003200370006
:1046F0004E0090000000E00006003A00D0C2B30077
:10470000007A02000000000010002000000F780076
:104710002900370070C0B300007A020000000000DA
:10472000250037004E0890000000E0000300320032
:104730000080EB00500F98005D003700AE489000FD
:10474000F0C2B30080CF500018003400AE48900093
:1047500090C3B30080CF500014003C004E00900086
:10476000E30F50000600340070C0B300007A02006E
:104770000000000040002000400798000E003700B5
:104780002E489000007A020000000000CE00900049
:104790006B0047002E499000827078004E00900018
:1047A0000000E800400798000300370070C0B30025
:1047B000007A0200000000002E0090000000E000DF
:1047C00096FF320040882800D075020000000000EB
:1047D0004E0090000000E00003003A001E08900028
:1047E000500F9800320037000000EB0010079800CF
:1047F0004E0090000000E90040079800CE009000B5
:1048000031079800110037001E0090006A00B900BF
:1048100010079800BE0090004E009000808050006D
:104820006B004700614078008000FB001E00900094
:104830008080400000FD2F0000804000100798009D
:104840004E0090000000E900400798004E009000E4
:104850000000E000ECFF3D009E0090002E0890005C
:10486000808F50000D0035009E0090003E089000A3
:10487000808F500009003C001E00E0000400320060
:104880001E0090000000EA00500F9800080037005A
:104890001E019000520F980005003700B101200062
:1048A000E0EA200036A302000000000049FF3700C4
:1048B0005E0890000080FA00000006000400FA0084
:1048C000208E2800A475020000000000A0812000B6
:1048D00010407800007A02000000000040882800A4
:1048E000D075020000000000008F2800A4750200AF
:1048F00000000000D100200070802000ACA2020067
:1049000000000000A1BF2A000000EB005A7B02005B
:1049100000000000000F78001E0078004800DE0054
:104920003C78020000000000E0C2B300007A020000
:10493000000000001E0078003C780200000000002B
:1049400040882800D07502000000000061002000AF
:1049500000762000ACA2020000000000B040800001
:10496000F6780200000000007100200070EA2000CC
:10497000ACA2020000000000C0408000F6780200F7
:104980000000000060902800A475020000000000F4
:10499000C040800010079800200423009E00900073
:1049A000808F500016003200200423009E009000EB
:1049B000808F500005003E00300023009E009000D4
:1049C000808F50000A0032001900370030042300A5
:1049D0009E009000808F50000D0032006004230084
:1049E0009E009000808F50000D00320010003700B4
:1049F00050912800A4750200000000000F0037004D
:104A000080912800A4750200000000000B00370010
:104A1000B0912800A47502000000000007003700D4
:104A2000E0912800A4750200000000000300370098
:104A300010922800A4750200000000005092280087
:104A4000D075020000000000E10120006076200027
:104A500036A30200000000000080FA0000000600FB
:104A60000000FA005100200020922000ACA20200B9
:104A700000000000C1BF2A000000EB005A7B0200CA
:104A800000000000F6780200000000006100200035
:104A900070922000ACA2020000000000E1BF2A00DA
:104AA0000000EB005A7B020000000000F6780200D4
:104AB0000000000040882800D075020000000000BF
:104AC000C10020004078200036A302000000000052
:104AD00070000700C2C2BF00614060000004E00037
:104AE000050032001101200080652000ACA2020008
:104AF0000000000004003700210120009066200023
:104B0000ACA2020000000000C0C2B300007A0200A4
:104B10000000000000C2B300007A020000000000A4
:104B2000CBC2BF00684060000004E0000500320016
:104B30004101200050602000ACA2020000000000F3
:104B40000400370051012000005F2000ACA20200E9
:104B500000000000C0C2B300007A020000000000A4
:104B600000C2B300007A020000000000C0B52000BF
:104B700010407800704060000004E0000500320042
:104B8000210220000079200036A30200000000006E
:104B900004003700E1012000207B200036A3020042
:104BA00000000000C0B520001040780068406000A0
:104BB0000004E00005003A00B1012000007D200063
:104BC000ACA202000000000004003700C101200078
:104BD000B07E2000ACA2020000000000C0C2B30002
:104BE000007A02000000000000C2B300007A020058
:104BF00000000000B1012000C0202100ACA2020092
:104C000000000000B0B42000104078003C780200A2
:104C10000000000040882800D0750200000000005D
:104C2000C0B520001040780063406000E14F5000A4
:104C300005003A0051012000E05B200036A302008D
:104C4000000000000400370061012000805A2000AD
:104C500036A3020000000000A1408000E002200016
:104C60000088B9004102200080804000E0932000CD
:104C7000008040001000780000000100C10020000A
:104C80004078200036A30200000000000080FA00F7
:104C9000000006000000FA00A1002000A00521008D
:104CA00036A302000000000061042000200B210058
:104CB00036A3020000000000A101200040062100F0
:104CC000ACA2020000000000A1408000E002200031
:104CD0000088B9002102200080804000E09320007D
:104CE000008040001000780000000100A1002000BA
:104CF000E0072100ACA202000000000000402000FC
:104D000050000700001020004E0007000020200087
:104D10004C000700000420004A00070000082000A3
:104D20004800070040882800D075020000000000FD
:104D300041002000800F2100ACA202000000000012
:104D400021E3A800A0C0B300B09E02000000000054
:104D5000407902000000000011002000903A20007D
:104D6000ACA202000000000090C0B300007A020074
:104D70000000000090C0B300B09E020000000000E0
:104D8000407902000000000011002000903A20004D
:104D9000ACA202000000000090C0B300007A020044
:104DA00000000000C0C0B300B09E02000000000080
:104DB000407902000000000011002000903A20001D
:104DC000ACA202000000000090C0B300007A020014
:104DD00000000000B0C0B300B09E02000000000060
:104DE000407902000000000011002000903A2000ED
:104DF000ACA202000000000090C0B300007A0200E4
:104E00000000000021E3A900004020001C00070072
:104E1000001020001A0007000020200018000700E2
:104E200000042000160007000008200014000700FE
:104E300040882800D0750200000000000080FA00C1
:104E4000000006000200FA00000F78004016800003
:104E50001E0060000000E000040032007092280094
:104E6000A47502000000000003003700A092280093
:104E7000A4750200000000000080FA000000060097
:104E80000200FA00000F7800501680001E0060003B
:104E90000000E00004003200D0922800A475020057
:104EA000000000000300370000932800A4750200F2
:104EB000000000000080FA00000006000200FA0076
:104EC000E06780008000E800F00F200000806000B4
:104ED000E067880024FD07003CFB0700000F780016
:104EE0001E00E00006003400400020009E0F10006D
:104EF00003003C001E00E900904088000D003700D0
:104F00000000EB00F06788002102200040812000B3
:104F100036A30200000000008001EB0042002000E8
:104F20001100200010002000A5FD07000000E9008E
:104F300090408800210120006083200036A30200F9
:104F4000000000000080FA00000006000200FA00E5
:104F5000E06780008000E800F00F20000080600023
:104F6000E067880000FD070018FB07001047980065
:104F70001E4090000004E000090032001E40900036
:104F8000EA4F500006003E001E4090000040E9003D
:104F90008040780000812000014878000F00370031
:104FA0000000EB00F0678800D10820003087200067
:104FB00036A30200000000008001EB00A2002000E8
:104FC00011002000900020007DFD07000040E90056
:104FD0008040780000812000014878000081200096
:104FE00010407800E94F500010003A00DEFC070046
:104FF000F6FA0700004F78001E04E0000B003A00AC
:105000000000EB00F067880030932800D0750200A4
:10501000000000008001EB00F2FF27008000EB00A1
:105020002002200066FD0700004F780041012000AB
:105030000090200036A302000000000011012000B3
:10504000B01F210036A302000000000023C2BF00F1
:10505000614060000004E000FCFF3200008120009D
:1050600010407800E94F500003003A001E407800DD
:105070001E7A0200000000003A9F020000000000BB
:1050800000003700E2790200000000000004E000A8
:10509000FCFF3200EE790200000000008040780042
:1050A00000C2B30080CF500001003200F5FF37008E
:1050B0000080FA00000006000000FA00F171800094
:1050C00060E42000008040009040780030C8B300C9
:1050D00080CF50000E003A00F07180000000E80020
:1050E000F071880003003700F07180000000E800D4
:1050F000F0718800F171800060E4200000804000C1
:105100009040780000CEB30080CF5000F6FF36000C
:105110000080FA00000006000A00FA00300798003C
:105120000000EB0020079800AE00900060E4200033
:10513000008040009040780000CEB30080CF500047
:1051400003003E000080EB0040079800230037007A
:10515000AE00900060E42000008040001040780025
:105160008080FB0000F22F000080400010079800B4
:105170002E0090008000E80060E4200000804000E5
:10518000104078000080FB004801DD002E009000F8
:105190008080E80060E4200000804000104078003B
:1051A0000080FB00000F41009E0078003E00900050
:1051B000808F500003003A002E00900040079800B6
:1051C000060037009E0090002E00900000804000F6
:1051D0006300400020079800D3FF37004E00900086
:1051E0000080FA00000006000600FA00881F780020
:1051F0000000EB00000F7800F171800060E42000F7
:10520000008040009040780080C2B30080CF500002
:1052100010003A00F07180000000E800F071880092
:1052200030010700000F7800F171800060E4200079
:10523000008040009040780090C2B30080CF5000C2
:10524000BD003A00F07180000000E800F0718800B5
:10525000B9003700F171800060E420000080400058
:105260009040780000C4B30080CF50001600360094
:10527000F171800060E420000080400090407800E0
:10528000A0C5B30080CF50000F003E00F271800037
:1052900060E4200000004100104078008080FB00A6
:1052A000F0FB2F000080400080004000E0DD200087
:1052B0000080400010007800200798000200E800FD
:1052C000F07188009E003700F171800060E42000DA
:1052D000008040009040780000C8B30080CF5000AC
:1052E00087003600F171800060E4200000804000FB
:1052F000104078000080FB00100798000100E800D3
:10530000F0718800700920009E009000808F50008E
:105310004A003200700920009E009000808F5000EB
:105320000D003C00400920009E009000808F50003E
:105330001F003200600920009E009000808F500006
:1053400034003200300920009E009000808F500011
:105350002100320059003700A00920009E00900073
:10536000808F50003F003200A00920009E00900076
:10537000808F500005003C00800920009E009000B6
:10538000808F5000460032004C003700B0092000EA
:105390009E009000808F500037003200D00920001E
:1053A0009E009000808F50001600320043003700AE
:1053B000A1408000E00220000088B900EA0040001F
:1053C000E093200000804000100078000000010001
:1053D000000F780058003700A1408000E002200054
:1053E0000088B900E8004000E09320000080400001
:1053F000100478008C00070008000100000F7800FE
:105400004D0037003084020000000000000F7800DB
:1054100049003700A1408000E00220000088B90068
:10542000F4004000E093200000804000100078006D
:1054300000000100000F78003F003700A14080000D
:10544000E00220000088B900F8004000E09320004E
:10545000008040001000780000000100000F78007C
:1054600035003700C2C2BF00614060000080FB0011
:10547000000F780030003700CBC2BF000080FB0077
:105480004300DE00614060000081FB000200780004
:105490000080EA008180EA00000F780026003700D3
:1054A00021E3A800C0C0B300B09E020000000000CD
:1054B000000F780021E3A9001F0037000000EB0077
:1054C000000F78001C0037001E0078006A00B90049
:1054D000000F7800F171800060E42000008040003F
:1054E000104078000080FB009E00400000FD2F006F
:1054F000008F4000F07180000000E800F07188002B
:10550000F171800060E4200000804000904078004D
:10551000F0C2B30080CF500007003600F171800068
:1055200060E42000008040009040780090C3B30009
:1055300080CF5000E4FF36001E007800200798005E
:105540002E0090004F0478000080FA000000060052
:105550000600FA0024FF0700000F78000000370063
:10556000F171800060E420000080400090407800ED
:10557000A0C2B30080CF50000A003200F171800059
:1055800060E420000080400090407800F0C2B3004A
:1055900080CF5000030032001E00780020079800E2
:1055A0001E003700F171800060E4200000804000A0
:1055B000104078000080FB00100798000100E80010
:1055C000F0718800A00220009E009000808F5000A3
:1055D00005003200F00220009E009000808F5000F5
:1055E00007003200DEFF3700FFFE07008000780072
:1055F0001E0078000180B900000F7800D8FF370046
:10560000F9FE0700000178001E0078001100090073
:105610000200D800000F7800D1FF37002E00900064
:105620000080FA00000006000600FA00C8FF07002C
:10563000000F780000003700F171800060E4200066
:105640000080400090407800D0C2B30080CF50006E
:105650000A003200F171800060E420000080400008
:1056600090407800B0C2B30080CF500003003200F9
:105670001E0078002007980017003700F1718000A5
:1056800060E4200000804000104078000080FB00B3
:10569000100798000100E800F0718800B0022000B7
:1056A0009E009000808F500008003200D002200041
:1056B0009E009000808F500001003200DEFF370016
:1056C000A3FF07001E0F1000DBFF3700A0FF07003D
:1056D0001E0F4000D8FF37002E0090000080FA0017
:1056E000000006000C00FA00F271800060E4200067
:1056F00000004100104078008080FB00F0FB2F008C
:105700000080400080004000E0DD2000008040007C
:1057100090007800210798000200E800F0718800EE
:105720000000EB00000F78000B0037009E017800AE
:10573000F271800060E42000000041001040780019
:105740008040780066004700817178000200E80020
:10575000F07188001E0FE800F171800060E4200005
:10576000008040009040780000C4B30080CF50001B
:1057700007003600F171800060E4200000804000E6
:1057800090407800A0C5B30080CF50000E003600D6
:10579000F171800060E420000080400090407800BB
:1057A000F0C2B30080CF5000E0FF3600F1718000FE
:1057B00060E42000008040009040780090C3B30077
:1057C00080CF5000D9FF3E0097FF070010079800D8
:1057D00066004700104078000000FB00500798006A
:1057E000C0032000DE009000808F500032003200A5
:1057F000C0032000DE009000808F500005003C00B8
:1058000010022000DE009000808F50004100320026
:105810004E003700D0032000DE009000808F500043
:1058200005003200E0032000DE009000808F500071
:105830000A003200450037000000EB0040079800E6
:10584000AE0090001E009000808F500041003A0092
:1058500011002000410798003E0037006600470015
:1058600090409000D0C3B30080CF500009003A00B0
:105870000000EB0040079800AE0090001E00900072
:10588000808F500033003500110020004107980040
:10589000300037000000EB0040079800AE00900099
:1058A0001E009000808F50002A003400110020005C
:1058B000410798002700370066004700904090009D
:1058C000D0C3B30080CF500009003A000000EB00C5
:1058D00040079800AE0090001E009000808F50009E
:1058E0001C003C00110020004107980019003700FF
:1058F0000000EB0040079800AE0090001E009000F2
:10590000808F500013003D001100200041079800D7
:10591000100037006600470090409000D0C3B300ED
:1059200080CF500009003A000000EB0040079800CB
:10593000AE0090001E009000808F500005003200E5
:105940001100200041079800020037000000EB0022
:10595000400798004E0090000080FA00000006000A
:105960001C00FA00881F78000000EB00F07188002E
:105970000000EB00300798000000EB0020079800C3
:105980000000EB00100798000000EB000072880098
:105990000000EB00107288000000EB00207288000D
:1059A0000000EB0050079800D04080000080A0006D
:1059B000D04088000000EB00400798000900370045
:1059C0004E00900080004000E0DD2000808040001C
:1059D0000000EB00800878004E0090000000E80016
:1059E000400798004E009000F90F5000F4FF34007B
:1059F000340437001E0090000000E00021003A004F
:105A0000F171800060E42000008040009040780048
:105A1000F0CDB30080CF500003003E0020002000F6
:105A2000300798002A043700F171800060E42000FC
:105A300000804000104078008080FB0000F22F00C2
:105A40000080400060079800F07180008000E8004E
:105A500060E4200000804000104078000080FB00DF
:105A60004801DD00F07180008080E80060E42000E3
:105A700000804000104078000080FB0000007100B2
:105A8000500798000000EB0010079800F0718000AC
:105A9000E300400060E420000080400010407800F7
:105AA0000080FB006101B90000F82F00F1FF2F001A
:105AB0000201400083814800420F9800530F980074
:105AC00010022000010020004E099000DE09900025
:105AD000800F5100818F5900EE033E004E08900068
:105AE000DE0890000060010021003700350037001B
:105AF000E8033700E7033700710037008100370003
:105B0000A3003700B7003700BE0037003B01370065
:105B100088013700DF033700EE0137003502370018
:105B200099023700AF0237009F023700CB023700DF
:105B3000BB023700D8023700D6033700780337009E
:105B40005C033700D3033700D2033700000337006C
:105B5000F00237009F033700AD033700DE02370045
:105B60001203370032033700B5033700C60337008E
:105B70001000200020079800F071800066004000AF
:105B8000F0718800F07180008080E90060E42000FE
:105B900000804000104078008080FB00F0FB2F0068
:105BA00000844000A0FE0700000178008800440047
:105BB000E0DD200000804000020878003EFD070084
:105BC000B60337001000200020079800F071800015
:105BD00064004000F0718800C2FE07000000E00091
:105BE0001C003200F1718000310F980060E4200049
:105BF0003E09900000004100904078008041EB0099
:105C00004357980020C8B30080CF500002003A00EC
:105C100010C0B30040579800BE0890000100E80093
:105C2000F07188004E5190000204E0009B033200A6
:105C30001000200010079800F071800063005000F1
:105C4000F071880095033700F07180000000E800D3
:105C5000F0718800F171800060E420000080400055
:105C60009040780030C8B30080CF50000700320069
:105C7000F171800060E420000080400090407800D6
:105C800000CEB30080CF5000EFFF3600F1718000EE
:105C900060E42000008040009040780030C8B300ED
:105CA00080CF50007D033A001000200010079800BC
:105CB000F07180000080E900F07188007703370000
:105CC0001000200020079800F07180006400400060
:105CD000F071880054FE07000FFD0700000F7800E8
:105CE0008081EB009E8F1100030032001E007800BF
:105CF000F0718800690337006000200030079800C9
:105D0000660337001000200020079800F071800023
:105D100064004000F071880010728000E90F5000AC
:105D200018003C0012728000F17180006E0090003B
:105D3000008040008001E9008200410020E1200055
:105D40000080400003087800107280000000E80026
:105D50001072880034FE0700EFFC0700000F780087
:105D60008080EB009E8F1000030032001E0178003F
:105D7000F271880049033700600020003007980066
:105D800046033700700020003007980043033700B7
:105D900080962800A475020000000000100020007A
:105DA00020079800107280000000E0000A00320016
:105DB000107280000000E9001072880010728000EC
:105DC0008000400020E120000080400010007800AA
:105DD000F071880031033700800020003007980000
:105DE0002E0337001000200020079800F17180007A
:105DF0006E0090000080400063004000F071880059
:105E0000260337001000200020079800F071800062
:105E100064004000F071880057003700F171800085
:105E200060E42000008040009040780020C2B30071
:105E300080CF50001F003A00F07180000000E800A1
:105E4000F071880010003700D04080000080A10071
:105E5000D0408800F171800060E4200000804000A4
:105E600010407800004178000100E800F0718800DF
:105E700002407800007A020000000000D04080005C
:105E80000080A000D0408800F171800060E4200014
:105E9000008040009040780020C2B30080CF5000C6
:105EA000E9FF3A00F07180000000E800F07188001E
:105EB00031003700F171800060E420000080400074
:105EC0009040780000C4B30080CF50000700360037
:105ED000F171800060E42000008040009040780074
:105EE000A0C5B30080CF50000D003600F1718000D6
:105EF00060E4200000804000104078000004E000D2
:105F000013003D00F171800060E42000008040003B
:105F100090407800F0CDB30080CF50000C003E00E0
:105F2000C1FD0700000F7800D04080000080A10074
:105F3000D04088001E007800DE77020000000000DC
:105F4000D04080000080A000D04088000A003700C8
:105F5000F171800060E420000080400090407800F3
:105F6000B0C3B30080CF500003003A00F07180004E
:105F70000000E800F0718800F171800060E420000A
:105F80000080400090407800F0CDB30080CF5000FA
:105F900007003E00F171800060E4200000804000B6
:105FA0009040780030C8B30080CF50009BFF3A008B
:105FB000F07180008000E90060E420000080400073
:105FC00090407800B0C3B30080CF50000900320089
:105FD000D04080000080A100D0408800E09F2800D1
:105FE000D075020000000000D04080000080A000BA
:105FF000D040880030FC0700A802370010002000C5
:1060000020079800D04080000080A100D040880088
:10601000F071800064004000F0718800F171800030
:1060200060E42000008040009040780020C2B3006F
:1060300080CF500018003A00F07180000000E800A6
:10604000F07188000A003700F171800060E42000E0
:106050000080400010407800004178000100E80016
:10606000F071880002407800007A02000000000011
:10607000F171800060E420000080400090407800D2
:1060800020C2B30080CF5000EFFF3A00F0718000D3
:106090000000E800F0718800F171800060E42000E9
:1060A0000080400090407800C0C2B30080CF500014
:1060B00004003A00F07180000000E800F0718800F0
:1060C000020037003000200030079800F171800096
:1060D00060E4200000804000104078008080FB00D9
:1060E000F0FB2F00008440008001EB00F2FF27004E
:1060F0008000EB000000EB00E02202000000000046
:106100000001780088004400E0DD200000804000AD
:1061100002087800F07180000000E800F07188004B
:10612000E5FB0700D04080000080A000D040880040
:106130005A0237001000200020079800F0718000FC
:1061400064004000F071880000728000E30F50008E
:1061500004003C00007280000000E800007288002B
:1061600002003700400020003007980002728000D3
:10617000F371800060E4200000804100104078004E
:106180008080FB0000FC2F00008240006610B900F8
:106190008080E80060E22000008040000408780071
:1061A0000300E800F0718800F171800060E42000D5
:1061B0000080400090407800D0C3B30080CF5000F2
:1061C00011003A00F07180000000E800F0718800D2
:1061D000007280006600B9008080E80060E2200064
:1061E00000804000100078000004E9000EFD070068
:1061F0000001780088004400E0DD200000804000BD
:1062000002087800020037003000200030079800B4
:10621000F3718000130F980060E420009E08900046
:1062200000804000904078000041EB000257980049
:10623000B0C8B30080CF500002003A0013C0B300D2
:10624000035798009E0890000100E800F071880054
:106250000E5190000204E000090032000872800034
:10626000F1FC0700000178006640B900E40040003E
:1062700060E2200000804000020878000200370041
:106280003000200030079800F171800060E42000A9
:106290000080400090407800F0CDB30080CF5000E7
:1062A0000800360000728000F27180006600B900BC
:1062B0008000780060E22000008040000208780042
:1062C0000200370030002000300798007AFB0700FA
:1062D000F20137001000200020079800F0718000C4
:1062E00064004000F0718800F271800060E42000DA
:1062F00000004100104078008080FB0000FC2F006F
:10630000008F40000200E800F0718800500020007B
:10631000300798000000EB00400798002F0037007E
:106320004E0090006600B9008080E80060E2200026
:1063300000804000100078009E0F500024003A00BA
:106340001E00E90080004000E0DD200000804000E9
:10635000100178004E0090006600B900E400400093
:1063600060E220000080400010007800800F5100A3
:1063700012003D009E00E90001814000E0DD2000A8
:1063800000004100100078000001E800818040001A
:10639000E0DD200000804000020878004E00900000
:1063A0006600B9008000780060E2200000804000B4
:1063B00010007800F0718800030037000072800040
:1063C0000000E900007288000000EB003007980030
:1063D0004E0090000000E800400798000172800025
:1063E0004E009000810F5000CDFF340032FB0700BB
:1063F000AA0137001000200020079800F0718000EB
:1064000064004000F0718800207280000000E0000D
:1064100027003A000000EB00400798000A00370010
:10642000CE00900060E42000008040001040780022
:106430008080FB004E0090008080400030F22F00F2
:1064400000804000400798004E009000E3004000AC
:1064500060E420000080400090407800E0C8B30075
:1064600080CF500006003200CE00900060E4200093
:1064700000804000104078000004E000E8FF3A008F
:10648000CE00900060E420000080400010407800C2
:106490000004E000040032004E0090006400400060
:1064A000207288000200370090002000300798001A
:1064B000F3718000030F780020728000F071880073
:1064C0009E00780060E420000080400010407800CA
:1064D0008080FB00F0FB2F000084400042FB07009F
:1064E0000001780088004400E0DD200000804000CA
:1064F00002087800F0718000207288001E00E80019
:10650000F07188002172800060E42000008040006B
:1065100090407800C0C2B30080CF500003003A0022
:10652000207280000000E800207288002172800044
:1065300060E42000008040009040780000CEB3006E
:1065400080CF50000E00360020728000E300400033
:1065500060E420000080400090407800E0C8B30074
:1065600080CF5000030032000000EB002072880052
:106570000300370020728000640040002072880011
:10658000CDFA0700450137001000200020079800D1
:10659000F17180006E0090000080400063004000B8
:1065A000F07188003D01370010002000200798009E
:1065B000F071800064004000F0718800A14080000C
:1065C000E00220000088B90080007800E0932000FD
:1065D000008040001000780000000100B6FA0700BB
:1065E0002E0137001000200020079800F071800075
:1065F00064004000F0718800A1408000E0022000AB
:106600000088B9008080E800E0932000008040000E
:106610001000780000000100A7FA07001F013700F2
:106620001000200020079800F071800064004000F6
:10663000F0718800A1408000E00220000088B900CD
:10664000E4004000E093200000804000100078004B
:106650000000010098FA0700100137001000200028
:1066600020079800F071800064004000F0718800FD
:10667000A1408000E00220000088B900E600400050
:10668000E09320000080400010007800000001002E
:1066900089FA070001013700100020002007980048
:1066A000F071800064004000F0718800A14080001B
:1066B000E00220000088B900E8004000E0932000DC
:1066C0000080400010047800D7FB0700080001009C
:1066D00079FA0700F1003700100020002007980029
:1066E000F071800064004000F0718800CEFB07006C
:1066F0000000E00003003200EC8302000000000014
:10670000020037000E840200000000006AFA070051
:10671000E20037001000200020079800F071800090
:1067200064004000F0718800BFFB07000000E0003B
:1067300003003200C002A900C202A8000200370014
:10674000C002A900C202A9005BFA0700D30037000B
:106750001000200020079800F071800064004000C5
:10676000F0718800B0FB07000000E0000700320075
:10677000C0B52000104078000000A0000010A1006B
:10678000C1B520008048780006003700C0B5200061
:10679000104078000000A0000010A100C1B520004A
:1067A0008048780044FA0700BC0037001000200041
:1067B00020079800F071800064004000F0718800AC
:1067C00099FB0700B05F8800B05F80000000E00028
:1067D00002003D000000EB00B05F8800B15F800068
:1067E00000FA2000808F50000200340000FA2000E0
:1067F000B05F8800C05F8000E10F500002003C00E5
:1068000020002000C05F8800C15F800030062000AB
:10681000808F50000200340030062000C05F8800E6
:10682000968002000000000023FA07009B0037005A
:106830001000200020079800F071800064004000E4
:10684000F071880078FB0700C05F8800B05F8000AF
:106850000000E00002003D000000EB00B05F880097
:10686000B15F800000FA2000808F500002003400E9
:1068700000FA2000B05F8800C05F8000E10F500088
:1068800002003C0020002000C05F8800C15F800043
:1068900030062000808F50000200340030062000B7
:1068A000C05F8800968002000000000002FA070026
:1068B0007A0037001000200020079800F071800057
:1068C00064004000F071880057FB07000000E00002
:1068D00009003200A1408000E00220000088B900D9
:1068E000F0004000E093200000804000100078009D
:1068F0000000010008003700A1408000E0022000F5
:106900000088B900F2004000E093200000804000C1
:106910001000780000000100E7F907005F00370071
:106920001000200020079800F071800064004000F3
:10693000F07188003CFB0700700798007E00900013
:10694000E10F500010003200FE009000E28F500076
:10695000160032007E0190000200E00001003200CB
:106960001A003700A1408000E00220000088B90032
:10697000EE004000E093200000804000100078000E
:106980000000010011003700A1408000E00220005B
:106990000088B900EC004000E09320000080400037
:1069A000100078000000010008003700A1408000BE
:1069B000E00220000088B900F6004000E0932000CB
:1069C000008040001000780000000100BAF90700C4
:1069D000320037001000200020079800F07180007E
:1069E00064004000F07188000FFB07000000E00029
:1069F00003003200C962A800CB62A9000200370080
:106A0000CB62A900C962A900ABF9070023003700D7
:106A10001000200020079800F07180006400400002
:106A2000F071880000FB0700000F78001E0078005E
:106A30000EA00200000000009FF9070017003700B9
:106A40001000200020079800F071800064004000D2
:106A5000F0718800F4FA0700000F7800A140800070
:106A6000E00220000088B900FC004000E093200014
:106A700000804000900078001E00780001000100B6
:106A80008DF907000500370010002000300798003E
:106A90000200370030002000300798002E009000E0
:106AA0000000E00005003A00F17180006E009000E7
:106AB0000080400063004000F07188000000EB009F
:106AC000200798003E0090000000E000C9FB320063
:106AD000D04080000080A100D04088003E0090009F
:106AE000E10F50001800320061002000A03A2000A1
:106AF000ACA20200000000003E009000DE77020021
:106B00000000000081002000003B2000ACA2020039
:106B1000000000005E009000DE7702000000000030
:106B2000B1002000803B2000ACA202000000000069
:106B3000F0718000DE77020000000000E09F280076
:106B4000D0750200000000004F0478000080FA00B9
:106B5000000006000200FA00000F780000C2B30037
:106B6000007A0200000000001E007800A4750200F8
:106B70000000000000C2B300007A02000000000024
:106B80000080FA00000006000400FA000000EB009C
:106B9000F07188003F003700F171800060E4200050
:106BA0000080400090407800214798002E409000DF
:106BB0000004E000040035002E409000007A02003E
:106BC0000000000030003700AE40900000CEB3005F
:106BD00080CF50001C003600E09F2800D0750200D6
:106BE00000000000F07180008000E80060E42000F8
:106BF00000804000104078000080FB004801DD006C
:106C0000F07180008080E80060E420000080400097
:106C1000104078000080FB0000004100000F780069
:106C2000F07180000080E800F07188001E0078009C
:106C3000DE7702000000000000C2B300007A02000C
:106C4000000000001000370000C2B300007A02000C
:106C5000000000002E4090008080FB0000F82F0014
:106C6000008040008000400040B0200000804000D4
:106C700010007800A47502000000000000C2B300FC
:106C8000007A020000000000F07180000000E800BF
:106C9000F0718800F171800060E420000080400005
:106CA000104078000004E000BBFF3A00E09F28009D
:106CB000D075020000000000F07180000000E900C3
:106CC000DE7702000000000071002000303C200050
:106CD00036A30200000000000080FA000000060059
:106CE0000600FA0010079800E0678000000F7800A7
:106CF000150037001E00900010417800E167800009
:106D0000A0BF20000080400010407800804F51005C
:106D1000050032001E007800E06788000000EB00EC
:106D2000200798000E003700E06780008000E80030
:106D3000F00F200000806000E06788001E009000D7
:106D40000000E800100798001E0090001040780036
:106D50000004E000E7FF3A00100020002007980040
:106D60002E0090000080FA00000006000400FA00E7
:106D70000000EB00000F7800100037001E007800C4
:106D80008000400040B020000080400010007800EB
:106D9000D3FF07000000E000070032001E0078006B
:106DA0008040780000C8B30000C040000080FB00B5
:106DB00010079800060037001E0FE80010022000A0
:106DC0009E0F1000EDFF34000000EB00100798004C
:106DD0001E0090000080FA00000006003600FA0055
:106DE000E0678000000F98001F0037008E089000B9
:106DF000A0BF2000008040009040780000C6B30093
:106E000080CF5000110034008E089000A0BF2000F9
:106E10000080400090407800A0C7B30080CF5000B1
:106E20000A003C000E0990008E089000A0BF2000D0
:106E30000080400090407800F0CDB30080C060003A
:106E4000A0BF200000004100014878000E0890001B
:106E50000000E800000F98008E089000F00F20005E
:106E600000806000000F98008E089000D0678000BE
:106E7000808F5000DDFF3A000000EB00000F98000B
:106E8000E1678000A0BF20000080400090407800B3
:106E9000F0C2B30080CF50002D013400E1678000C4
:106EA000A0BF2000008040009040780090C3B30055
:106EB00080CF500026013C000000EB00000F98003E
:106EC000070037000E099000F20047000040EB0079
:106ED00000F178000E0890000000E800000F980014
:106EE0008E08900020022000808F5000F5FF3400B3
:106EF000E61D020000000000600798006E00900090
:106F00004880DE0080407800720047001140980001
:106F10006E0090008040780000C0EB0080C06000F0
:106F200072004700214098006E0090007AF8070038
:106F3000500798005E009000E10F40002B003200E7
:106F4000DE00900060E420000080400010407800E7
:106F50008080FB0030F22F00008040003007980056
:106F60005E009000000F98000D0037000E099000A1
:106F70008E0890003E0090008080400060E4200079
:106F8000008040009040780060E420000000410054
:106F9000014878000E0890000000E800000F9800FB
:106FA000014020003E009000808050000E089000BC
:106FB000808F5000EDFF3C00080037008E089000E5
:106FC00060E42000808040000040EB0080487800B2
:106FD0000E0890000000E800000F98008E08900056
:106FE000F03F2000808F5000F4FF3400300020007C
:106FF000000F98000000EB0020079800B421020069
:1070000000000000430037002E0090000000E00068
:1070100002003A00B4210200000000002E0090009F
:107020000000E00004003A0050FF07000080FB0071
:1070300060079800020037000000EB00600798002E
:107040006E0090009E780200000000006E0090002C
:107050000000E0000C0032000E0990006E0090006D
:10706000804078007200470001717800EE009000C7
:1070700070082000808F50001A003A001000200095
:107080002007980017003700E1678000A0BF2000AC
:10709000008040009040780020C2B30080CF5000B4
:1070A00003003A002E0090000000A2002007980084
:1070B0000E099000E1678000A0BF20000080400022
:1070C000104078008040780072004700017178001D
:1070D000E06780008000E800F00F20000080600082
:1070E000E06788000E0890000000E800000F98009C
:1070F0008E08900030022000808F50000500340080
:1071000091002000A03C200036A3020000000000F7
:10711000D4003700E1678000D0678000808F500086
:10712000B9FF3A000E089000E30F5000CD00320086
:107130000E089000E40F5000CA0032000E089000C4
:1071400080407800C0CDB30000C04000804078008F
:1071500072004700014878000000EB00000F980023
:107160000000EB00400798000000EB00500798007B
:10717000460037008E08900060E420000080400048
:107180009040780000CEB30080CF50002E00360033
:107190008E08900060E420000080400010407800DD
:1071A0008080FB0000F22F00008040003007980034
:1071B0000E0890008000E80060E42000008040009D
:1071C000104078000080FB004801DD000E089000B0
:1071D0008080E80060E420000080400010407800DB
:1071E0000080FB000000410010079800720047007B
:1071F000104090000080FB00C800DD0072004700D6
:10720000204090000080FB0000804000000F7800CC
:107210001E0090009E0F5000050031008E08900067
:107220003E0090000080400063004000500798003E
:10723000BE0090000E0890000080400063004000F7
:10724000000F9800020037000E08900040079800D9
:107250000E0890008000E80060E4200000804000FC
:10726000104078000080FB004801DD000E0890000F
:107270008080E80060E4200000804000104078003A
:107280000080FB0000004100600798004E00900065
:107290000000E000B7FF32007200470010407800A5
:1072A0008080FB0030F22F000080400060079800D3
:1072B0004E009000000F98000D0037008E089000DF
:1072C0006E009000008140008E08900060E4200075
:1072D000008040009040780060E420000000410001
:1072E000014878000E0890000000E900000F9800A7
:1072F0008E0890005E009000808F5000EFFF3D00F0
:107300000000EB00000F98000C003700DE0090003A
:107310000E089000008140008E0890007200470027
:10732000E140780060E4200000004100014878005E
:107330000E0890000000E800000F98008E089000F2
:107340006E009000808F5000F0FF35004500370040
:10735000F09F280062FE07000000E00005003200F8
:107360007FF90700E09F2800D075020000000000B0
:107370003C00370030A0280059FE07000000E00064
:107380000200320000FE07003600370080A028000F
:1073900053FE07000000E00004003200D0408000EF
:1073A0000090A100D04088002E003700D0A0280017
:1073B0004BFE07000000E000200032000000EB0060
:1073C000000F9800180037000000EB0070079800CD
:1073D0000F0037008E0890007E00900080804000F3
:1073E00060E4200000804000104078000080FB0036
:1073F0009E7802000000000000C2B300007A020084
:10740000000000007E0090000000E8007007980077
:107410007E009000EF0F5000EEFF34000E08900049
:1074200070004000000F98008E089000F03F200090
:10743000808F5000E4FF34000A00370030A128009C
:1074400027FE07000000E0000200320007000700EE
:1074500004003700C1002000303D200036A30200A8
:10746000000000000080FA00000006000200FA00A0
:107470000000EB00000F7800060037009E00780047
:1074800060E42000808040000040EB0080487800ED
:107490001E0FE800F03F20009E0F1000F7FF3400A1
:1074A00011CEB30060E420000148780080C0EB00FA
:1074B00070E420000148780080C0EB0080E42000E8
:1074C0000148780011CAB30090E420000148780018
:1074D0000080FA0000000600575249005445200081
:1074E000424954003A2020002A6E6500787420003A
:1074F000636C6F00636B2000285E290020776900B1
:107500006C6C20007573650020746800697320003E
:1075100076616C0075653100574952004520720054
:107520006F757400696E6500732028004329200080
:107530003230300030204D006963680061656C00B6
:107540002050650061726300652047004E552000A1
:1075500047504C004E6F20006465760069636500FB
:107560002C2074007279200028414C0041524D00BB
:107570002920530045415200434820006D616300BB
:10758000726F2000666972007374410044445200B7
:1075900045535300204D410043524F0020203000FE
:1075A0002E4D610063726F00206D65006E754D0099
:1075B000616372006F2020002020200031574900B5
:1075C000524520006164640072657300730D0A0007
:1075D000202020002A3157004952450020524F00F8
:1075E0004D2043004F4D4D00414E4400204D410081
:1075F00043524F00733A0D000A203500312E5200DD
:107600004541440020524F004D202800307833007F
:10761000332920002A666F0072207300696E6700AC
:107620006C65200064657600696365002062750002
:10763000730D0A00203835002E4D41005443480098
:1076400020524F004D202800307835003529200089
:107650002A666F006C6C6F007765640020627900A9
:107660002036340062697400206164006472650031
:1076700073730D000A20320030342E00534B490042
:10768000502052004F4D20002830780043432900FD
:10769000202A66006F6C6C006F77650064206200C2
:1076A000792063006F6D6D00616E64000D0A20002B
:1076B000323336002E414C0041524D0020534500DC
:1076C00041524300482028003078450043290D00EE
:1076D0000A20320034302E00534541005243480006
:1076E00020524F004D2028003078460030294100BC
:1076F0004C4152004D205300454152004348200068
:107700002830780045432900534541005243480042
:1077100020283000784630002944650076696300EF
:107720006520490044732000617265002061760085
:1077300061696C0061626C006520620079204D0017
:10774000414352004F2C2000736565002028300013
:10775000292E52004541440020524F004D20280060
:107760003078330033293A00204D4100544348001B
:1077700020524F004D202800307835003529530025
:107780004B49500020524F004D20280030784300D4
:10779000432955006E6B6E006F776E00206D61009F
:1077A00063726F002C207400727920003F206F00FC
:1077B0007220280030292000666F72002068650062
:1077C0006C70420055532000524553004554200030
:1077D000576172006E696E00673A20002A53680094
:1077E0006F727400206F7200206E6F002070750041
:1077F0006C6C2D00757020002A4E6F0020646500AF
:1078000076696300652064006574650063746500D3
:10781000642044005331380053323000204869005E
:10782000676820005072650073204400696720007B
:1078300054686500726D44005331380042323000A4
:10784000205072006F672000526573002044690069
:1078500067205400686572006D445300313832006F
:1078600032204500636F6E00204469006720540099
:10787000686572006D445300323430003420450096
:10788000636F6E0072616D00207469006D65200089
:1078900043686900704453003234330031203100B2
:1078A0004B204500455052004F4D55006E6B6E0009
:1078B0006F776E002064650076696300655057003D
:1078C0004D20640069736100626C650064314B0097
:1078D000487A2D00342C300030304B00487A20009C
:1078E00050574D0046726500717565006E637900F2
:1078F00020696E00204B48007A20500072657300AA
:1079000063616C00653A500052323A00447574006D
:107910007920630079636C00652069006E20250082
:10792000205057004D206100637469007665450062
:1079300052524F00523A200050574D0020616300D0
:1079400074697600652C2000672074006F20640045
:1079500069736100626C65004155580020467200F1
:1079600065717500656E6300793A200041555800D5
:1079700020494E00505554002F4849002D5A4100CF
:1079800055582000484947004841550058204C00B0
:107990004F5756004F4C54004D455400455220005F
:1079A0004D4F440045564F004C5441004745200080
:1079B00050524F0042453A002056450072726F0007
:1079C0007228290020406C00696E65003A20400052
:1079D00070676D007370610063653A002062790022
:1079E000746573002E546F006F206C006F6E67001B
:1079F000215379006E7461007820650072726F0007
:107A0000724E6F002045450050524F004D457200A8
:107A1000617369006E6764006F6E65005361760084
:107A2000696E670020746F0020736C006F74200013
:107A3000496E7600616C6900642073006C6F74009D
:107A40004C6F610064696E0067206600726F6D00A4
:107A500020736C006F742000455252004F523A0060
:107A600020636F006D6D61006E64200068617300BB
:107A7000206E6F00206566006665630074206800F4
:107A80006572650041434B004E4143004B49320053
:107A900043205300544152005420420049544900AD
:107AA0003243200053544F005020420049544900B3
:107AB000324320006D6F6400653A0D000A203100EA
:107AC0002E2053006F66740077617200650D0A0006
:107AD00020322E00204861007264770061726500D8
:107AE0005365740020737000656564003A0D0A00E8
:107AF00020312E00207E35004B487A000D0A2000F0
:107B0000322E20007E3530004B487A000D0A2000CE
:107B1000332E20007E313000304B48007A0D0A00B1
:107B200020342E00207E340030304B00487A57003D
:107B300041524E00494E47003A204800415244000D
:107B4000574152004520490032432000697320000C
:107B500062726F006B656E00206F6E0020746800AB
:107B600069732000504943002120280052455600E7
:107B7000204133002953650074207300706565004F
:107B8000643A0D000A2031002E20310030304B00C5
:107B9000487A0D000A2032002E20340030304B008D
:107BA000487A0D000A2033002E2031004D487A001B
:107BB0004932430020286D006F6420007370640018
:107BC000293D2800202030002E4D610063726F0097
:107BD000206D65006E750D000A2031002E376200A1
:107BE000697420006164640072657300732073001F
:107BF0006561720063680D000A2032002E49320070
:107C0000432073006E69660066657200536561000B
:107C100072636800696E670020493200432061008A
:107C200064647200657373002073700061636500A3
:107C30002E2046006F756E00642064006576690032
:107C400063657300206174003A536E0069666600D4
:107C50006572280042415300494329005265610082
:107C6000647961002F412F00402063006F6E740023
:107C7000726F6C00732041005558200070696E00CF
:107C8000612F41002F402000636F6E0074726F00FF
:107C90006C7320004353200070696E00436F6D00C9
:107CA0006D616E0064206E006F7420007573650056
:107CB000642069006E20740068697300206D6F0095
:107CC00064655000756C6C002D7570002072650045
:107CD00073697300746F720073204F004646500042
:107CE000756C6C002D7570002072650073697300EF
:107CF000746F720073204F004E5365006C662D0048
:107D000074657300742069006E204800695A200071
:107D10006D6F640065206F006E6C790052455300F2
:107D2000455442004F4F54004C4F410044455200CF
:107D30004155580020494E00505554002F484900E5
:107D40002D5A2C002052450041443A0020506F002B
:107D5000776572002073750070706C006965730040
:107D6000204F4E00506F77006572200073757000D1
:107D7000706C6900657320004F4646004441540012
:107D80004120530054415400453A200044454C00E2
:107D9000415920007573570052495400453A20005C
:107DA00052454100443A2000434C4F00434B2C00C5
:107DB000203143004C4F43004B2C20003044410005
:107DC000544120004F555400505554002C20310090
:107DD0004441540041204F005554500055542C004C
:107DE000203020002A7069006E20690073206E0028
:107DF0006F77200048695A00434C4F00434B2000E6
:107E0000544943004B533A0020524500414420005E
:107E1000424954003A205300796E74006178200082
:107E2000657272006F7220006174200063686100E7
:107E3000722078002E206500786974002877690028
:107E400074686F0075742000636861006E67650078
:107E5000296E6F00206D6F0064652000636861000B
:107E60006E6765004E6F6E0065786900737465001B
:107E70006E74200070726F00746F63006F6C21006D
:107E8000782E200065786900740D0A00496E76002E
:107E9000616C690064206300686F690063652C0091
:107EA0002074720079206100676169006E444500AA
:107EB000564944003A68740074703A002F2F6400E9
:107EC000616E670065726F0075737000726F740089
:107ED0006F747900706573002E636F006D2A2D003A
:107EE0002D2D2D002D2D2D002D2D2D002A4F700014
:107EF000656E200064726100696E20006F75740009
:107F00007075740073202800483D4800692D5A00A0
:107F10002C204C003D474E0044294E006F726D00EE
:107F2000616C20006F7574007075740073202800F8
:107F3000483D33002E3376002C204C003D474E0048
:107F400044294D0053422000736574003A204D00CF
:107F50004F53540020736900672062006974200049
:107F60006669720073744C0053422000736574009C
:107F70003A204C00454153005420730069672000AB
:107F800062697400206669007273740020426F0099
:107F90006F746C006F6164006572200076203100A0
:107FA0002E20480045580D000A2032002E204400A3
:107FB00045430D000A2033002E204200494E0D009B
:107FC0000A2034002E20520041574400697370008B
:107FD0006C61790020666F00726D6100742073001F
:107FE000657456006F6C740061676500206D6F00EA
:107FF0006E6974006F7273003A203500563A2000A3
:10800000207C2000332E3300563A2000207C2000B4
:10801000565055004C4C5500503A200053657400A2
:1080200020736500726961006C2070006F727400CB
:1080300020737000656564003A2028006270730048
:10804000290D0A0020312E0020333000300D0A00A7
:1080500020322E002031320030300D000A20330053
:108060002E203200343030000D0A2000342E200043
:1080700034383000300D0A0020352E00203936000B
:1080800030300D000A2036002E2031003932300009
:10809000300D0A0020372E002033380034303000F5
:1080A0000D0A2000382E20003537360030300D0004
:1080B0000A2039002E2031003135320030300D00D9
:1080C0000A3130002E2042005247200072617700B2
:1080D000207661006C75650041646A0075737400F8
:1080E00020796F0075722000746572006D696E00F2
:1080F000616C410072652000796F75002073750016
:1081000072653F002043460047313A002043460055
:1081100047323A00285C2D002F5F5C002D29280093
:108120005C5F2F002D295300656C6500637420008F
:108130006F757400707574002074790070653A0072
:108140000D0A2000312E20004F7065006E20640063
:10815000726169006E202800483D4800692D5A0070
:108160002C204C003D474E0044290D000A203200CF
:108170002E204E006F726D00616C200028483D007B
:10818000332E3300562C20004C3D47004E4429002E
:1081900052325700202873007064200068697A000A
:1081A000293D2800202030002E4D610063726F00B1
:1081B000206D65006E750D000A2031002E495300B8
:1081C0004F37380031362D003320410054520D0016
:1081D0000A2032002E4953004F37380031362D0027
:1081E000332070006172730065206F006E6C79003F
:1081F00049534F002037380031362D0033204100DD
:10820000545220002852450053455400206F6E0000
:1082100020435300290D0A005245530045542000C5
:1082200048494700482C2000434C4F00434B200056
:10823000544943004B2C2000524553004554200024
:108240004C4F570049534F002037380031362D002E
:108250003320720065706C0079202800757365000A
:108260007320630075727200656E7400204C5300B9
:108270004220730065747400696E6700293A20001B
:1082800050726F00746F63006F6C3A00207365006A
:10829000726961006C3320007769720065322000DA
:1082A000776972006552460055756E006B6E6F00FF
:1082B000776E5200656164002074790070653A0041
:1082C00020746F0020656E00647661007269610041
:1082D000626C6500206C65006E6774006844610024
:1082E00074612000756E690074733A00206E6F002F
:1082F00020696E0064696300617469006F6E4400F8
:108300006174610020756E00697420006C656E00F8
:10831000677468002028620069747300293A20009D
:1083200043532000454E4100424C45004443530016
:1083300020444900534142004C4544005233570009
:10834000202873007064200063736C00206869004B
:108350007A293D00282029000D0A44006973630032
:108360006F6E6E006563740020616E00792064009A
:1083700065766900636573000D0A43006F6E6E00D9
:10838000656374002028560070752000746F20000B
:108390002B355600292061006E64200028414400DE
:1083A000432074006F202B00332E330056294300E6
:1083B00074726C00415558004D4F440045204C00EC
:1083C00045445000554C4C00555020004850550035
:1083D0004C4C55005020480056524500474144003F
:1083E000432061006E64200073757000706C79002A
:1083F00035565600505533002E3356004144430045
:108400004275730020686900676842007573200038
:1084100048692D005A2030004275730020486900D9
:108420002D5A2000314D4F0044452000616E6400FC
:1084300020565200454720004C45440073207300ED
:10844000686F75006C642000626520006F6E21000B
:10845000466F75006E64200020657200726F7200B6
:10846000732E4D004F534900434C4B004D49530070
:108470004F435300204F4B0020464100494C5300CE
:10848000657420007370650065643A000D0A200071
:10849000312E200033304B00487A0D000A20320084
:1084A0002E20310032354B00487A0D000A2033006F
:1084B0002E20320035304B00487A0D000A2034005F
:1084C0002E2031004D487A00436C6F00636B200012
:1084D000706F6C006172690074793A000D0A2000B7
:1084E000312E200049646C0065206C006F772000FD
:1084F0002A646500666175006C740D000A20320004
:108500002E204900646C65002068690067684F0090
:108510007574700075742000636C6F00636B2000CD
:1085200065646700653A0D000A2031002E2049007D
:10853000646C650020746F002061630074697600CC
:10854000650D0A0020322E00204163007469760018
:10855000652074006F206900646C6500202A640047
:1085600065666100756C7400496E7000757420005A
:1085700073616D00706C6500207068006173650048
:108580003A0D0A0020312E00204D690064646C0011
:1085900065202A006465660061756C00740D0A0030
:1085A00020322E0020456E006453500049202800E0
:1085B0007370640020636B00702073006B65200093
:1085C000736D7000206373006C206800697A290065
:1085D0003D28200020302E004D616300726F200086
:1085E0006D656E00750D0A0020312E00536E690016
:1085F00066662000435320006C6F77000D0A200050
:10860000322E53006E696600662061006C6C20009B
:108610007472610066666900632D7000202D66002B
:10862000202A42007974650073206400726F700024
:10863000706564002A464100494C4500442C2000E6
:108640004E4F2000444154004144610074612000B9
:1086500062697400732061006E64200070617200B2
:10866000697479003A0D0A0020312E0020382C0060
:10867000204E4F004E4520002A646500666175005B
:108680006C7420000D0A2000322E2000382C2000AF
:10869000455645004E200D000A2033002E2038009C
:1086A0002C204F00444420000D0A2000342E2000CE
:1086B000392C20004E4F4E00455374006F7020003F
:1086C00062697400733A0D000A2031002E203100D7
:1086D000202A640065666100756C74000D0A200034
:1086E000322E2000325265006365690076652000F5
:1086F000706F6C006172690074793A000D0A200095
:10870000312E200049646C0065203100202A64006D
:1087100065666100756C74000D0A2000322E200021
:1087200049646C00652030005541520054202800F7
:108730007370640020627200672064006270200021
:108740007362200072787000206869007A293D0009
:1087500028202000302E4D00616372006F206D00D4
:10876000656E75000D0A2000312E540072616E0096
:108770007370610072656E0074206200726964003B
:1087800067650D000A2032002E204C0069766500D6
:10879000206D6F006E6974006F720D000A20330047
:1087A0002E42720069646700652077006974680072
:1087B00020666C006F772000636F6E0074726F002C
:1087C0006C55410052542000627269006467650074
:1087D0005265730065742000746F2000657869002D
:1087E00074526100772055004152540020696E0098
:1087F000707574005541520054204C004956450094
:108800002044490053504C0041592C00207D200049
:10881000544F200053544F00504C490056452000FF
:1088200044495300504C410059205300544F5000CC
:1088300050454400574152004E494E00473A2000EF
:1088400070696E0073206E006F7420006F70650099
:108850006E206400726169006E20280048695A0029
:108860002920520045564900443A0D000A496E003D
:1088700076616C006964200063686F00696365005D
:108880002C2074007279200061676100696E6D00B0
:1088900073525300204C4F00572C2000434F4D0083
:1088A0004D414E0044204D004F444500525320009E
:1088B00048494700482C20004441540041204D00C5
:1088C0004F444500416464007265730073206F007B
:1088D0006620500043463800353734003F54680066
:1088E000697320006D6F640065207200657175000A
:1088F00069726500732061006E2061006461700020
:10890000746572004C4344002074790070653A002D
:108910000D0A2000312E200048443400343738003E
:1089200030202800757369006E67200050434600B0
:1089300038353700342049004F20650078706100D9
:108940006E64650072294C0043442000287479004D
:10895000702061006464720029203D0020282000FE
:1089600020302E004D616300726F20006D656E0037
:10897000750D0A0020312E004C4344002052650042
:10898000736574000D0A2000322E49006E69740070
:10899000204C4300440D0A0020332E00436C650038
:1089A000617220004C4344000D0A2000342E430025
:1089B000757273006F722000706F730069746900C4
:1089C0006F6E200065783A002834290020300D00B1
:1089D0000A2036002E577200697465002074650005
:1089E000737420006E756D006265720073206500FF
:1089F000783A28003629200038300D000A20370048
:108A00002E5772006974650020746500737420002D
:108A100063686100726163007465720073206500B1
:108A2000783A2800372920003830440069737000F4
:108A30006C617900206C69006E6573003A0D0A0064
:108A400020312E00203120000D0A2000322E20007F
:108A50004D756C00746970006C6549004E49540096
:108A6000434C450041524300555253004F522000A1
:108A7000534554004E6F200041434B002C206300AF
:108A8000686563006B20610064617000746572004A
:108A9000434C4B00094D4F00534909004353090013
:108AA0004D4953004F5069006E7374006174650046
:108AB000733A47004E440900332E330056093500FF
:108AC0002E30560009414400430956005055090014
:108AD0004155580009500900500950000949090042
:108AE00049092D00094F570044092D00092D2D007B
:108AF0000954780044092D0009527800445343007A
:108B00004C095300444109002D092D0050474300F2
:108B10000950470044092D00092D31002E2842003C
:108B200052290900322E28005244290009332E0010
:108B3000284F5200290934002E28590057290900CE
:108B4000352E2800474E290009362E0028424C00B9
:108B5000290937002E28500055290900382E2800F1
:108B60004752290009392E0028575400290930009E
:108B70002E2842006C6B2900474E440009474E00E6
:108B80004409410044430900352E300056093300A2
:108B90002E3356000956500055094100555809001A
:108BA000657865006375740065203A0020205400E4
:108BB000494D45004F55540020302E00204D610096
:108BC00063726F00206D65006E750D000A20310024
:108BD0002E204C006976650020696E007075740067
:108BE000206D6F006E6974006F7249006E707500C1
:108BF00074206D006F6E6900746F7200202A73001C
:108C000074617200746269007420650072726F0092
:108C100072202A0070617200697479002065720008
:108C2000726F7200202A7300746F700062697400A2
:108C300020657200726F7200204E4F004E4520007A
:108C4000554E4B004E4F57004E20450052524F009C
:108C50005220610075746F0072616E0067652000BC
:108C60002B4D48007A292B006B487A00295261006D
:108C700077207600616C7500652066006F722000B9
:108C80004252470020284D00494449003D313200FE
:108C90003729570041524E00494E47003A205000B4
:108CA0006F73730069626C00652062007566660010
:108CB00065726F0076657200666C6F0077416E00BA
:108CC00079206B0065792000746F20006578690059
:108CD000745370006163650020746F0020636F003F
:108CE0006E7469006E7565004E756D006265720088
:108CF000206F660020626900747320007265610055
:108D0000642F770072697400653A200043533A007B
:108D10000D0A2000312E200043530D000A2032009E
:108D20002E202F00435320002A64650066617500E1
:108D30006C7450006F73690074696F006E20690075
:108D40006E2064006567720065657300536572008C
:108D5000766F2000616374006976650047656E0078
:108D6000657261006C0909000909090050726F0001
:108D7000746F63006F6C2000696E7400657261002F
:108D8000637469006F6E2D002D2D2D002D2D2D008B
:108D90002D2D2D002D2D2D002D2D2D002D2D2D00B7
:108DA0002D2D2D002D2D2D002D2D2D002D2D2D00A7
:108DB0002D2D2D002D2D2D002D2D2D002D2D2D0097
:108DC0002D2D2D002D2D2D002D2D2D002D2D2D0087
:108DD0002D2D2D002D2D2D002D2D2D002D2D2D0077
:108DE0002D2D2D002D2D2D002D2D3F000954680017
:108DF0006973200068656C0070090900092830005B
:108E000029094C0069737400206375007272650053
:108E10006E7420006D616300726F73003D582F0007
:108E20007C580900436F6E007665720074732000F1
:108E3000582F72006576650072736500205809002E
:108E40000928780029094D00616372006F207800BD
:108E50007E095300656C660074657300740909002F
:108E6000095B0900537461007274230009526500A4
:108E70007365740009090900095D090053746F00E6
:108E8000702409004A756D00702074006F20620024
:108E90006F6F74006C6F61006465720009097B007C
:108EA00009537400617274002077690074682000AF
:108EB0007265610064262F0025094400656C61001D
:108EC00079203100207573002F6D730009090900A6
:108ED0007D095300746F7000612F41002F4009001D
:108EE0004155580050494E0020286C006F772F00E4
:108EF00048492F00524541004429090009226100D8
:108F000062632200095365006E642000737472006E
:108F1000696E670062095300657420006261750024
:108F2000647261007465090009093100323363001D
:108F30002F43090041555800206173007369670091
:108F40006E6D65006E74200028617500782F4300F7
:108F5000532909000930780031323300642F44006E
:108F6000094D65006173750072652000414443003E
:108F700020286F006E6365002F434F004E542E0073
:108F8000290930006231310030095300656E6400F8
:108F9000207661006C75650066094D00656173009F
:108FA000757265002066720065717500656E6300FC
:108FB000790909007209520065616400672F530046
:108FC000094765006E6572006174650020505700A6
:108FD0004D2F5300657276006F0909002F09430079
:108FE0004C4B20006869680009436F006D6D61009B
:108FF0006E646800697374006F7279000909090072
:109000005C0943004C4B20006C6F690009566500F9
:10901000727369006F6E69006E666F002F73740063
:109020006174750073696E00666F0900095E09005E
:10903000434C4B0020746900636B6C002F4C09009B
:10904000426974006F72640065722000286D7300BD
:10905000622F4C005342290009092D0009444100A8
:1090600054206800696D0900436861006E676500FF
:10907000206D6F006465090009095F000944410023
:1090800054206C006F6F090053657400206F7500E9
:109090007470750074207400797065000909090006
:1090A0002E094400415420007265610064702F0055
:1090B00050095000756C6C0075702000726573006B
:1090C000697374006F72730020286F0066662F004A
:1090D0004F4E290009210900426974002072650081
:1090E0006164730009536300726970007420650045
:1090F0006E6769006E65090009093A00095265004A
:1091000070656100742065002E672E0020723A00A1
:1091100031307600095368006F772000766F6C005D
:1091200074732F00737461007465730009093B0048
:109130000942690074732000746F20007265610039
:10914000642F770072697400652065002E672E0019
:109150002030780035353B0032772F00570950001A
:1091600053552000286F6600662F4F004E290900D6
:10917000093C78003E2F3C00783D20003E2F3C000B
:10918000303E090055736500726D610063726F00B7
:1091900020782F006173730069676E0020782F00BC
:1091A0006C697300742061006C6C00000000FA00B0
:1091B000C0B52000104078000060A000C1B52000BC
:1091C00080487800A0B62000104078006840600019
:1091D0000004E00002003200CAC2A900010037000A
:1091E000CAC2A800A0B62000104078006840600005
:1091F0000004E00003003200F0C2B300007A020075
:1092000000000000A100200060AB200036A3020097
:10921000000000000080FA00000006000000FA00D4
:10922000C0B52000104078000060A100C1B520004A
:1092300080487800A0B620001040780068406000A8
:109240000004E00002003200CAC2A9000100370099
:10925000CAC2A800A0B62000104078006840600094
:109260000004E00003003200F0C2B300007A020004
:1092700000000000A100200060AB200036A3020027
:10928000000000000080FA00000006000000FA0064
:10929000A0B6200010407800684060000004E000A4
:1092A00002003200CAC2A80001003700CAC2A900E9
:1092B000A0B6200010407800684060000004E00084
:1092C00003003200F0C2B300007A02000000000088
:1092D000B100200000AC200036A302000000000016
:1092E0000080FA00000006000000FA0000C0EB0059
:1092F000820207000080FB000080FA0000000600E8
:109300000600FA00100798001E0090007B0207007C
:10931000004F7800C0B52000104078000044B20033
:109320000004E000030032001E80FB0020079800CC
:1093300001003700010037002E0090000080FA0085
:10934000000006000000FA0001022000D0C9200041
:10935000ACA2020000000000A0B420001040780081
:109360000040E8003C7802000000000000C2B300AA
:10937000007A020000000000A0B620001040780033
:10938000614060003C7802000000000000C2B300B1
:10939000007A020000000000A0B620001040780013
:1093A0000080FB000000D100614060003C780200BA
:1093B0000000000000C2B300007A020000000000BC
:1093C000A0B62000104078000080FB004200DE00C4
:1093D000614060003C7802000000000000C2B30061
:1093E000007A020000000000A0B6200010407800C3
:1093F0000080FB004300DE00614060003C7802001A
:109400000000000000C2B300007A0200000000006B
:10941000C0B52000104078000080FB004400DE0052
:10942000614060003C7802000000000000C2B30010
:10943000007A02000000000031002000F0AD2000A2
:10944000ACA20200000000000080FA00000006004C
:109450000C00FA00B421020000000000E61D02002A
:109460000000000050079800B42102000000000036
:10947000E61D02000000000040079800B421020031
:1094800000000000E61D0200000000003007980008
:10949000B421020000000000E61D020000000000F0
:1094A00020079800B421020000000000E61D020021
:1094B00000000000000F7800B4210200000000004E
:1094C000E61D020000000000100798005E009000FA
:1094D0000000E000090034005E009000E40F50003E
:1094E00006003C005E0090000040E90080407800EB
:1094F000A0B4200001487800020037000000EB0013
:10950000500798004E0090000000E0000F0034006B
:109510004E009000E20F50000C003C004E00900006
:109520000040E900E1406000A0B620001040780053
:1095300061C16000E1CFB3000140600002407000F3
:10954000A1B6200080487800020037000000EB0040
:10955000500798003E0090000000E000100034002A
:109560003E009000E20F50000D003C003E009000D5
:109570000040E90061416000A0B620009040780002
:109580006140610000414000D0CFB30080C0600066
:1095900082C07000A0B620000148780002003700A9
:1095A0000000EB00500798002E0090000000E00043
:1095B000100034002E009000E20F50000D003C001F
:1095C0002E0090000040E90061416000A0B620003C
:1095D00090407800614061004201DD00B0CFB300EF
:1095E00080C0600082C07000A0B6200001487800F2
:1095F000020037000000EB00500798001E00E0005A
:1096000010003400200020009E0F10000D003C00D0
:109610001E0078000040E90061416000A0B6200013
:1096200090407800614061004301DD0070CFB300DD
:1096300080C0600082C07000A0B6200001487800A1
:10964000020037000000EB00500798001E00900059
:109650000000E000100034001E009000E20F5000F7
:109660000D003C001E0090000040EA0061416000D7
:10967000C0B5200090407800614061004401DD00E9
:10968000F0CEB30080C0600082C07000C0B5200082
:1096900001487800020037000000EB0050079800F6
:1096A0005E0090000000E00079003A000000EB004E
:1096B000F067880071032000D0BB200036A30200B1
:1096C000000000008001EB0042002000110020009B
:1096D00010002000E0220200000000000040E9002D
:1096E00080407800A0B42000014878005103200099
:1096F00040BF200036A30200000000008001EB0004
:10970000220020001100200010002000E0220200B2
:10971000000000000040E900E1406000A0B6200029
:109720001040780061C16000E1CFB30001406000EB
:1097300002407000A1B6200080487800310420006B
:1097400090C2200036A30200000000008001EB0060
:10975000220020001100200020002000E022020052
:10976000000000000040E90061416000A0B6200058
:10977000904078006140610000414000D0CFB300CC
:1097800080C0600082C07000A0B620000148780050
:1097900011032000C0C6200036A302000000000014
:1097A0008001EB00220020001100200010002000AA
:1097B000E0220200000000000040E900614160007A
:1097C000A0B6200090407800614061004201DD00B9
:1097D000B0CFB30080C0600082C07000A0B620008F
:1097E00001487800D10120007022210036A3020038
:1097F000000000008001EB0022002000110020008A
:1098000020002000E0220200000000000040E900EB
:1098100061416000A0B62000904078006140610086
:109820004301DD0070CFB30080C0600082C07000D3
:10983000A0B6200001487800F1042000B093200079
:1098400036A30200000000008001EB00220020008F
:109850001100200010002000E022020000000000A3
:109860000040EA0061416000C0B5200090407800EF
:10987000614061004401DD00F0CEB30080C06000B3
:1098800082C07000C0B52000014878000100370098
:10989000ACFE0700C0B52000104078000060A100B9
:1098A000C1B5200080487800A0B4200010407800A6
:1098B0008080FB00E08120000080400010407800A4
:1098C000A6000700A0B62000104078000080FB0032
:1098D0004300DE0061406000614060004601DD0041
:1098E000A12C200091407800F0CBB30000C06000B4
:1098F00002407000CAE2B7000080FA0000000600D3
:109900000000FA00E90007000080FA0000000600ED
:109910000600FA00000F78001E0078006101B80010
:109920001207980023079800F00020000100200093
:109930001E019000AE019000800F5100818F5900F0
:1099400079003E001E009000AE0090000060010013
:109950000F003700130037001E0037007600370075
:1099600071003700700037006F0037006E0037005D
:109970006D0037006C0037002200370027003700E9
:109980002C00370031003700360037003B0037002D
:1099900041032000D0CB200036A3020000000000CD
:1099A00065003700710020005059200036A30200E6
:1099B00000000000F1002000C01E210036A30200BC
:1099C0000000000011C0B3000040EB00D900070008
:1099D00059003700710020005059200036A30200C2
:1099E00000000000F1002000C01E210036A302008C
:1099F0000000000011C0B30010C0B300CD0007008C
:109A00004D003700A0B62000104078000000A100F3
:109A1000A1B62000804878001D003700A0B62000C5
:109A2000104078000000A000A1B620008048780017
:109A300017003700A0B62000104078000010A100E9
:109A4000A1B620008048780011003700A0B62000A1
:109A5000104078000010A000A1B6200080487800D7
:109A60000B003700A0B62000104078000020A100B5
:109A7000A1B620008048780005003700A0B620007D
:109A8000104078000020A000A1B620008048780097
:109A9000A0B6200010407800614060006140600086
:109AA0004601DD002124200091407800F0CBB30076
:109AB00000C060000240700042E2B700A0B6200083
:109AC000104078000080FB000000D1006140600081
:109AD000614160003124200091407800E0CFB30064
:109AE00000C060000240700043E2B700A0B6200052
:109AF000104078000080FB004200DE006140600002
:109B00006140600000414000312420009140780015
:109B1000D0CFB30000C060000240700043E2B70045
:109B200008FE07000400370041022000C02020008A
:109B300036A30200000000000080FA0000000600CA
:109B40000000FA0001012000A004210036A3020059
:109B5000000000000080FA00000006000200FA0089
:109B6000004F780041E2A900C0B520001040780005
:109B7000704060000004E00004003200CEE2A80063
:109B8000CF02A800CEC2A80003003700CEE2A90091
:109B9000CF02A900CEC2A900816A200091407800BE
:109BA00000CEB30000C060007040B300A8E6B7006C
:109BB000916C20009140780000CEB30000C060009E
:109BC0007040B300C9E6B700816C20009140780076
:109BD00000CEB30000C060000034A000C8E6B700AB
:109BE000CAC2A800C8C2A900C902A900C8E2A80048
:109BF000C922A9001E80FB001012880042A2A80002
:109C0000A0B6200010407800614060006140600014
:109C10004601DD002124200091407800F0CBB30004
:109C200000C060000240700042E2B700A0B6200011
:109C3000104078000080FB000000D100614060000F
:109C4000614160003124200091407800E0CFB300F2
:109C500000C060000240700043E2B700A0B62000E0
:109C6000104078000080FB004200DE006140600090
:109C700061406000004140003124200091407800A4
:109C8000D0CFB30000C060000240700043E2B700D4
:109C90000000EB00201288000000EB00001288009A
:109CA00041E2A8000080FA00000006000000FA006F
:109CB00041E2A900A8C6BF00F041B300A8E6B70082
:109CC000916C20009140780000CEB30000C060008D
:109CD000C9E6B700816C20009140780000CEB30047
:109CE00000C06000C8E6B700CEE2A900CF02A9001C
:109CF000CEC2A9000080FA00000006000200FA00AF
:109D0000004F78001E80FB004012880085C0BF0015
:109D1000644060000004E000FCFF3200401280005C
:109D2000004F78008540A9001E80FB000080FA00EB
:109D3000000006000400FA00204798003147980010
:109D400010C0B300004F7800A87A020000000000A5
:109D5000D6FF0700850007002E4090000004E000B9
:109D600002003A0042E2A80062E2A8002E40900001
:109D7000E14F500002003E0041E2A80061E2A8006D
:109D80001E04E00009003A00CAC2BF000044B2004D
:109D90000004E00005003200D0C5B300BC7A020028
:109DA0000000000010C0B300004F780040C2BF00A8
:109DB0000042B2000004E0002F003A0060C2BF0081
:109DC0000042B2000004E0002B003A004012800084
:109DD0001047980010C0B3009E4F100005003A00D5
:109DE000B0C5B300BC7A0200000000000040EB00E8
:109DF000004F78003E4090000004E0000500320073
:109E00001E4090000080FB00C878020000000000A7
:109E100006003700C0C5B300BC7A02000000000095
:109E20001E409000BC7A0200000000004013800039
:109E3000104798003E4090000004E0000B00320004
:109E400080C2B300BC7A0200000000001E409000F7
:109E50000080FB00C87802000000000090C2B30040
:109E6000BC7A020000000000030037001E40900092
:109E7000BC7A02000000000040C2BF000044B200F3
:109E80000004E00009003A0060C2BF000044B200D4
:109E90000004E00005003A00D040800001402000AE
:109EA000010060000000E00014003200D04080009B
:109EB00001402000010060000000E00002003A00C4
:109EC000247B0200000000000000EB00001288006C
:109ED0000000EB00001388003E4090000004E0000A
:109EE0000400320060A32800D075020000000000CA
:109EF00093FF3700C222A9001200370023C2BF001F
:109F0000624060000004E00002003A00F27A0200C1
:109F10000000000022C2BF00614060000004E000B9
:109F200097FF320030118000104798003E409000AB
:109F30000004E0000300320070A42800D075020085
:109F40000000000088000700A0B420001040780046
:109F50008080FB00E08120000080400010407800FD
:109F6000FEFE07000080FA00000006000000FA0074
:109F7000C8C2A800C902A800C8E2A800C922A80057
:109F8000A16A20009140780000CEB30000C06000BC
:109F90006040B300AAE6B700E16A20009140780073
:109FA00000CEB30000C060006040B300AEE6B70072
:109FB000816A20009140780000CEB30000C06000AC
:109FC0009040B300A8E6B700916A20009140780065
:109FD00000CEB30000C060000034A000A9E6B700C6
:109FE000C16A20009140780000CEB30000C060003C
:109FF0007040B300ACE6B700D16A20009140780011
:10A0000000CEB30000C060000034A000ADE6B70091
:10A01000A0B42000104078008080FB00E081200088
:10A0200000804000104078000080FB001012880083
:10A03000A0B62000104078006140600061406000E0
:10A040004601DD002124200091407800F0CBB300D0
:10A0500000C060000240700042E2B700A0B62000DD
:10A06000104078000080FB000000D10061406000DB
:10A07000614160003124200091407800E0CFB300BE
:10A0800000C060000240700043E2B7000000EB0037
:10A09000201288000000EB0000128800A0B420000D
:10A0A000104078008080FB00E081200000804000AC
:10A0B000104078000080FB0010138800A0B620003C
:10A0C0001040780061406000614060004601DD00A2
:10A0D0002126200091407800F0CBB30000C0600042
:10A0E0000240700062E2B700A0B620001040780085
:10A0F0000080FB000000D100614060006141600011
:10A100003126200091407800E0CFB30000C060000D
:10A110000240700063E2B7000000EB0020138800EB
:10A120000000EB00001388000000EB0040128800E4
:10A130000000EB00401388004322A9006322A9001D
:10A140004362A80042A2A9006362A80062A2A9001B
:10A1500040C2A90060C2A9004402A8006402A8008D
:10A160000080FA00000006000000FA0041E2A900A9
:10A170004362A90061E2A9006362A900AAC6BF0008
:10A18000F041B300AAE6B700AEC6BF00F041B3008D
:10A19000AEE6B700A8C6BF00F041B300A8E6B7001E
:10A1A000A9C6BF00F041B300A9E6B700ACC6BF0026
:10A1B000F041B300ACE6B700ADC6BF00F041B3005C
:10A1C000ADE6B7000080FA00000006000000FA00CB
:10A1D00080A42800A4750200000000000080FA009E
:10A1E000000006000A00FA00881F780011C0B300C2
:10A1F000A0B4200001487800A0B6200010407800EC
:10A200000000A100A1B6200080487800A0B6200080
:10A21000104078000010A000A1B62000804878000F
:10A22000A0B62000104078000020A100A1B62000B8
:10A2300080487800C0B52000104078000040A000A1
:10A24000C1B5200080487800A0B4200010407800FC
:10A250008080FB00208220000080400010407800B9
:10A260003EFE0700D9FF07000000370022C2BF00F2
:10A27000614060000004E000FCFF3200301180000B
:10A280008040780080B620000148780080B6200029
:10A29000104078000080FB004400DE008040780021
:10A2A00070B620000148780070B620001040780099
:10A2B0000080FB00400798004E009000E40F500023
:10A2C000EF0032004E009000E40F500007003C0009
:10A2D0004E0090000000E0000B0032004E009000A5
:10A2E000E10F5000C0003200510137004E009000D5
:10A2F000E60F5000EA0032004E009000E80F5000D8
:10A30000FC0032004A01370080B62000104078007F
:10A310000080FB00300798003E009000E30F5000E3
:10A32000230032003E009000E30F50000A003C0082
:10A330003E009000E10F5000130032003E009000FC
:10A34000E10F500012003C003E0090000000E000D1
:10A350000B003200A00037003E009000ED0F5000CF
:10A360001B0032003E009000EE0F50001F00320034
:10A370003E009000E40F50002300320096003700AA
:10A380004AFE07002E01370090FF0700B7FF370095
:10A3900060168000F1FB2F0001006000601688004D
:10A3A00010C0B300007A020000000000AFFF3700C9
:10A3B0006016800001042000010070006016880013
:10A3C00010C0B300007A020000000000A7FF3700B1
:10A3D00010C0B300007A0200000000008040EB00D3
:10A3E00010C0B30053FE0700A0FF370010C0B30039
:10A3F000007A0200000000008040EB000040EB000B
:10A400004CFE070099FF370022C2BF006140600088
:10A410000004E000FCFF32003011800010079800BB
:10A420001E0090004800DD001007980022C2BF0007
:10A43000614060000004E000FCFF32003011800049
:10A440009E009000008070001007980022C2BF009C
:10A45000614060000004E000FCFF32003011800029
:10A46000000F78001E0078004800DD00000F780023
:10A4700022C2BF00614060000004E000FCFF320027
:10A48000301180001E0F70009E009000000021001F
:10A49000808F500003003E00000021009E0F10003E
:10A4A000040036000040EB00007A020000000000CB
:10A4B0006EFF37000000EB00200798000C0037000B
:10A4C00022C2BF00614060000004E000FCFF3200D7
:10A4D000714080002E00900080804000301180008C
:10A4E000804878002E0090000000E80020079800C7
:10A4F000AE0090001E009000808F5000F0FF3900E9
:10A50000CAC2A9000000EB0020079800080037002D
:10A51000714080002E0090000080400010407800C4
:10A52000F6FD07002E0090000000E80020079800CC
:10A53000AE0090001E009000808F5000F4FF3900A4
:10A54000100020003AA00200000000000000EB0014
:10A550002007980009003700714080002E0090000D
:10A560000084400000C0EB00E4FD0700004C7800D0
:10A570002E0090000000E800200798002E009000B8
:10A580009E0F5000F4FF3900CAC2A80010C0B300EB
:10A59000007A0200000000000000EB002007980095
:10A5A00009003700714080002E00900000804000BC
:10A5B00010407800007A0200000000002E00900099
:10A5C0000000E800200798002E0090009E0F500029
:10A5D000F4FF390025FF37000040EB00007A02004D
:10A5E0000000000021FF370080B620009040780076
:10A5F000F0C0B30080C0600080B620000148780041
:10A6000080B62000104078008040E80080B620002E
:10A610000148780010C0B300007A0200000000007A
:10A620008040EB0060B62000014878000D00370044
:10A6300022C2BF00614060000004E000FCFF320065
:10A6400030118000ADFD0700007A0200000000001C
:10A6500060B62000104078008040E80060B620001E
:10A660000148780060B620009040780080B6200055
:10A670001040780080CF5000EDFF3900FBFE37001E
:10A6800080B6200010407800A2A602000000000062
:10A6900010C0B300007A020000000000F3FE370093
:10A6A00080B620009040780070C0B30080C0600089
:10A6B00080B620000148780080B6200090407800E5
:10A6C000A0B4200001487800A0B420001040780019
:10A6D0008080FB0020822000008040001040780035
:10A6E0001EFD070010C0B300007A02000000000049
:10A6F000DEFE3700A0B62000104078000000A10068
:10A70000A1B6200080487800A0B620001040780054
:10A710000010A100A1B6200080487800A0B620005B
:10A72000104078000020A100A1B6200080487800E9
:10A73000C0B52000104078000040A100C1B5200045
:10A740008048780080B62000104078000080FB0030
:10A750004200DE00610060000004E00005003200FD
:10A76000A0B62000104078000000A000A1B6200094
:10A770008048780080B62000104078000080FB0000
:10A780000000D100610060000004E000050032001C
:10A79000A0B62000104078000010A000A1B6200054
:10A7A0008048780080B62000104078000080FB00D0
:10A7B000610060000004E00005003200A0B6200047
:10A7C000104078000020A000A1B62000804878004A
:10A7D00080B62000104078000080FB004300DE00BF
:10A7E0000000A200610060000004E00005003200EB
:10A7F000C0B52000104078000040A000C1B5200086
:10A8000080487800A0B42000104078008080FB00D1
:10A81000208220000080400010407800CFFC07001C
:10A8200010C0B300007A0200000000008FFE370065
:10A830000040EB00007A0200000000008BFE3700B1
:10A840004F0478000080FA00000006000400FA00BF
:10A85000EAA40200000000000004E0002200320030
:10A8600032C2BF00684060000004E0000400320013
:10A870003100200010CF2000ACA202000000000038
:10A8800032C2BF00644060000004E00004003200F7
:10A890003100200040CF2000ACA2020000000000E8
:10A8A000DAA4020000000000000F780032C2BF00EE
:10A8B000624060000004E00008003200F100200067
:10A8C00070CF2000ACA202000000000090118000B8
:10A8D000D1FF2F0001006000901188001E00780059
:10A8E0001007980006003700F100200060D020001B
:10A8F000ACA20200000000000000EB00100798006E
:10A900001E0090000080FA00000006000200FA001D
:10A91000000F78001E007800C6A4020000000000AE
:10A920000000EB000080FA00000006000000FA00C2
:10A9300001022000C0DB2000ACA2020000000000E9
:10A94000A0B42000104078003C7802000000000015
:10A9500000C2B300007A020000000000A0B4200092
:10A9600010407800E94F500007003A00C011800005
:10A97000DE7702000000000000C2B300007A02008F
:10A98000000000000C003700A0B420001040780048
:10A990000080FB0080004000C0AD2000008040002F
:10A9A00010007800DE7702000000000000C2B30053
:10A9B000007A020000000000C0DA20001040780099
:10A9C000634060003C7802000000000000C2B30059
:10A9D000007A020000000000C0DA20001040780079
:10A9E0000080FB004200DE00614060003C78020015
:10A9F0000000000000C2B300007A02000000000066
:10AA0000C0DA2000104078000080FB004300DE0028
:10AA1000614060003C7802000000000000C2B3000A
:10AA2000007A020000000000C0B52000104078004D
:10AA30000080FB004400DE00614060003C780200C2
:10AA40000000000000C2B300007A02000000000015
:10AA500031002000F0AD2000ACA202000000000098
:10AA60000080FA00000006000C00FA00B421020089
:10AA700000000000E61D02000000000050079800E2
:10AA80005E009000EA0F500005003A00B421020079
:10AA900000000000E61D020000000000000F78002A
:10AAA000B421020000000000E61D020000000000CA
:10AAB00040079800B421020000000000E61D0200DB
:10AAC0000000000030079800B421020000000000E0
:10AAD000E61D02000000000020079800B4210200DB
:10AAE00000000000E61D02000000000010079800B2
:10AAF0005E0090000000E000090034005E0090005D
:10AB0000EA0F500006003C005E0090000040E900A3
:10AB100080407800A0B4200001487800020037008F
:10AB20000000EB00500798004E0090000000E0008D
:10AB30000F0034004E009000E40F50000C003C0069
:10AB40004E0090000040E900E3406000C0DA2000C1
:10AB50001040780063C16000C1CFB30001406000C5
:10AB600002407000C1DA20008048780002003700FF
:10AB70000000EB00500798003E0090000000E0004D
:10AB8000100034003E009000E20F50000D003C0029
:10AB90003E0090000040E90061416000C0DA200002
:10ABA00090407800614061004201DD00B0CFB30009
:10ABB00080C0600082C07000C0DA200001487800C8
:10ABC000020037000000EB00500798002E009000B4
:10ABD0000000E000100034002E009000E20F500052
:10ABE0000D003C002E0090000040E9006141600033
:10ABF000C0DA200090407800614061004301DD0030
:10AC000070CFB30080C0600082C07000C0DA200046
:10AC100001487800020037000000EB005007980060
:10AC20001E0090000000E000100034001E009000A4
:10AC3000E20F50000D003C001E0090000040EA00B2
:10AC400061416000C0B52000904078006140610023
:10AC50004401DD00F0CEB30080C0600082C070000F
:10AC6000C0B5200001487800020037000000EB006A
:10AC7000500798005E0090000000E00073003A006A
:10AC80000000EB00F0678800D1082000308720002A
:10AC900036A30200000000008001EB00A2002000AB
:10ACA0001100200010002000E0220200000000003F
:10ACB0000040E90080407800A0B4200001487800FE
:10ACC000A0B4200010407800E94F50000B003A007B
:10ACD000C1012000001B210036A30200000000007B
:10ACE0008001EB00F2FF270011002000200220006D
:10ACF000E022020000000000000F78004105200063
:10AD000050D12000ACA20200000000008001EB0046
:10AD1000420020001100200010002000E02202006C
:10AD2000000000000040E900E3406000C0DA2000BD
:10AD30001040780063C16000C1CFB30001406000E3
:10AD400002407000C1DA2000804878001102200023
:10AD500090D62000ACA20200000000008001EB00B1
:10AD6000220020001100200010002000E02202003C
:10AD7000000000000040E90061416000C0DA2000EE
:10AD800090407800614061004201DD00B0CFB30027
:10AD900080C0600082C07000C0DA200001487800E6
:10ADA00021032000A0D82000ACA202000000000077
:10ADB0008001EB0022002000110020001000200084
:10ADC000E0220200000000000040E9006141600054
:10ADD000C0DA200090407800614061004301DD004E
:10ADE00070CFB30080C0600082C07000C0DA200065
:10ADF00001487800F1042000B093200036A302003F
:10AE0000000000008001EB00220020001100200063
:10AE100010002000E0220200000000000040EA00D4
:10AE200061416000C0B52000904078006140610041
:10AE30004401DD00F0CEB30080C0600082C070002D
:10AE4000C0B520000148780001003700B7FE0700B8
:10AE5000A0B4200010407800E94F50001C003A00D8
:10AE6000C0DA2000104078000080FB004200DE00C5
:10AE70006140600080417800C0DA20001040780016
:10AE80006340600080427800C0DA20001040780003
:10AE90000080FB004300DE0061406000004178005C
:10AEA000C0B52000104078000080FB004400DE00A8
:10AEB00061406000804078001E0078000342780006
:10AEC000854178001AA4020000000000220037002B
:10AED000C0DA2000104078000080FB004200DE0055
:10AEE0006140600000417800C0DA20001040780026
:10AEF0006340600080417800C0DA20001040780094
:10AF00000080FB004300DE0061406000804278006A
:10AF1000C0B52000104078000080FB004400DE0037
:10AF20006140600000437800A0B420001040780029
:10AF30000080FB0080004000C0AD20000080400089
:10AF400010007800024278000541780086407800C1
:10AF50001AA4020000000000C0DA200010407800AF
:10AF600063406000E34F500003003A0091C0B3001B
:10AF7000B0B42000014878009EA402000000000048
:10AF8000C111800040118000808F5000040031000A
:10AF900001022000C01C210036A3020000000000B6
:10AFA0000080FA00000006000000FA00AAA40200D7
:10AFB000000000000080FA00000006000400FA0013
:10AFC000000F78001E007800100798001E00900007
:10AFD000E10F5000130032001E009000E10F5000FE
:10AFE000070039001E009000E20F50005E003200A2
:10AFF0001E009000E30F500006003200770037007B
:10B0000031052000C0DD2000ACA2020000000000DD
:10B0100076003700C062A900C082A800C8C2A8009C
:10B02000C902A900B1002000F0E2200036A302000E
:10B0300000000000D1002000A0E3200036A30200A1
:10B0400000000000DCA30200000000000000E0009F
:10B050006600320090118000D1FF2F0001006000D7
:10B06000901188000000370032C2BF0061406000CC
:10B070000004E0000600320023C2BF00624060000E
:10B080000004E00002003A00B011800020118800A6
:10B0900022C2BF00614060000004E00006003200F0
:10B0A00033C2BF00624060000004E00002003A00CA
:10B0B00030118000A011880032C2BF0062406000E1
:10B0C0000004E00004003A0022C2BF0062406000B9
:10B0D0000004E0000900320091118000D0FF2F0031
:10B0E000008060009011880011118000D0FF2F00B7
:10B0F0000080600010118800C222A90030002000EA
:10B100009E0F1000D8FF3A00C2C2BF000080FB00B3
:10B110004400DE006140600061416000B12C20000D
:10B1200091407800E0CFB30000C0600002407000A2
:10B13000CBE2B700CAC2BF000080FB004600DE00C1
:10B1400061406000614060004301DD00212C20006F
:10B150009140780070CFB30000C0600002407000E2
:10B16000C2E2B700C0FF3700E100200070E4200019
:10B1700036A3020000000000F1002000C01E2100E4
:10B1800036A302000000000090118000D1FF2F00C4
:10B19000010060009011880032C2BF006140600071
:10B1A0000004E0000600320023C2BF0062406000DD
:10B1B0000004E00002003A00B01180002011880075
:10B1C00022C2BF00614060000004E000F2FF3200D4
:10B1D00030118000000F7800040037004102200089
:10B1E000C020200036A30200000000000080FA000A
:10B1F000000006000000FA0091118000D0FF2F002F
:10B200000080600090118800C0DA200010407800B3
:10B210000040A000C1DA200080487800C0B52000BE
:10B22000104078000020A000C1B5200080487800C0
:10B23000C101200050E5200036A3020000000000FC
:10B240000080FA00000006000000FA00C0DA2000CA
:10B25000104078000040A100C1DA2000804878004A
:10B26000C0B52000104078000020A100C1B520002A
:10B27000804878004101200010E7200036A302003A
:10B28000000000000080FA00000006000200FA0042
:10B290000000EB00000F780034003700C0DA200017
:10B2A00010407800704060000004E0002B00320085
:10B2B00060A72800D0750200000000006100200097
:10B2C00060692000ACA202000000000032C2BF0092
:10B2D000684060000004E0000400320031002000FB
:10B2E00010CF2000ACA202000000000032C2BF005C
:10B2F000644060000004E0000400320031002000DF
:10B3000040CF2000ACA2020000000000DAA402003E
:10B3100000000000689F02000000000032C2BF0071
:10B32000624060000004E00008003200F1002000EC
:10B3300070CF2000ACA2020000000000901180003D
:10B34000D1FF2F00010060009011880060A7280045
:10B35000D07502000000000002003700DAA40200ED
:10B360000000000010002000000F7800EAA4020096
:10B37000000000000004E000C8FF3A001E00780052
:10B380000080FA00000006000000FA00B100200072
:10B390001009210036A30200000000000080FA001E
:10B3A000000006000000FA0070A72800A475020043
:10B3B000000000000080FA00000006000400FA000F
:10B3C000C0DA2000104078000000A1000010A100A9
:10B3D000C1DA200080487800C0DA200010407800F0
:10B3E0000020A100C1DA200080487800C0DA2000E7
:10B3F000104078000030A100C1DA200080487800B9
:10B40000C0B52000104078000040A000C1B5200069
:10B410008048780080578000306D8800C0DA2000B6
:10B42000104078000040A100C1DA20008048780078
:10B43000C0DA2000104078000080FB004200DE00EF
:10B440006140600080417800C0DA20001040780040
:10B450006340600080427800C0DA2000104078002D
:10B460000080FB004300DE00614060000041780086
:10B47000C0B52000104078000080FB004400DE00D2
:10B480006140600080407800306D800003427800A9
:10B49000854178001AA40200000000009EA402006A
:10B4A00000000000BFFF070000003700EAA4020010
:10B4B000000000000004E0000C003200C0DA2000B0
:10B4C00010407800704060000004E0000500320089
:10B4D000DAA4020000000000007A02000000000070
:10B4E00002003700DAA402000000000032C2BF00F0
:10B4F000624060000004E00004003200901180000F
:10B50000D1FF2F00010060009011880022C2BF000F
:10B51000614060000004E000E4FF32003011800070
:10B5200080407800A0DA200001487800A0DA2000EE
:10B53000104078000080FB004400DE00804078006E
:10B5400090DA20000148780090DA2000104078005E
:10B550000080FB00100798001E009000E40F5000D0
:10B56000D00032009E009000E48F500007003C00A5
:10B570001E0090000000E0000F0032009E009000CE
:10B58000E18F50009F0032008A0137001E009000BA
:10B59000E60F5000CB0032009E009000E68F500076
:10B5A000840135009E00900068805000E10F50003B
:10B5B00080013E00FB003700A0DA20001040780038
:10B5C0000080FB00000F78001E007800E20F5000A2
:10B5D000190032009E007800E28F500007003C0006
:10B5E0001E0078000000E0000E0032009E0078008F
:10B5F000E18F50000E0032007E0037001E00780000
:10B60000E70F5000260032009E007800EF8F5000B8
:10B610005B0032001E007800E30F5000170032007C
:10B6200074003700AAA40200000000006501370082
:10B630005CFF07009DFF370010C0B300007A0200D6
:10B640000000000032C2BF00624060000004E00061
:10B650000400320090118000D1FF2F000100600033
:10B6600090118800C0DA2000104078000040A0004F
:10B67000C1DA2000804878008CFF3700C0DA200053
:10B68000104078000040A100C1DA20008048780016
:10B6900010C0B300007A02000000000083FF3700F2
:10B6A00010C0B300007A020000000000AAA402004B
:10B6B0000000000022C2BF00614060000004E00002
:10B6C000FCFF3200301180004800DD00306D880042
:10B6D00010C0B300007A02000000000022C2BF00C8
:10B6E000614060000004E000FCFF3200316D80002A
:10B6F0003011800000807000306D8800C0DA2000BA
:10B70000104078000080FB004200DE0061406000D5
:10B7100080417800C0DA200010407800634060006B
:10B7200080427800C0DA2000104078000080FB00E2
:10B730004300DE006140600000417800C0B5200099
:10B74000104078000080FB004400DE006140600093
:10B7500080407800306D8000034278008541780099
:10B760001AA40200000000009EA4020000000000D5
:10B7700010C0B300007A0200000000004BFF370049
:10B7800010C0B300007A0200000000009011800099
:10B79000D1FF2F00010060009011880000003700E9
:10B7A00032C2BF00614060000004E00006003200C9
:10B7B00023C2BF00624060000004E00002003A00C3
:10B7C000B01180002011880022C2BF0061406000DB
:10B7D0000004E000F2FF320033C2BF0062406000AC
:10B7E0000004E000EEFF3A0030118000A011880054
:10B7F000EBFF37000040EB00007A02000000000081
:10B800002AFF3700A0DA200090407800F0C0B30093
:10B8100080C06000A0DA200001487800A0DA200093
:10B82000104078008040E800A0DA2000014878004D
:10B8300010C0B300007A0200000000008040EB005E
:10B8400080DA2000014878000F00370022C2BF00D4
:10B85000614060000004E000FCFF32003011800015
:10B86000C6A402000000000010C0B300007A02006D
:10B870000000000080DA2000104078008040E800DE
:10B8800080DA20000148780080DA200090407800BB
:10B89000A0DA20001040780080CF5000EBFF390084
:10B8A00002FF3700A0DA200010407800A2A60200B4
:10B8B0000000000010C0B300007A02000000000089
:10B8C000FAFE3700A0DA200090407800F0C0B30004
:10B8D00080C06000A0DA200001487800A0DA2000D3
:10B8E00010407800EA4F500003003600A1C0B300BA
:10B8F000A0DA200001487800A0DA2000104078008B
:10B900000080FB008000400000AF2000008040006D
:10B9100010007800306D8800AAA40200000000002A
:10B92000C0DA2000104078000080FB004200DE00FA
:10B930006140600080417800C0DA2000104078004B
:10B940006340600080427800C0DA20001040780038
:10B950000080FB004300DE00614060000041780091
:10B96000C0B52000104078000080FB004400DE00DD
:10B970006140600080407800306D800003427800B4
:10B98000854178001AA40200000000009EA4020075
:10B990000000000010C0B300007A020000000000A8
:10B9A000C2FE3700C0DA2000104078000000A1007D
:10B9B0000010A100C1DA200080487800C0DA200021
:10B9C000104078000020A100C1DA200080487800F3
:10B9D000C0DA2000104078000030A100C1DA200059
:10B9E00080487800C0B52000104078000040A100D9
:10B9F000C1B5200080487800A0DA2000104078000F
:10BA00000080FB004300DE00610060000004E000F5
:10BA10000D003200C0DA2000104078006340600062
:10BA20000014A000E3406000C0DA2000104078005D
:10BA300063C16000C1CFB3000140600002407000EC
:10BA4000C1DA200080487800A0DA20001040780099
:10BA50000080FB004200DE00610060000004E000A6
:10BA60000D003200C0DA2000104078006340600012
:10BA70000004A000E3406000C0DA2000104078001D
:10BA800063C16000C1CFB30001406000024070009C
:10BA9000C1DA200080487800A0DA20001040780049
:10BAA0000080FB000000D100610060000004E000A5
:10BAB00005003200C0DA2000104078000020A0000D
:10BAC000C1DA200080487800A0DA20001040780019
:10BAD0000080FB00610060000004E000050032000F
:10BAE000C0DA2000104078000030A000C1DA200049
:10BAF00080487800A0DA2000104078000080FB0029
:10BB00004400DE000000A200610060000004E000CC
:10BB100005003200C0B52000104078000040A000B1
:10BB2000C1B5200080487800AAA4020000000000EF
:10BB3000C0DA2000104078000080FB004200DE00E8
:10BB40006140600080417800C0DA20001040780039
:10BB50006340600080427800C0DA20001040780026
:10BB60000080FB004300DE0061406000004178007F
:10BB7000C0B52000104078000080FB004400DE00CB
:10BB80006140600080407800306D800003427800A2
:10BB9000854178001AA40200000000009EA4020063
:10BBA0000000000010C0B300007A02000000000096
:10BBB0003EFE37000040EB00007A0200000000006B
:10BBC0003AFE37000080FA00000006000000FA008C
:10BBD000D6A10200000000000080FB000080FA00F7
:10BBE000000006000200FA00000F78001E00780036
:10BBF0003EA1020000000000001020000080FA00BA
:10BC0000000006000000FA003CA202000000000054
:10BC10000080FB000080FA00000006000000FA002F
:10BC200080B72000104078009CA1020000000000B6
:10BC30000080FA00000006000000FA0080B7200033
:10BC4000104078000080FB000080FA000000060031
:10BC50000000FA008040EB0080B720000148780027
:10BC600041022000B000200036A3020000000000C6
:10BC70000080FA00000006000000FA0011C0B300C6
:10BC800080B720000148780041022000B000200069
:10BC900036A30200000000000080FA000000060049
:10BCA0000000FA00C0B52000104078000040A0005D
:10BCB000C1B52000804878008040EB00A0B820008B
:10BCC00001487800C922A800CB22A900E102200087
:10BCD000F002200036A30200000000000080FA00FD
:10BCE000000006000400FA00881F7800000F7800AA
:10BCF0001E00E00044003200200320009E0F1000D0
:10BD000041003E001E0FE900A0B82000104078005E
:10BD10000080FB009E0F500005003E0091022000B5
:10BD2000D005200036A302000000000063013700A8
:10BD3000E100200060082000ACA20200000000002A
:10BD40001E0078000040E8003C780200000000007F
:10BD5000C0A52800A4750200000000008040EB0090
:10BD600040B82000014878001F0037001E0178000D
:10BD700040B82000104078008080FB004310DD00B8
:10BD800081004000B0B820000080400010407800E2
:10BD90000080FB00689F02000000000000C2B300AA
:10BDA000007A0200000000001E01780040B8200068
:10BDB000104078008080FB004310DD0081004000CF
:10BDC000B0B8200000804000104078003EA1020082
:10BDD0000000000040B82000104078008040E800DB
:10BDE00040B820000148780040B82000104078009A
:10BDF000E74F5000DDFF3600F0A52800D0750200A7
:10BE0000000000002D0137001E0078001007980088
:10BE1000500520009E009000808F500011013200DC
:10BE2000500520009E009000808F500008003E00CA
:10BE30001E0090000000E0001200320030032000DD
:10BE40009E009000808F5000DD0032001701370007
:10BE5000C00E20009E009000808F500063003200D2
:10BE6000000F20009E009000808F50005F00320085
:10BE7000C00C20009E009000808F50000201320014
:10BE80000A013700D10020004009200036A302003B
:10BE90000000000071012000100A200036A30200FB
:10BEA00000000000A0B82000104078000004E0006E
:10BEB00005003A0091022000D005200036A30200C0
:10BEC00000000000440037008040EB0050B8200024
:10BED000014878003A00370000C2B300007A02003F
:10BEE0000000000050B82000104078000040E8003A
:10BEF0003C7802000000000000A62800A4750200A3
:10BF0000000000008040EB0040B8200001487800AD
:10BF10001600370050B82000104078000081FB0068
:10BF200040B82000104078008080FB004310DD0006
:10BF300081004000B0B82000008040001040780030
:10BF40000080FB00689F02000000000000C2B300F8
:10BF5000007A02000000000040B820001040780085
:10BF60008040E80040B820000148780040B8200038
:10BF700010407800E74F5000E6FF360061002000D7
:10BF8000800B2000ACA202000000000050B820008E
:10BF9000104078000080FB00C300DD00B0B8200036
:10BFA0000080400010407800F700070050B82000E3
:10BFB000104078008040E80050B820000148780028
:10BFC000A0B820009040780050B8200010407800C1
:10BFD00080CF5000C0FF3E00310D2000E00B20005C
:10BFE00036A3020000000000B40037001E007800F5
:10BFF00080407800C083200001487800C00E2000F7
:10C000009E0F100005003A00310120001019200099
:10C0100036A302000000000004003700D100200019
:10C02000401A200036A30200000000007101200029
:10C03000100A200036A30200000000008040EB0040
:10C0400040B82000014878000A01070080407800CD
:10C0500050B82000014878008040EB00A0B82000D4
:10C06000014878004D00370000C2B300007A02009A
:10C070000000000040B82000104078000040E800B8
:10C080003C7802000000000000A62800A475020011
:10C09000000000000000EB00105C88000D0037007D
:10C0A000115C8000B0BD200000804000104078008E
:10C0B0000080FB00689F02000000000000C2B30087
:10C0C000007A020000000000105C80000000E80020
:10C0D000105C8800105C8000E70F5000F0FF360015
:10C0E00061002000800B2000ACA2020000000000D4
:10C0F000B0BD200010407800A300070040B8200029
:10C1000010407800E94F50001B003E000000EB009B
:10C11000105C880010003700A0B8200010407800A4
:10C120008081FB00145C8000115C8000B0BD2000A9
:10C1300000804000104178004318DD00840040007A
:10C14000B0B820000080400002487800105C8000F9
:10C150000000E800105C8800105C8000E70F5000D1
:10C16000EDFF3600A0B82000104078008040E800C5
:10C17000A0B820000148780040B8200010407800A6
:10C180008040E80040B8200001487800C700070060
:10C190008040780050B820000148780050B8200056
:10C1A000104078000004E000AFFF3A00B102200028
:10C1B000101B200036A30200000000003F003700E3
:10C1C0004800070011012000C01D2000ACA20200A1
:10C1D0000000000030C3B3003EA1020000000000D8
:10C1E0000000EB00105C880014003700185C800031
:10C1F000D6A10200000000008040780090B7200027
:10C200000000440001487800115C800090B72000D5
:10C2100000804000104078000080FB00689F020012
:10C220000000000000C2B300007A0200000000001D
:10C23000105C80000000E800105C8800105C80004A
:10C24000E70F5000E9FF3600F0A52800D075020086
:10C250000000000090B72000104078004A0007005E
:10C26000160037001F00070001012000D01E20002B
:10C2700036A302000000000050C5B3003EA102003A
:10C28000000000000D00370016000700F10020003C
:10C29000D01F200036A3020000000000C0CCB30075
:10C2A0003EA102000000000004003700410220000F
:10C2B000C020200036A30200000000004F047800D8
:10C2C0000080FA00000006000000FA009100200043
:10C2D0008008210036A30200000000000080FA0060
:10C2E000000006000200FA00B8A0020000000000F2
:10C2F000004F7800A100200000232000ACA2020023
:10C30000000000001E04E00005003A00310020009B
:10C3100050BB200036A302000000000018003700C8
:10C3200091002000A0232000ACA202000000000029
:10C330001E80FB00610060000004E0000400320089
:10C340005101200030242000ACA2020000000000B7
:10C350001E80FB000000D100610060000004E000CE
:10C36000040032004101200080252000ACA2020020
:10C3700000000000F0A52800D075020000000000B9
:10C380000080FA00000006000400FA00004F780068
:10C390001E80FB0010079800200220009E009000E5
:10C3A000808F50001E003200200220009E0090006E
:10C3B000808F500007003C001E009000E40F5000EA
:10C3C0001C0032009E009000F08F50000A003200E6
:10C3D00022003700800220009E009000808F5000D5
:10C3E0000A003200D00220009E009000808F500092
:10C3F0001500320019003700B1012000C0262000CE
:10C4000036A302000000000018003700A101200040
:10C410007028200036A3020000000000130037003F
:10C4200051012000102A200036A302000000000065
:10C430000E00370081012000602B200036A302008F
:10C44000000000000900370001012000E02C20005E
:10C4500036A302000000000004003700E1002000C5
:10C46000E02D2000ACA20200000000000080FA00D5
:10C47000000006000000FA008040EB0030BE200003
:10C48000014878008040EB0050BE20000148780051
:10C490008040EB0040BE2000014878000800070003
:10C4A0000080FB000080FA00000006000000FA0097
:10C4B000030007000080FB000080FA000000060077
:10C4C0000A00FA0010C0B300704798000040EB006B
:10C4D000604798000040EB005047980010C0B30040
:10C4E000104798000040EB00404798008040EB0068
:10C4F00060BE20000148780050BE20001040780047
:10C500000004E0009C003A00B8A002000000000017
:10C510000004E0000C0032008040EB0030BE200040
:10C52000014878008040EB0050BE200001487800B0
:10C530008040EB0040BE2000014878000000EB0086
:10C5400040079800A1003700C08320001040780009
:10C550003EA10200000000003CA20200000000001A
:10C56000304798003CA202000000000020479800DD
:10C570003E409000E14F500003003A002E409000F2
:10C58000E14F500068003200BE4090002E40900005
:10C5900080CF500003003200BE409000014F780071
:10C5A0002600370030BE2000904078007E4090008A
:10C5B000814F50000E0031005E4090008080FB00F3
:10C5C000B0BD200000804000904078001E409000E8
:10C5D00080C060000040EB00004F78000104E000E4
:10C5E0000C00320010C0B300004F78000900370083
:10C5F00030BE2000904078000040EB00004F7800F3
:10C600007E409000814F500002003A0010C0B300FD
:10C61000004F78001E04E00008003A007E409000C1
:10C62000604798006E409000E84F500003003E00C5
:10C6300040BE2000EE4090000148780010C0B300DA
:10C640009E4F10000D003A005E4090000081FB00FC
:10C650005E4090008080FB00B0BD20000080400064
:10C66000904078001E40900080C07000B0BD200057
:10C670000000410001487800110037005E40900042
:10C680000082FB005E4090008080FB00B0BD200077
:10C690000080400010407800804178001E419000EA
:10C6A000024078000080EA008180EA0000C061005A
:10C6B00080407800B0BD20000000420001487800B2
:10C6C0001E4078009CA10200000000007E40900007
:10C6D0000040E800704798001E4090000040400075
:10C6E000104798001E4090000004E0000B003A0044
:10C6F0005E4090008080FB00B0BD200000804000C4
:10C7000010407800920007005E4090000040E80072
:10C710005047980010C0B300104798005E4090004A
:10C72000E74F50008CFF3600FE40900000C4B3007D
:10C7300080CF50001000360060BE2000104078000E
:10C740000004E0000C003A0030BE2000EE409000F3
:10C750000148780030BE2000104078000004E0005E
:10C7600003003A0011C0B30050BE20000148780019
:10C7700010C0B300404798004E4090000004E00015
:10C7800004003200B0BD2000104078000004E0003A
:10C790000B003A008040EB0030BE200001487800DA
:10C7A0008040EB0050BE2000014878008040EB0044
:10C7B00040BE2000014878000040EB004047980050
:10C7C0004E4090000080FB00400798004E00900013
:10C7D0000080FA00000006000E00FA000040EB00A6
:10C7E000404798000C0037004E4090000081FB004D
:10C7F0004E4090008080FB00B0BD200000804000D3
:10C800009040780065004700017178004E4090002C
:10C810000040E800404798004E409000E74F50002D
:10C82000F1FF360030BE200090407800214798008C
:10C8300050BE2000904078001147980040BE200074
:10C84000104F780001C4B30030BE200001487800CA
:10C850008040EB0050BE20000148780018FF070020
:10C860000004E0001A00320010C0B3003047980006
:10C870000040EB0040479800110037004E40900008
:10C880008080FB0065004700614178004E409000C9
:10C890008080FB00B0BD2000008040001040780088
:10C8A000804F5100030032000040EB0030479800F9
:10C8B000090037004E4090000040E80040479800D3
:10C8C0004E409000E74F5000ECFF3600020037006A
:10C8D0000040EB00304798000040EB0040479800D4
:10C8E0000C0037004E4090000081FB004E4090004D
:10C8F0008080FB0065004700E1407800B0BD20006B
:10C9000000004100014878004E4090000040E800DF
:10C91000404798004E409000E74F5000F1FF36002E
:10C9200030BE2000AE4090000148780050BE20008C
:10C930009E4090000148780040BE20001E487800CC
:10C940003E4090000080FB000080FA0000000600DE
:10C950000200FA00004F780060BE2000104078000E
:10C960001E4068008080FB00D083200000804000D3
:10C970009040780060BE20000148780060BE200032
:10C98000104078000080FB000080FA0000000600E4
:10C990000000FA0020A62800A47502000000000094
:10C9A0000080FA00000006000400FA00C922A80076
:10C9B000CB22A900C8C2A900C0B520001040780051
:10C9C0000040A000C1B5200080487800C0B520001C
:10C9D000104078000030A100C1B5200080487800E8
:10C9E000EBFF07000000370022C2BF00614060007B
:10C9F0000004E000FCFF320030118000804078002D
:10CA000090B820000148780090B8200010407800CD
:10CA10000080FB004400DE008040780080B82000E9
:10CA20000148780080B82000104078000080FB00AA
:10CA3000100798001E009000E10F500078003200AF
:10CA40009E009000E48F50009D0032001E00900078
:10CA50000000E00001003200A100370090B8200083
:10CA6000104078000080FB00000F78009E007800E6
:10CA7000E28F5000170032001E007800E20F5000D5
:10CA800007003C009E0078000100E00098003200A2
:10CA90001E007800E10F50000C0032005C003700EF
:10CAA0009E007800E48F5000130032001E007800D2
:10CAB000E40F5000560035009E007800688050005A
:10CAC000E10F500052003E0010003700B0FF070099
:10CAD000C5FF3700B8A002000000000080407800C9
:10CAE00060B820000148780010C0B300007A02004E
:10CAF00000000000BCFF3700D6A1020000000000CB
:10CB0000007A020000000000B7FF370010C0B30039
:10CB1000007A02000000000090B820001040780069
:10CB2000E94F500004003A00C1CEB300C08320009A
:10CB3000014878000300370001CFB300C083200014
:10CB4000014878004BFE07008040780060B8200064
:10CB500001487800190037008040EB0070B82000D1
:10CB6000014878000D00370070B8200010407800B0
:10CB70008080FB00B0BD20000080400010407800A5
:10CB8000007A02000000000070B820001040780019
:10CB90008040E80070B820000148780070B820009C
:10CBA00010407800E74F5000EFFF36003FFE0700CF
:10CBB0008040780060B820000148780060B820000C
:10CBC000104078000004E000E3FF3A008040EB00F2
:10CBD00070B82000014878000800370000C0EB0062
:10CBE000007A02000000000070B8200010407800B9
:10CBF0008040E80070B820000148780070B820003C
:10CC000010407800E74F5000F4FF360076FF370001
:10CC10000040EB00007A02000000000072FF3700C5
:10CC200090B8200090407800F0C0B30080C0600051
:10CC300090B820000148780090B82000104078009B
:10CC40008040E80090B820000148780010C0B30090
:10CC5000007A0200000000008040EB0070B8200065
:10CC6000014878000F00370022C2BF006140600019
:10CC70000004E000FCFF3200301180003EA1020001
:10CC80000000000010C0B300007A020000000000A5
:10CC900070B82000104078008040E80070B8200094
:10CCA0000148780070B820009040780090B82000CB
:10CCB0001040780080CF5000EBFF39004AFF37006A
:10CCC00090B8200010407800A2A6020000000000EA
:10CCD00010C0B300007A02000000000042FF3700DD
:10CCE0000040EB00007A0200000000003EFF370029
:10CCF0000080FA00000006000000FA0020A82800CA
:10CD0000A4750200000000000080FA000000060088
:10CD10000000FA000040EB009087020000000000D5
:10CD20000040EB0090870200000000000040EB0094
:10CD300090870200000000000040EB009087020096
:10CD4000000000000000EB00CC86020000000000A4
:10CD50000000EB00CC860200000000000000EB00A9
:10CD6000CC860200000000000080FA0000000600EF
:10CD70000C00FA00C0B52000104078000040A00070
:10CD8000C1B5200080487800C0B520001040780070
:10CD90000030A100C1B520008048780011C0B30068
:10CDA000A0B420000148780081C0B300B0B42000D6
:10CDB0000148780021C0B30030DC20000148780031
:10CDC00080C0EB0020C0B3006C85020000000000B2
:10CDD000C922A900C902A900C8E2A80010C0B30076
:10CDE000FC87020000000000C3FF070000003700BE
:10CDF00022C2BF00614060000004E000FCFF32007E
:10CE0000301180008040780070DC200001487800FC
:10CE100070DC2000104078000080FB004400DE0041
:10CE20008040780060DC20000148780060DC200051
:10CE3000104078000080FB00300798003E00900012
:10CE4000E30F500017013200BE009000E38F500046
:10CE50000A003C003E019000E10F5100A5003200A5
:10CE6000BE019000E18F5100FB003C003E009000AD
:10CE70000000E00012003200E8023700BE0090001F
:10CE8000E68F5000910232003E019000E60F510003
:10CE900004003C00BE019000E48F51008302320088
:10CEA000DE0237003E009000E80F50009E02320084
:10CEB000BE009000EA8F500034013200D7023700E4
:10CEC00070DC2000104078000080FB006101B90098
:10CED0004207980053079800D0002000010020006E
:10CEE0004E019000DE019000800F5100818F5900AB
:10CEF0007C003E004E009000DE00900000600100CB
:10CF0000CA0237000C0037000D003700120037004E
:10CF1000170037001D00370023003700440037009A
:10CF2000480037004C0037005200370058003700E7
:10CF30005E003700640037006FFF0700ACFF37006A
:10CF4000FA8502000000000010C0B300007A020061
:10CF500000000000A6FF37003A8602000000000033
:10CF600010C0B300007A020000000000A0FF3700EC
:10CF70000040EB00FC8702000000000010C0B3007E
:10CF8000007A02000000000099FF370010C0B300D3
:10CF9000FC8702000000000010C0B300007A02000D
:10CFA0000000000092FF370030DC200010407800C5
:10CFB000E24F500006003A00208702000000000007
:10CFC0008040780050DC20000148780006003700DF
:10CFD000F00F20005A860200000000008040780018
:10CFE00050DC200001487800C0B5200010407800D7
:10CFF000684060000004E0000800320050DC2000BF
:10D00000104078000080FB0070A0020000000000CB
:10D010008040780050DC20000148780050DC20007F
:10D0200010407800007A02000000000070FF370016
:10D030006E87020000000000007A0200000000007D
:10D040006BFF37000E88020000000000007A02002B
:10D050000000000066FF370010C0B300B287020076
:10D060000000000010C0B300007A020000000000C1
:10D070005FFF37000040EB00EA870200000000007D
:10D0800010C0B300007A02000000000058FF370013
:10D0900010C0B300EA8702000000000010C0B30017
:10D0A000007A02000000000051FF37000040EB0052
:10D0B000D88702000000000010C0B300007A020010
:10D0C000000000004AFF370010C0B300D8870200FC
:10D0D0000000000010C0B300007A02000000000051
:10D0E00043FF37000040EB00007A02000000000020
:10D0F0003FFF370070DC200090407800F0C0B300A4
:10D1000080C0600070DC20000148780070DC2000E6
:10D11000104078008040E80070DC20000148780072
:10D1200010C0B300007A0200000000008040EB0055
:10D1300050DC2000014878004000370022C2BF00C8
:10D14000614060000004E000FCFF3200301180000C
:10D150008040780040DC200001487800C0B5200005
:10D1600010407800684060000004E00008003200D1
:10D1700040DC2000104078000080FB0070A002001E
:10D18000000000008040780040DC2000014878006A
:10D1900030DC200010407800E24F500009003A00D7
:10D1A00040DC2000104078000080FB00CC860200AC
:10D1B0000000000010C0B300007A02000000000070
:10D1C0001900370040DC2000104078000080FB0090
:10D1D0005A860200000000008040780040DC2000F9
:10D1E00001487800C0B52000104078006840600019
:10D1F0000004E0000800320040DC2000104078000D
:10D200000080FB0070A00200000000008040780059
:10D2100040DC20000148780040DC2000104078000D
:10D22000007A02000000000050DC2000104078006E
:10D230008040E80050DC20000148780050DC2000ED
:10D240009040780070DC20001040780080CF5000C3
:10D25000BAFF3900E6FE370070DC2000904078000D
:10D26000F0C0B30080C0600070DC2000014878008E
:10D2700070DC2000104078008040E80070DC200066
:10D280000148780070DC200010407800B28702006E
:10D290000000000010C0B300007A0200000000008F
:10D2A000D3FE370070DC200090407800F0C0B3005F
:10D2B00080C0600070DC20000148780070DC200035
:10D2C000104078008040E80070DC200001487800C1
:10D2D00010C0B300007A02000000000022C2BF00AC
:10D2E000614060000004E000FCFF3200301180006B
:10D2F0008040780060DC2000014878008040EB002E
:10D3000050DC2000014878001600370060DC200067
:10D31000104078000004E00004003D0010C0B3009D
:10D320009087020000000000030037000040EB007F
:10D33000908702000000000060DC200010407800B0
:10D34000004040008040780060DC20000148780008
:10D3500050DC2000104078008040E80050DC2000C5
:10D360000148780050DC20009040780070DC2000FC
:10D370001040780080CF5000E4FF390010C0B300A7
:10D38000007A02000000000099FE370070DC2000E7
:10D39000104078000080FB0020079800400A200021
:10D3A000AE009000808F500015003200500A20001F
:10D3B0002E019000800F5100C5003200000A2000AD
:10D3C000AE019000808F5100010032003301370020
:10D3D00022C2BF00614060000004E000FCFF320098
:10D3E000301180008040780020DC20000148780067
:10D3F00010C0B300007A0200000000007CFE37007D
:10D4000020DC2000104078000080FB00100798000E
:10D410001E009000E10F5000040032009E009000BA
:10D42000E28F50003B003200A500370022C2BF004F
:10D43000614060000004E000FCFF32003011800019
:10D44000006E8800006E80006300B900006E8800E6
:10D450000000EB00F06D88000C00370022C2BF0016
:10D46000614060000004E000FCFF32007140800079
:10D47000F06D80008080400030118000804878008E
:10D48000F06D80000000E800F06D8800F16D800014
:10D49000006E8000808F5000F0FF39000000EB002C
:10D4A000F06D88001300370071408000F06D80003F
:10D4B000008040000080E80010417800714080004A
:10D4C000F06D8000008040000000E800904178008E
:10D4D00071408000F06D80000080400010407800B6
:10D4E0008340780053010700F06D80006300400026
:10D4F000F06D8800F16D8000006E8000808F50001C
:10D50000E9FF390010C0B300007A020000000000FB
:10D5100037FE370022C2BF00614060000004E00017
:10D52000FCFF320030118000006E8800006E800029
:10D530004200DD00006E88000000EB00F06D880006
:10D540000C00370022C2BF00614060000004E00010
:10D55000FCFF320071408000F06D80008080400050
:10D560003011800080487800F06D80000000E800F5
:10D57000F06D8800F16D8000006E8000808F50009B
:10D58000F0FF39000000EB00F06D88004400370028
:10D590000040EB0090870200000000000040EB001C
:10D5A00090870200000000000040EB00908702001E
:10D5B000000000000040EB00908702000000000027
:10D5C00071408000F06D80000080400010407800C5
:10D5D0000080FB00CC86020000000000714080004B
:10D5E000F06D8000008040000000E80010407800EE
:10D5F0000080FB00CC86020000000000714080002B
:10D60000F06D8000008040000080E800104078004D
:10D610000080FB00CC86020000000000714080000A
:10D62000F06D800000804000630140007140800088
:10D63000F06D8000008040006300400010407800E2
:10D640006F406000004978008040EB0050DC200013
:10D650000148780006003700ADFD070050DC2000CF
:10D66000104078008040E80050DC2000014878003D
:10D6700071408000F06D8000008040006300400039
:10D680009040780050DC20001040780080CF50009F
:10D69000F1FF3E00F06D800064004000F06D8800F6
:10D6A000F16D8000006E8000808F5000B8FF39005F
:10D6B00010C0B300007A020000000000CCFD37006B
:10D6C0000040EB00007A020000000000C8FD3700B7
:10D6D00020DC2000104078000080FB00000F780064
:10D6E0001E017800E10F5100040032009E01780015
:10D6F000E28F510045003200BDFD370022C2BF005D
:10D70000614060000004E000FCFF32003011800046
:10D71000006E880022C2BF00614060000004E0008B
:10D72000FCFF3200301180008040780060DC200077
:10D73000014878000000EB00F06D88002E003700F3
:10D7400060DC20009040780040DC20000148780038
:10D750008040EB0050DC20000148780019003700C1
:10D7600040DC2000104078000080FB006100600079
:10D770000004E0000400320010C0B30090870200F3
:10D7800000000000030037000040EB00908702001B
:10D790000000000040DC2000104078000080FB000A
:10D7A0000000D1008040780040DC20000148780073
:10D7B00050DC2000104078008040E80050DC200061
:10D7C0000148780050DC200010407800E34F500002
:10D7D000E3FF3600208702000000000020870200DF
:10D7E00000000000007A020000000000F06D8000E0
:10D7F0000000E800F06D8800F16D8000006E800090
:10D80000808F5000CEFF390079FD370022C2BF0063
:10D81000614060000004E000FCFF32003011800035
:10D82000006E88000000EB00F06D880016003700E5
:10D8300022C0B30060B92000A10B2000B700070090
:10D84000EA00070022C0B30060BB2D00A10B20003E
:10D85000B200070022C0B300603D2D00A10B2000E4
:10D86000AE000700E100070022C0B30060BB20004B
:10D87000A10B2000A9000700DC000700F06D80006C
:10D880000000E800F06D8800F16D8000006E8000FF
:10D89000808F5000E6FF390055FD37000040EB0057
:10D8A000007A02000000000051FD370070DC20000B
:10D8B00010407800A2A602000000000010C0B300D3
:10D8C000007A02000000000049FD370070DC2000F3
:10D8D0009040780030C0B30080C0600070DC200051
:10D8E0000148780070DC200090407800A0B420004F
:10D8F00001487800A0B420009040780030DC20007F
:10D90000104078006C8502000000000010C0B300D9
:10D91000FC8702000000000010C0B300007A020083
:10D920000000000032FD3700C0B520001040780034
:10D930000040A100C1B520008048780070DC2000C4
:10D94000104078000080FB004300DE000000A200D1
:10D95000610060000004E00005003200C0B5200056
:10D96000104078000040A000C1B520008048780039
:10D9700021C0B30030DC20000148780070DC2000BA
:10D98000104078000080FB004200DE006100600073
:10D990000004E0000300320031C0B30030DC20009E
:10D9A00001487800C0B52000104078000030A10088
:10D9B000C1B520008048780070DC2000104078005D
:10D9C0000080FB000000D100610060000004E00066
:10D9D00005003200C0B52000104078000030A000E3
:10D9E000C1B5200080487800A0B4200090407800A5
:10D9F00030DC2000104078006C8502000000000040
:10DA000010C0B300FC8702000000000010C0B3008B
:10DA1000007A020000000000F5FC37000040EB0037
:10DA2000007A020000000000F1FC37000080FA00DC
:10DA3000000006000600FA002047980031479800D1
:10DA4000424798002E4090000080FB004600DE0018
:10DA5000004F78000040EB0010479800220037008C
:10DA60001E409000E34F50000C003A001E04E000FE
:10DA70000A00320010C0B300EA8702000000000074
:10DA80001E80FB000EA00200000000000040EB0022
:10DA9000EA87020000000000100037002E409000CE
:10DAA0000080FB00610060000004E0000400320020
:10DAB00010C0B30090870200000000000300370090
:10DAC0000040EB0090870200000000002E40900014
:10DAD0000080FB000000D100204798001E4090000D
:10DAE0000040E800104798001E409000E34F5000AF
:10DAF000DBFF36003E4090000080FB00CC86020039
:10DB0000000000004E4090000080FB00CC86020028
:10DB1000000000000080FA00000006000800FA0083
:10DB20001007980021079800624798000040EB001A
:10DB300090870200000000000040EB009087020088
:10DB4000000000000040EB00908702000000000091
:10DB50000040EB0090870200000000001E009000D3
:10DB600070A0020000000000CC860200000000004F
:10DB70001E009000AE0090004809DD004800DE0065
:10DB800000007100C808DE0070A002000000000064
:10DB9000CC860200000000001E009000AE00900045
:10DBA0004008DE000100200070A00200000000001C
:10DBB000CC860200000000006E4090006F406000C4
:10DBC000604798000040EB00004F780002003700EB
:10DBD0004FFC07001E4FE8006E4090009E4F100063
:10DBE000FBFF39000080FA00000006000000FA0088
:10DBF00010C0B30090870200000000000040EB005E
:10DC000090870200000000000040EB0090870200B7
:10DC1000000000000040EB009087020000000000C0
:10DC20000000EB00CC86020000000000208702000C
:10DC300000000000007A02000000000020870200BF
:10DC400000000000007A02000000000030FC070025
:10DC50002FFC07000080FA00000006000200FA0016
:10DC6000905B80000000E0001200320000C2B300B0
:10DC7000007A020000000000310020001044200063
:10DC8000ACA202000000000000C2B300007A020053
:10DC900000000000805B80000000E00003003A000C
:10DCA0000040EB0090870200000000000000EB0045
:10DCB000905B8800805B80000000E00003003A0079
:10DCC0002087020000000000004F780010002000B4
:10DCD000905B88001E80FB000080FA0000000600B8
:10DCE0000400FA00000F7800905B80000000E00064
:10DCF0001200320000C2B300007A020000000000EF
:10DD00003100200010442000ACA2020000000000FE
:10DD100000C2B300007A020000000000805B8000B7
:10DD20000000E00003003A000040EB009087020092
:10DD3000000000000000EB00905B8800805B80002A
:10DD40000000E00007003A001E007800CC860200C8
:10DD5000000000006E870200000000000080FB0051
:10DD6000000F780000C2B300007A0200000000003B
:10DD70001E00E00007003A0031002000104420009F
:10DD8000ACA2020000000000003020001007980044
:10DD9000060037004100200040442000ACA20200F1
:10DDA0000000000000102000100798001E009000E6
:10DDB0000080FA00000006000000FA00905B80007E
:10DDC0000000E0000F00320041002000404420002D
:10DDD000ACA2020000000000E0A42800D075020000
:10DDE00000000000805B80000000E00003003A00BB
:10DDF00010C0B30090870200000000000000EB009C
:10DE0000905B8800805B80000000E0000F003A001B
:10DE1000FA850200000000000000E0000B00320064
:10DE200091002000A0232000ACA20200000000000E
:10DE30005101200030242000ACA2020000000000AC
:10DE4000E0A42800D075020000000000D1002000EE
:10DE50008044200036A30200000000000080FA0089
:10DE6000000006000000FA00905B80000000E00067
:10DE70000F0032004100200040442000ACA202000C
:10DE800000000000E0A42800D0750200000000009F
:10DE9000805B80000000E00003003A0010C0B30087
:10DEA00090870200000000000000EB00905B8800FB
:10DEB000805B80000000E00002003A003A86020029
:10DEC00000000000C10020005045200036A30200E1
:10DED000000000000080FA00000006000000FA00C8
:10DEE0000101200020522000ACA20200000000002E
:10DEF0000040EB003C7802000000000000C2B300CC
:10DF0000007A020000000000A0B420001040780059
:10DF10003C7802000000000000C2B300007A02005A
:10DF200000000000F0A42800D075020000000000EE
:10DF30000080FA00000006000400FA000000EB0078
:10DF4000100798000000EB00805B8800B4210200FD
:10DF500000000000E61D020000000000000F780035
:10DF60001E00E00009003400400020009E0F100059
:10DF700006003C001E0078000040E9008040780068
:10DF8000A0B4200001487800020037000000EB0038
:10DF9000000F78001E00E0002D003A000000EB00AA
:10DFA000F06788000000EB00805B8800805B8000E9
:10DFB0000000E0000F003A00B1032000604820009C
:10DFC00036A30200000000008001EB0042002000A8
:10DFD0001100200010002000E022020000000000DC
:10DFE0000040E90080407800A0B42000014878009B
:10DFF00022003700C140800030002300808F500095
:10E0000004003E0051032000104C2000ACA202008E
:10E0100000000000C1022000604F2000ACA20200FE
:10E02000000000008001EB00320020001100200001
:10E0300010002000E0220200000000000040E90083
:10E0400080407800A0B42000014878000B00370021
:10E05000C140800030002300808F500004003E004B
:10E0600051032000104C2000ACA202000000000070
:10E070009AFF07000000EB00905B8800C0B520000D
:10E08000104078000040A000C1B520008048780012
:10E09000805B80000000E00009003A00C922A8006F
:10E0A000C902A800CB02A900CB22A900A0B420007D
:10E0B0009040780020C0B3006C8502000000000092
:10E0C0000080FA00000006000000FA000000EB00EB
:10E0D000905B8800805B8000E10F500001003A00F7
:10E0E00007E2A9000080FA00000006000600FA001E
:10E0F000100798001E009000200798002E00900046
:10E10000E10F50000C0032002E009000E10F500093
:10E11000040039002E009000E20F5000650032002C
:10E12000730037005103200020532000ACA20200EE
:10E1300000000000720037008040EB00003020003B
:10E140001A88020000000000E10220007056200042
:10E1500036A3020000000000CBC2BF006140600097
:10E160000004E00004003200CBC2BF006240600047
:10E170000004E0000C003A0091002000A0232000E1
:10E18000ACA2020000000000510120003024200059
:10E19000ACA2020000000000E0A42800D07502003C
:10E1A00000000000560037000000EB00000F780070
:10E1B00039003700805B80000000E00009003A0071
:10E1C000FA850200000000001E007800CC860200E4
:10E1D000000000006E870200000000000080FB00CD
:10E1E000100798001E0090000000E00024003A0094
:10E1F0001E007800689F02000000000080C2B3008B
:10E20000007A0200000000001E0078000080D100AB
:10E21000689F0200000000001E0078000000A200BD
:10E22000610060000004E0000400320010A5280036
:10E23000A4750200000000000B003700805B800026
:10E240000000E00005003A00208702000000000006
:10E2500010C0B300908702000000000040A5280015
:10E26000A475020000000000F0A42800A4750200BC
:10E270000000000000C2B300007A020000000000AD
:10E28000805B80000000E00002003A003A86020055
:10E29000000000001E0FE800F00F20009E0F10008D
:10E2A000C4FF3400E0A42800D07502000000000084
:10E2B00013003700805B8000E10F500001003A003E
:10E2C00007E2A900710020005059200036A3020087
:10E2D00000000000F1002000C01E210036A3020053
:10E2E0000000000010C0B3000E000700040037005B
:10E2F00041022000C020200036A3020000000000E0
:10E300000080FA00000006000000FA00B1002000C2
:10E31000C009210036A30200000000000080FA00BE
:10E32000000006000A00FA00004F98000040EB00D1
:10E33000204798000040EB00104798000040EB0099
:10E34000004F7800A87A020000000000C922A8004F
:10E35000C902A800CB02A900CB22A90062A0A80094
:10E3600062C0A8008660A900CBC2BF000080FB008D
:10E370000000D10061406000604798006E4090004E
:10E3800050479800CBC2BF006140600060479800D2
:10E390006E409000304798000000370086C0BF00F4
:10E3A000684060000004E00012003A0023C2BF0091
:10E3B000624060000004E0000E003A00F27A0200C1
:10E3C0000000000022C2BF00614060000004E000C5
:10E3D000F2FF320030118000004F780062A0A900E7
:10E3E00062C0A9000E4890000004E00061003A00FD
:10E3F000630037008660A900CBC2BF000080FB002D
:10E400000000D1006140600060479800CBC2BF00AF
:10E4100061406000404798002E4090000004E000FA
:10E420002E0032003E4090000004E0002B003A0035
:10E430004E4090000004E000280032001E40900092
:10E44000E74F50000B003E001E40780000404000A7
:10E45000004F78006E4090000004E00001003200A0
:10E460001E04A0001E4090000040E80010479800E5
:10E470003B0037000E4890000004E000040032002A
:10E480001E80FB00C8780200000000000600370074
:10E49000C0C5B300BC7A0200000000001E40780036
:10E4A000BC7A0200000000006E4090000004E00012
:10E4B00004003200D0C2B300BC7A020000000000A9
:10E4C00003003700B0C2B300BC7A020000000000B5
:10E4D0000040EB0010479800210037003E409000BC
:10E4E0000004E0001E0032004E4090000004E000F6
:10E4F0001B0032005E4090000004E0000B00320080
:10E500006E4090000004E00008003A0010C0B30024
:10E51000204798000040EB0010479800B0C5B300BA
:10E52000BC7A0200000000000D0037005E40900041
:10E530000004E0000A003A006E4090000004E00091
:10E54000070032000040EB00204798000040EB003D
:10E5500010479800D0C5B300BC7A0200000000004C
:10E560006E409000504798004E4090003047980011
:10E570008AFF3700E0A42800D075020000000000E8
:10E580000080FA00000006000000FA0070A52800D4
:10E59000A4750200000000000080FA0000000600E0
:10E5A0000A00FA00881F7800C922A800C902A80042
:10E5B000CB02A900CB22A900C8C2A900C0B5200087
:10E5C000104078000040A000C1B5200080487800CD
:10E5D000C0B52000104078000030A100C1B5200077
:10E5E0008048780080C0EB0020C0B3006C8502003A
:10E5F00000000000E4FF07000000370022C2BF0057
:10E60000614060000004E000FCFF32003011800037
:10E6100080407800E0B6200001487800E0B6200095
:10E62000104078000080FB004400DE00804078004D
:10E63000D0B6200001487800D0B620001040780005
:10E640000080FB00400798004E009000E10F500052
:10E65000EB0032004E009000E10F500004003C003F
:10E660004E0090000000E000080032002401370056
:10E670004E009000E40F5000190132004E0090004F
:10E68000E60F5000070132001D013700E0B6200000
:10E69000104078000080FB00300798003E0090009A
:10E6A000E40F5000330032003E009000E40F5000B1
:10E6B00011003C003E009000E10F50001F003200AE
:10E6C0003E009000E10F500004003C003E0090002E
:10E6D0000000E0000E013200C50037003E0090004F
:10E6E000E20F5000170032003E009000E30F500090
:10E6F0001A003200BE0037003E009000E70F5000C5
:10E70000280032003E009000E70F500004003C005B
:10E710003E009000E60F50001B003200B4003700AE
:10E720003E009000E80F5000250032003E009000AF
:10E73000EF0F5000A8003200AD00370092FF070035
:10E74000AEFF3700FA8502000000000010C0B300E1
:10E75000007A020000000000A8FF37003A8602009D
:10E760000000000010C0B300007A020000000000AA
:10E77000A2FF37002087020000000000007A02009C
:10E78000000000009DFF37000040EB009087020072
:10E790000000000010C0B300007A0200000000007A
:10E7A00096FF370010C0B300908702000000000001
:10E7B00010C0B300007A0200000000008FFF370095
:10E7C00022C2BF00614060000004E000FCFF320094
:10E7D00030118000100798001E0090004800DD00F6
:10E7E0001007980022C2BF00614060000004E000F2
:10E7F000FCFF3200301180009E009000008070000D
:10E800001007980022C2BF00614060000004E000D1
:10E81000FCFF320030118000000F78001E007800ED
:10E820004800DD00000F780022C2BF006140600098
:10E830000004E000FCFF3200301180001E0F700069
:10E840009E00900000002100808F500003003E00D9
:10E85000000021009E0F1000040036000040EB0075
:10E86000007A02000000000064FF37000000EB00A7
:10E87000200798000C00370022C2BF0061406000F2
:10E880000004E000FCFF3200714080002E00900088
:10E890008080400030118000804878002E00900079
:10E8A0000000E80020079800AE0090001E009000D5
:10E8B000808F5000F0FF3900FA8502000000000050
:10E8C0000000EB00200798000E0037007140800028
:10E8D0002E00900000804000104078000080FB0077
:10E8E000CC860200000000006E87020000000000DD
:10E8F000E14F5000D9FF32002E0090000000E800E8
:10E9000020079800AE0090001E009000808F5000FD
:10E91000EEFF39001E00E900100798000000EB0030
:10E920002007980014003700714080002E009000EE
:10E93000008440002087020000000000004C7800A6
:10E94000AE0090001E009000808F50000400310047
:10E950000040EB0090870200000000000300370039
:10E9600010C0B30090870200000000002E0090004D
:10E970000000E800200798002E0090009E0F500035
:10E98000E9FF39003A8602000000000010C0B30021
:10E99000007A0200000000000000EB002007980051
:10E9A00009003700714080002E0090000080400078
:10E9B00010407800007A0200000000002E00900055
:10E9C0000000E800200798002E0090009E0F5000E5
:10E9D000F4FF390009FF37000040EB0051FE07004B
:10E9E00010C0B300007A02000000000003FF3700EF
:10E9F0000040EB00007A020000000000FFFE37003C
:10EA0000E0B6200090407800F0C0B30080C0600005
:10EA1000E0B6200001487800E0B620001040780001
:10EA20008040E800E0B620000148780010C0B30044
:10EA3000007A0200000000008040EB00C0B6200019
:10EA4000014878001000370022C2BF00614060001A
:10EA50000004E000FCFF320030118000CC86020090
:10EA6000000000006E87020000000000007A020033
:10EA700000000000C0B62000104078008040E80090
:10EA8000C0B6200001487800C0B620009040780051
:10EA9000E0B620001040780080CF5000EAFF390037
:10EAA000D6FE3700E0B620009040780030C0B300BA
:10EAB00080C06000E0B6200001487800E0B6200089
:10EAC0009040780020C0B3006C8502000000000078
:10EAD00010C0B300007A020000000000C7FE37003B
:10EAE000E0B6200010407800A2A60200000000005E
:10EAF00010C0B300007A020000000000BFFE370023
:10EB00000040EB00007A020000000000BBFE37006E
:10EB10004F0478000080FA00000006000200FA00AE
:10EB2000000F78001E00E0000300320010C3B300A5
:10EB3000330207000200370000C3B30030020700B1
:10EB40000080FA00000006000600FA001007980096
:10EB5000020037001E407800290207001E009000C6
:10EB6000104F78001E407800404798004E409000BB
:10EB70000004E0000200320010C0B30040479800DB
:10EB80004E4090009E0090008100E8001107980020
:10EB90000004E000EFFF3A000080FA0000000600E9
:10EBA0000600FA0010079800020037001E407800A7
:10EBB000130207001E009000104F78001E407800DE
:10EBC000404798004E4090000004E00002003200F0
:10EBD00010C0B300404798004E4090009E00900047
:10EBE0008100E800110798000004E000EFFF3A0000
:10EBF000D0C0B30002020700A0C0B30000020700AB
:10EC00000080FA00000006000400FA002047980087
:10EC100000C8B300004F780080A12800CAFF070099
:10EC20000040EB00104798000F0037002E40900086
:10EC30001E4060000004E0000300320010C3B30077
:10EC4000EF0107000200370000C3B300EC0107002A
:10EC50001E80FB000000D100004F78001E40900095
:10EC60000040E800104798001E409000E74F500019
:10EC7000EEFF36000080FA00000006000E00FA00E9
:10EC800050079800610798000040EB00004F7800A3
:10EC900000102E00515F20003007980041079800B7
:10ECA0000040EB0010479800320037003E01900012
:10ECB000CE0190005E009000EE009000240602005D
:10ECC0000000000010079800210798001E04E000D3
:10ECD00005003A001E009000AE009000E00F5000CA
:10ECE000E08F5800180032001E0090000043B00072
:10ECF000C30107009E0090003E009000000AB8008B
:10ED00009E0090004E0090000088B9000501780038
:10ED100000014100BE0090002E0090000088B90064
:10ED200000014100820278005E009000EE00900039
:10ED30000400500085805800500798006107980033
:10ED400010C0B300004F78003E009000CE0090004D
:10ED5000A2002000030020002406020000000000A2
:10ED600030079800410798001E4090000040E800DE
:10ED7000104798001E409000E74F5000CBFF360030
:10ED80005E0090000043B0009D0107000080FA0083
:10ED9000000006000C00FA00400798005107980098
:10EDA0000000EB00100798000000EB00000F780057
:10EDB0006000B80020079800310798004E019000CD
:10EDC000DE019000F0232400F1002000800F5100AC
:10EDD000818F5900210036004E009000DE00900027
:10EDE00002242400F300200024060200000000009A
:10EDF00020079800310798002E0090006F00070050
:10EE0000C0C2B3007E0107004E009000DE009000FB
:10EE100002242400F3002000440602000000000049
:10EE200040079800510798004E019000DE019000C5
:10EE3000703E200001002000800F5100818F59009A
:10EE400002003E00B0A128003FFF07001000200094
:10EE50001007980010002000000F78004E0190006D
:10EE6000DE019000703E200001002000800F510064
:10EE7000818F5900320036004E009000DE00900075
:10EE8000823E200003002000240602000000000053
:10EE900020079800310798002E019000BE019000D5
:10EEA0004006200001002000800F5100818F590092
:10EEB000030036002E0090004000070014003700C9
:10EEC0001E0090000000E0000F0032002E019000B4
:10EED000BE019000A000200001002000800F510022
:10EEE000818F59000300360000C3B30044010700BE
:10EEF0000200370000A2280013FF07002E00900038
:10EF00002E000700020037002E0090002B000700A3
:10EF1000C0C2B3003A0107004E009000DE0090002E
:10EF2000823E200003002000440602000000000092
:10EF3000400798005107980010002000000F78004B
:10EF40004E019000DE0190004006200001002000EC
:10EF5000800F5100818F5900030036004E00900051
:10EF600016000700130037001E00E0000F003200FB
:10EF70004E019000DE019000A00020000100200062
:10EF8000800F5100818F59000300360000C3B30089
:10EF90001B0107000200370000A22800EAFE07005C
:10EFA0004E00900005000700020037004E00900060
:10EFB000020007000080FA00000006000800FA00C6
:10EFC000300798000040EB00004F780000712200ED
:10EFD000200798000040EB00104798001E00370003
:10EFE0003E0090002E019000110009000280D80020
:10EFF000100798001E04E00003003A001E00900075
:10F000000000E0000C0032001E0090000043B00041
:10F01000FB0007009E0090002E0090000088B900C1
:10F02000800078003E0090000100500030079800FA
:10F0300010C0B300004F78002E009000A200200006
:10F04000110009000280D800200798001E4090009F
:10F050000040E800104798001E409000E34F500029
:10F06000DFFF36003E0090000043B000E4000700E0
:10F070000080FA00000006000600FA0040479800F1
:10F080000040EB00004F780040C6B30030479800C6
:10F090000040EB0020479800200037004E409000D1
:10F0A0008080FB003E4090000081FB0011000900C1
:10F0B0008280D800104798001E04E00003003A0048
:10F0C0001E4090000004E0000B0032001E40900043
:10F0D0000043B000CA0007004E4190009E409000DF
:10F0E0003E4090000088B900004051004047980021
:10F0F00010C0B300004F78003E4090000080FB003D
:10F10000A2002000110009000280D80030479800BA
:10F110002E4090000040E800204798002E409000CC
:10F12000E14F5000DDFF36004E4090000043B0003C
:10F13000B30007000080FA00000006000400FA0097
:10F140001007980030A328007FFE07001E009000E3
:10F150004400DE006F0F60009E00780030A228009F
:10F160000080400010407800A50007001E009000BD
:10F170006F0F60009E00780030A2280000804000E1
:10F18000104078009E0007000080FA000000060092
:10F190000400FA001007980000C3B300F60007004F
:10F1A00080C7B300F40007001E0090004400DE009A
:10F1B0006F0F60009E00780030A2280000804000A1
:10F1C00010407800EC0007001E0090006F0F6000F8
:10F1D0009E00780030A22800008040001040780097
:10F1E000E50007000080FA00000006000400FA00B5
:10F1F0001007980030A3280053FE07001E0090005F
:10F200004C00DE006F0F60009E00780030A22800E6
:10F210000080400010407800790007001E00900038
:10F220004800DE006F0F60009E00780030A22800CA
:10F230000080400010407800710007001E00900020
:10F240004400DE006F0F60009E00780030A22800AE
:10F250000080400010407800690007001E00900008
:10F260006F0F60009E00780030A2280000804000F0
:10F2700010407800620007000080FA0000000600DD
:10F280000800FA00300798003E009000CF80DE00B2
:10F29000E803020000000000926C2200B331240059
:10F2A00046040200000000001007980021079800A3
:10F2B0001E009000AE0090004A0602000000000010
:10F2C000004F78001E4078006BFF0700E0C2B300DB
:10F2D0004B0007001E009000AE0090004A0602009E
:10F2E00000000000CF80DE00E80302000000000004
:10F2F0000001BE001E009000AE009000CA04020093
:10F30000000000001007980021079800020020006C
:10F31000031224001E009000AE009000860502003B
:10F320000000000010079800210798001E009000C0
:10F33000AE0090004A06020000000000004F780076
:10F340001E4078004CFF07001E009000AE009000A9
:10F350004A06020000000000CF80DE00E803020041
:10F36000000000000001BE001E009000AE009000F2
:10F37000CA0402000000000010079800210798004E
:10F3800002002000031224001E009000AE00900036
:10F390008605020000000000100798002107980071
:10F3A0001E009000AE0090004A060200000000001F
:10F3B000004F78001E4078002FFF07000080FA0001
:10F3C000000006000000FA0022C2BF006140600099
:10F3D0000080FB000080FA00000006000000FA0038
:10F3E00022C2BF00614060000004E000FCFF320068
:10F3F000301180000080FB000080FA000000060051
:10F400000200FA00004F7800D04080000110200078
:10F41000010060000000E00006003A0023C2BF00C7
:10F42000624060000004E000FCFF3A001E00FB00A8
:10F43000201188000080FA00000006000200FA0097
:10F44000004F78001E80FB00401188000080FA0009
:10F45000000006000000FA0095C0BF007040600088
:10F460000004E00010003A0051408000404080005D
:10F47000808F50000C00320023C2BF006240600049
:10F480000004E000FCFF3A008580A9009580A800F8
:10F4900031408000404080000080400010407800F3
:10F4A0000080FB00201188000080FA0000000600A8
:10F4B000809FBE000000FA000140800020408000D4
:10F4C000808040003011800080487800204080001B
:10F4D0000000E800204088002140800010408000AB
:10F4E000808F500001003A009560A9008560A90056
:10F4F0000080FA004F00BE0000400600809FBE0062
:10F500000000FA00404080000000E8004040880011
:10F510004140800050408000808F500002003A003F
:10F520009580A900060037003140800040408000EF
:10F5300000804000104078000080FB00201188000F
:10F540008580A9000080FA004F00BE000040060040
:10F550000000FA000000EB00206D88001000200081
:10F56000106D8800D040800000A0A100D04088002D
:10F570000080FA00000006000200FA00004F780048
:10F58000116D8000206D8000808F500005003A00D2
:10F59000C222A900D040800000A0A000D040880076
:10F5A0000E00370071408000106D800080804000A8
:10F5B0001E40780080487800106D80000000E80050
:10F5C000106D8800116D800000002100808F5000B8
:10F5D00002003A000000EB00106D88000080FA0085
:10F5E000000006000200FA00206D8000000FE80015
:10F5F000000021009E0F100002003A000000EB0006
:10F60000000F7800106D80009E0F10000C0032007B
:10F6100023C2BF00624060000004E00008003A001E
:10F620001E007800206D880071408000206D8000F1
:10F6300000804000104078000080FB00201188000E
:10F640000080FA00000006000200FA000000370007
:10F65000206D8000000FE800000021009E0F1000C8
:10F6600002003A000000EB00000F7800106D8000EF
:10F670009E0F10000D00320023C2BF0062406000E8
:10F680000004E000F2FF3A001E007800206D8800C0
:10F6900071408000206D80000080400010407800A4
:10F6A0000080FB0020118800E9FF37000080FA008D
:10F6B000000006000800FA002007980031079800B3
:10F6C00090018000100798002E00900090018800A3
:10F6D0003E0090001080BA00C800DD003E0090009F
:10F6E0001000BA00008F70001E009000900188008A
:10F6F0001E0078000080FA00000006000000FA00FA
:10F70000C0A72800A4750200000000000080FA00D5
:10F71000000006000200FA00C222A800080107004B
:10F72000F6FF070000003700FC000700804078006B
:10F73000A0DB200001487800A0DB2000104078000A
:10F740000004E000EF003500A0DB2000104078004E
:10F750000004E00002003A00E8FF0700F2FF370073
:10F76000A0DB200010407800E14F500006003A0076
:10F77000F3000700F250020000000000F000070054
:10F78000DEFF0700E8FF3700A0DB20001040780014
:10F79000E24F500006003A00E9000700D072020074
:10F7A00000000000E6000700D4FF0700DEFF37007E
:10F7B000A0DB200010407800E34F500006003A0024
:10F7C000DF000700DE59020000000000DC00070037
:10F7D000CAFF0700D4FF3700A0DB200010407800EC
:10F7E000E44F500006003A00D5000700D464020040
:10F7F00000000000D2000700C0FF0700CAFF37006A
:10F80000A0DB200010407800E54F500006003A00D1
:10F81000CB000700B866020000000000C800070027
:10F82000B6FF0700C0FF3700A0DB200010407800C3
:10F83000E64F500004003A00C1000700C000070076
:10F84000AEFF0700B8FF3700A0DB200010407800B3
:10F85000E74F500004003A00B9000700B800070065
:10F86000A6FF0700B0FF3700A0DB200010407800A3
:10F87000EF4F50000A003A0010C0B300007A0200B7
:10F8800000000000C222A90023C2BF006140600046
:10F890000004E000FCFF32000000FE00A2FF370081
:10F8A000A0DB200010407800F04F500003003A0029
:10F8B0000040EB00DF0107009BFF3700A0DB2000CA
:10F8C00010407800F14F500003003A0010C0B30020
:10F8D000D801070094FF3700A0DB2000104078001B
:10F8E000F24F500035003A000000EB00800888001D
:10F8F0000000EB00F00888000000EB00E00C88003E
:10F90000A16C20009140780000CEB30000C06000E0
:10F910006041B300CAE6B700800007000080FB002A
:10F92000000F78001E0078000000D1006100600028
:10F930000004E0000100320010A1A8009E00780041
:10F94000618060000004E000010032001081A80026
:10F95000720007000080FB004800DD00000F780007
:10F960006E0007000080FB001E0F70001E00780074
:10F97000D00C88009E007800C10C88006000200038
:10F98000E00C8800650007000080FB004800DD00F7
:10F99000000F7800610007000080FB001E0F700060
:10F9A0001E0078006008880011E1A80010C0B300B4
:10F9B000007A0200000000005BFF3700A0DB20009F
:10F9C00010407800F34F50000D003A000000EB00AB
:10F9D000800888000000EB00E00C8800A16C20008B
:10F9E0009140780000CEB30000C06000CAE6B700C6
:10F9F00010C0B300007A0200000000004AFF370088
:10FA0000A0DB200010407800F44F50000E003A00B8
:10FA100021E3A800C0C0B300B09E020000000000B7
:10FA2000000F780021E3A9001E0078004800DE00E6
:10FA3000007A0200000000001E007800007A020038
:10FA40000000000038FF3700A0DB200010407800E5
:10FA5000F54F500018003A0021E3A800C0C0B300E1
:10FA6000B09E020000000000000F780023C2BF001B
:10FA7000614060000004E000FCFF32001E007800DE
:10FA80004800DE00007A0200000000001E0078003E
:10FA9000007A02000000000022C2BF006140600046
:10FAA0000004E000EDFF320031118000010F78000A
:10FAB00021E3A9001CFF3700A0DB200010407800E4
:10FAC0000080FB004500DE000080FB000000D1004C
:10FAD000610060000004E00006003200A0DB2000AE
:10FAE000104078001D000700007A020000000000AE
:10FAF0000DFF37000040EB00007A0200000000001C
:10FB000009FF3700A0DB200010407800A3000700A9
:10FB1000007A02000000000003FF37000000FA0036
:10FB200022C2BF00614060000004E000FCFF320020
:10FB3000301180000080FB000080FA000000060009
:10FB40000000FA0000C0EB00040007000040EB00DA
:10FB5000920007000080FA00000006000400FA008E
:10FB6000204798000040EB00004F78002E409000A6
:10FB70000080FB004400DE00610060000004E00043
:10FB80000200320010C0B300004F78009E407800A1
:10FB900061C06000614060004201DD00912C2000E6
:10FBA00091407800B0CFB30000C060000240700008
:10FBB000C9E2B7000040EB00004F78002E409000F3
:10FBC0000080FB004300DE00610060000004E000F4
:10FBD0000200320010C0B300004F78009E40780051
:10FBE00061C060006140600000414000912C200035
:10FBF00091407800D0CFB30000C060000240700098
:10FC0000C9E2B7000040EB00004F78002E409000A2
:10FC10000080FB004200DE00610060000004E000A4
:10FC20000200320010C0B300004F78009E40780000
:10FC300061C0600061416000912C2000914078001B
:10FC4000E0CFB30000C0600002407000C9E2B7001E
:10FC50000040EB00004F78002E4090000080FB0039
:10FC60000000D100610060000004E00002003200EA
:10FC700010C0B300004F78009E40780061C0600063
:10FC8000C700DD00C8C2BF000074A10001407000C1
:10FC9000C8E2B7000040EB00004F78002E40900013
:10FCA0000080FB00610060000004E0000200320000
:10FCB00010C0B300004F78009E40780061C0600023
:10FCC000614060004601DD00812C200091407800F9
:10FCD000F0CBB30000C0600002407000C8E2B70083
:10FCE000500020003AA0020000000000AE4090004A
:10FCF00000CEB30000C0600020479800CBC2BF0018
:10FD0000644060000004E000030032002E409000D8
:10FD10000044A00020479800CBC2BF0062406000B2
:10FD20000004E000030032002E4090000034A000E8
:10FD300020479800CBC2BF00614060000004E00093
:10FD4000030032002E4090000024A00020479800BD
:10FD5000CAC2BF0001C8B300014060000004E00057
:10FD6000030032002E4090000014A00020479800AD
:10FD7000CAC2BF000044B2000004E0000300320029
:10FD80002E4090000004A000204798002E409000D4
:10FD90000080FB000080FA00000006000400FA006A
:10FDA000204798002E4090000080FB004600DE00B7
:10FDB000610060000004E00003003200C002A900FE
:10FDC000C202A80002003700C002A900C202A900B6
:10FDD0002E4090000080FB004500DE0061006000C6
:10FDE0000004E00003003200C962A800CB62A90051
:10FDF00002003700CB62A900C962A9000040EB00F5
:10FE0000004F78002E4090000080FB004400DE0090
:10FE1000610060000004E0000200320010C0B30086
:10FE2000004F78009E40780061C060006140600033
:10FE30004201DD00B12C200091407800B0CFB3002A
:10FE400000C0600002407000CBE2B7000040EB0051
:10FE5000004F78002E4090000080FB004300DE0041
:10FE6000610060000004E0000200320010C0B30036
:10FE7000004F78009E40780061C0600061406000E3
:10FE800000414000B12C200091407800D0CFB30059
:10FE900000C0600002407000CBE2B7000040EB0001
:10FEA000004F78002E4090000080FB004200DE00F2
:10FEB000610060000004E0000200320010C0B300E6
:10FEC000004F78009E40780061C060006141600092
:10FED000B12C200091407800E0CFB30000C060005A
:10FEE00002407000CBE2B7000040EB00004F78000A
:10FEF0002E4090000080FB000000D10061006000F7
:10FF00000004E0000200320010C0B300004F78008F
:10FF10009E40780061C06000C700DD00CAC2BF001B
:10FF20000074A10001407000CAE2B7000040EB007D
:10FF3000004F78002E4090000080FB0061006000C0
:10FF40000004E0000200320010C0B300004F78004F
:10FF50009E40780061C06000614060004601DD00A5
:10FF6000A12C200091407800F0CBB30000C06000CD
:10FF700002407000CAE2B700500020003AA0020020
:10FF800000000000AE40900000CEB30000C0600052
:10FF900020479800CBC2BF00644060000004E0002E
:10FFA000030032002E4090000044A000204798003B
:10FFB000CBC2BF00624060000004E00003003200DA
:10FFC0002E4090000034A00020479800CBC2BF0014
:10FFD000614060000004E000030032002E40900009
:10FFE0000024A00020479800CAC2BF0001C8B30087
:10FFF000014060000004E000030032002E40900049
:020000040001F9
:100000000014A00020479800CAC2BF000044B200FC
:100010000004E000030032002E4090000004A00025
:10002000204798002E4090000080FB000080FA00DE
:10003000000006000400FA0020479800AE4090003F
:100040000040EB00869B0200000000001047980073
:100050001E4090000004E00001003200C222A8000F
:100060001E409000007A02000000000000003700EF
:10007000E2790200000000000004E0000F003200FE
:10008000EE79020000000000004F780000C0EB0095
:100090009E4F1000050032001E4090001E404000A0
:1000A000007A0200000000000400370010C0B30016
:1000B000007A0200000000001A0037001E40900085
:1000C0000004E000EAFF3A00E06D80000000E0007C
:1000D00010003A000080EB00E06D8800C2C2BF0053
:1000E0000080FB000000D100614060000004A2001D
:1000F000614060006140600000414000212C200010
:1001000091407800D0CFB30000C060000240700082
:10011000C2E2B700E06D80000000E900E06D8800F9
:10012000D3FF37000080FA00000006000600FA0046
:100130000000EB00800888000000EB00F008880059
:100140000000EB00E00C8800B05F80000000E000E1
:1001500008003A00A16C20009140780000CEB30066
:1001600000C06000CAE6B7000000EB00405F8800F6
:100170003D003700B05F8000E30F500005003C00F9
:10018000E0032000000F780010A1A8001081A80053
:1001900015003700B05F8000FE0F500005003C00E6
:1001A000A00F2000000F780010A1A8001081A90066
:1001B0000D003700B15F8000400F2000808F50009D
:1001C00005003C00007D2000000F780010A1A90070
:1001D0001081A8000400370000E82300000F780019
:1001E00010A1A9001081A900B05F80000001780073
:1001F0001E007800110009000280D8000000E9000C
:10020000200798002E00900060088800C05F8000E2
:10021000800078002E0090000088B900420620007F
:10022000110009000280D80010079800A16C20007E
:100230009140780000CEB30000C060006041B30080
:10024000CAE6B7001E009000D00C88001E00900087
:10025000C00C880060002000E00C880011E1A800BC
:1002600020002000405F88000080FA0000000600A7
:100270001200FA000000EB00800888000000EB008C
:10028000F00888000000EB00E00C8800405F800070
:10029000E20F500014003A00A16C20009140780059
:1002A00000CEB30000C06000CAE6B700C100200065
:1002B000C02E200036A30200000000000000EB006A
:1002C000405F8800E06780008000E800F00F2000B9
:1002D00080806000A0BF20000080400010407800B7
:1002E0000004E000AC0032000000EB0020079800A2
:1002F000E06780008000E800F00F200000806000D0
:10030000E0678800B421020000000000E61D020042
:100310000000000040079800B42102000000000027
:10032000E61D020000000000CF80DE00E8030200AE
:1003300000000000008FBE004E0090000000E000B2
:1003400007003200CE009000F0F92000808F5000AE
:1003500003003E002E0090000000E80020079800F7
:100360006011B8001E00BE003E0402000000000044
:100370000000E00001003C000B00370002002000FC
:10038000832C24001E00BE00420402000000000076
:100390000000E00001003500030037002E0090004F
:1003A0000000E800200798002E009000E20F5000A7
:1003B000110032000000EB00F067880011012000FE
:1003C000802F200036A30200000000001101200051
:1003D00090302000ACA20200000000008001EB0081
:1003E00002FA20001100200020032000E022020079
:1003F00000000000400798004E009000E30F5000FE
:1004000005003E00E00320003007980010A1A8007E
:100410001081A800150037004E009000FE0F50001C
:1004200005003E00A00F20003007980010A1A80092
:100430001081A9000D003700CE009000400F200071
:10044000808F500005003E00007D2000300798009E
:1004500010A1A9001081A8000400370000E82300C3
:100460003007980010A1A9001081A9003E0090005B
:100470004E019000110009000280D8000000E90040
:10048000600798002E009000E20F50000E0032002E
:100490000101200070322000ACA202000000000028
:1004A0008001EB00320620008000EB0020032000DA
:1004B000E022020000000000CF80DE00E80302001E
:1004C00000000000008FBE0002002000832C2400EA
:1004D0001E00BE004604020000000000008FBE00A7
:1004E0006E009000CF80DE00E803020000000000F4
:1004F00070079800010F98006E0090000000E00067
:1005000008003D0002002000037824007E009000D7
:100510008E089000CC0402000000000070079800D4
:10052000010F98001E01BE007E0090008E08900012
:100530008605020000000000EE0502000000000039
:1005400050079800A16C20009140780000CEB300C5
:1005500000C060006041B300CAE6B7005E009000D2
:10056000D00C88005E009000C00C88006000200065
:10057000E00C88006E0090006008880011E1A8007F
:10058000A10020007033200036A30200000000000C
:1005900020002000405F88000080FA000000060074
:1005A0000000FA00405F8000E20F500005003A00B2
:1005B000F10120001034200036A3020000000000EA
:1005C0003E003700F100200000362000ACA20200FF
:1005D000000000000000EB00F00888000000EB00C5
:1005E00080088800C942A800616820009140780016
:1005F00000CEB30000C06000A040B30086E6B700A4
:10060000A0032000800888002E000700505F8800AB
:10061000615F8800525F8000635F8000F00F200000
:1006200001002000800F5100818F59000900360021
:10063000505F8000615F8000C808DD000080FD0021
:10064000804078000040EB00505F8800615F8800C8
:1006500009003700B1002000B0192100ACA202004F
:1006600000000000A000200080088800150007009E
:10067000505F8800615F8800505F8000615F80008C
:10068000CA7602000000000000A72800A47502003E
:100690000000000040A72800D07502000000000004
:1006A00086C6BF00F041B30086E6B7000000EB004D
:1006B000F00888000000EB00800888000080FA0045
:1006C000000006000000FA000080EB0070088800BF
:1006D0000080EB00600888000000EB004008880004
:1006E0000000EB00300888000000EB00B008880034
:1006F0000000EB00A008880080002000F0088800BF
:10070000400F2000E008880000402200D008880048
:100710008780A9001FE1A80011E1A80087C0BF00E1
:10072000704060000004E000FCFF320011E1A9000D
:100730001FE1A90030088000A05F88004008800009
:10074000905F8800905F800001002000705F88004B
:10075000815F8800705F8000815F8000C000DD00E5
:1007600000002000705F8800815F8800A05F80002B
:100770006101B800705F8000815F8000020040006E
:1007800083804800705F8800815F8800705F800010
:10079000815F80000080FA00000006000000FA007F
:1007A000C0B5200010407800634060000004E00005
:1007B00002003A00C942A80001003700C8C2A800E0
:1007C000E1002000F0362000ACA202000000000092
:1007D0000080FA00000006000000FA00C0B520000A
:1007E00010407800634060000004E00003003A001D
:1007F000C942A900CB42A80002003700C8C2A90024
:10080000CAC2A80081002000D037200036A3020011
:10081000000000000080FA00000006000000FA005E
:10082000C0B5200010407800634060000004E00084
:1008300003003A00C942A900CB42A90002003700D8
:10084000C8C2A900CAC2A900710020005038200007
:1008500036A30200000000000080FA00000006003D
:100860000200FA00C0B5200010407800634060002C
:100870000004E00009003A00C942A800000000009E
:1008800000000000CBC2BF000080FB004200DE0081
:1008900061406000004F780008003700C8C2A8001F
:1008A0000000000000000000CAC2BF000080FB0082
:1008B0004600DE0061406000004F78001E80FB00B3
:1008C0000080FA00000006000C00FA000000EB00B7
:1008D000800888000000EB00F00888000000EB00B2
:1008E000E00C8800405F8000E20F500014003A00E6
:1008F000A16C20009140780000CEB30000C06000E1
:10090000CAE6B700C1002000C02E200036A30200B6
:10091000000000000000EB00405F8800E0678000FE
:100920008000E800F00F200080806000A0BF200061
:1009300000804000104078000004E00064003200B5
:10094000E06780008000E800F00F20000080600079
:10095000E0678800B421020000000000E61D0200EC
:1009600000000000CF80DE00E8030200000000006D
:10097000008FBE00F06780000000E00008003A0031
:1009800002002000433324001E00BE003E0402008B
:10099000000000000000E00001003C0010003700F3
:1009A0000000EB00F06788003101200040242100A6
:1009B00036A30200000000008001EB00420B200083
:1009C0008000EB00A0052000E022020000000000F3
:1009D000CF80DE00E803020000000000008FBE00B0
:1009E00010A1A8001081A800204E20003007980018
:1009F00002002C00A35524001E00BE004604020085
:100A000000000000008FBE003E009000CF80DE009E
:100A1000E80302000000000040079800510798001A
:100A20003E0090000000E00008003D0002002000B1
:100A3000037824004E009000DE009000CC040200F9
:100A40000000000040079800510798001E01BE00FA
:100A50004E009000DE0090008605020000000000BD
:100A60000200200083272400CC04020000000000C4
:100A7000EE0502000000000020079800A16C200095
:100A80009140780000CEB30000C060006041B30028
:100A9000CAE6B7002E009000D00C88002E0090000F
:100AA000C00C880060002000E00C88003E00900030
:100AB0006008880011E1A800C10020007025210015
:100AC00036A302000000000020002000405F8800E4
:100AD0000080FA00000006000400FA00004F7800D1
:100AE0001147980000DB20001E48780030C0B3009A
:100AF0009E4F100005003A0000202000906D8800F5
:100B000000082000A06D88000400370000202000AD
:100B1000906D880000202000A06D88001E4090008D
:100B20000080FB00100798001E009000E10F5000AD
:100B3000110032001E009000E20F50001800320039
:100B40001E0090000000E000010032001E0037008F
:100B500041C1B30060DB20000148780041C6B3000A
:100B600070DB20000148780021C3B30080DB200047
:100B7000014878001D00370021C0B30060DB200071
:100B800001487800A1C0B30070DB20000148780064
:100B900051C0B30080DB200001487800130037000B
:100BA00011C0B30060DB20000148780051C0B300E1
:100BB00070DB20000148780021C0B30080DB2000FA
:100BC00001487800090037008040EB0060DB20001E
:100BD000014878008040EB0070DB2000014878007D
:100BE0008040EB0080DB2000014878000080FA00A4
:100BF000000006000200FA000000EB00000F780081
:100C000070DB2000904078000030200009010700D0
:100C1000CBC2BF00614060000004E000040032006D
:100C2000CBC2BF00624060000004E00002003A0056
:100C300010002000000F780070DB2000904078004A
:100C4000002020001701070070DB20009040780092
:100C5000001020001301070070DB20009040780096
:100C600000202000F30007001E0078000080FA003A
:100C7000000006000000FA0070DB200090407800C1
:100C8000003020000701070070DB20009040780052
:100C900000102000E700070070DB20009040780083
:100CA00000202000E30007000000EB000080FA00B5
:100CB000000006000C00FA00500798000000EB004E
:100CC000000F7800B0B42000104078000080FB00D6
:100CD0008000E900100020000100DD0030079800CE
:100CE0005E009000200798000000EB00400798008D
:100CF0002000370060DB200010417800AE0090003B
:100D00003E0090000080600001202000FC000700F1
:100D100070DB20009040780000102000C500070024
:100D200000082000260107000080FB001007980043
:100D300070DB20009040780000102000D9000700F0
:100D40002E00900000004000200798001E00780050
:100D500000004000000F78001E0090000000E0003E
:100D6000010032001E0FE8004E0090000000E80075
:100D700040079800B0B42000104078008080FB004D
:100D80004E009000808F5000DAFF3E001E00780079
:100D90000080FA00000006000800FA003007980002
:100DA000B0B42000104078000080FB008000E90013
:100DB000100020000100DD00100798003E009000A8
:100DC000000F78000000EB002007980014003700A7
:100DD00060DB2000104178001E0090001E006000C3
:100DE00001202000C600070070DB20009040780042
:100DF000001020008F00070070DB2000904078007A
:100E000000102000A70007001E007800000040002E
:100E1000000F78002E0090000000E80020079800E6
:100E2000B0B42000104078008080FB002E009000BD
:100E3000808F5000E6FF3E000080FA0000000600B0
:100E40000600FA000000EB00000F780000202000F0
:100E5000DB0007000000EB002007980016003700B9
:100E600070DB200090407800001020007100070027
:100E700000202000D20007000080FB00100798002F
:100E800070DB2000904078000010200085000700F3
:100E90001E00780000004000000F78001E00900047
:100EA0000000E000010032001E0FE8002E0090005C
:100EB0000000E80020079800B0B42000104078003F
:100EC0008080FB002E009000808F5000E4FF3E00E9
:100ED0001E0078000080FA00000006000200FA0000
:100EE000A06D8000B600070070DB20009040780005
:100EF000001020004F000700A06D8000B000070028
:100F0000004F780070DB2000904078000010200037
:100F1000640007001E80FB000080FA00000006004D
:100F20000200FA00004F780060DB200010417800DA
:100F3000916D80001E80FB007100070070DB2000B7
:100F400090407800001020003A00070070DB20007D
:100F50009040780000102000520007000080FA0046
:100F6000000006000400FA00204798000040EB0053
:100F7000004F78000900370070DB200090407800B7
:100F8000001020002B00070070DB2000904078004C
:100F900000102000430007001E4FE8002E40900084
:100FA0009E4F1000F4FF39000080FA000000060098
:100FB0000200FA00004F780060DB2000104178004A
:100FC000916D80001E80FB004D0007000080FA003C
:100FD000000006000200FA00004F780060DB2000ED
:100FE000104178001E80FB00011020004400070023
:100FF0000080FA00000006000200FA00004F7800AE
:1010000060DB2000104178001E80FB0001042000FE
:101010003B0007000080FA00000006000000FA0014
:10102000A06D8000660007000080FB000080FA00D1
:10103000000006000400FA00000F78002147980025
:10104000C0B5200010407800704060000004E0004F
:101050000B003A00601680001E00700060168800C9
:101060001E0078000080EA008180EA00800078009D
:1010700040168000008060004016880003003700A2
:10108000401680001E007000401688002E40900020
:101090000080FB003AA00200000000000080FA007F
:1010A000000006000400FA00000F780021479800B5
:1010B0001E0078000080EA008180EA00800078004D
:1010C0006016800000806000601688001E007800B6
:1010D0000080EA008180EA008000780040168000ED
:1010E00000806000401688002E4090000080FB00C9
:1010F0003AA00200000000000080FA000000060094
:101100000600FA00000F7800110798004247980087
:101110001E00E0000F003A001E0090000080EA0070
:101120008180EA0080007800601680000080600006
:10113000601688001E0090000080EA008180EA00AE
:101140008000780040168000008060004016880013
:1011500015003700C0B520001040780070406000D6
:101160000004E0000C003A00611680001E009000B0
:1011700000807000601688001E0090000080EA0069
:101180008180EA00800078004016800000806000C6
:101190004016880004003700401680009E00900032
:1011A00001007000401688004E4090000080FB0057
:1011B0003AA00200000000000080FA0000000600D3
:1011C0000400FA00000F7800401680001E00700036
:1011D0004016880000000000000000000000000031
:1011E000501680001E0060000000E0000300320086
:1011F0001000200010079800020037000000EB00EC
:10120000100798001E0090000080FA000000060001
:101210000000FA0020870200000000000080FA00B1
:10122000000006000200FA00000F78001E0078009F
:10123000CC86020000000000001020000080FA00B0
:10124000000006000000FA00FA850200000000001D
:1012500081002000D0922000ACA20200000000001B
:10126000D10020008044200036A3020000000000CE
:101270000080FA00000006000000FA003A86020032
:10128000000000006100200050932000ACA202008A
:1012900000000000C10020005045200036A30200DD
:1012A000000000000080FA00000006000000FA00C4
:1012B0006E870200000000000080FB000080FA0042
:1012C000000006000000FA000E8802000000000086
:1012D0000080FB000080FA00000006000000FA0019
:1012E0000040EB00EA870200000000000080FA00E6
:1012F000000006000000FA0010C0B300EA870200F8
:10130000000000000080FA00000006000000FA0063
:1013100010C0B300B2870200000000000080FA0095
:10132000000006000000FA000040EB00D887020031
:10133000000000000080FA00000006000000FA0033
:1013400010C0B300D8870200000000000080FA003F
:10135000000006000000FA0001012000A098200013
:10136000ACA2020000000000A0B4200010407800F1
:101370003C7802000000000000C2B300007A0200C6
:1013800000000000C0B52000104078000080FB0085
:101390004400DE00614060003C7802000000000074
:1013A00000C2B300007A02000000000031002000FB
:1013B000F0AD2000ACA20200000000000080FA00A6
:1013C000000006000400FA00B42102000000000042
:1013D000E61D02000000000010079800B421020082
:1013E00000000000E61D020000000000000F780071
:1013F0001E0090000000E000090034001E00900074
:10140000E40F500006003C001E0090000040E90080
:1014100080407800A0B42000014878000200370026
:101420000000EB00100798001E00E00010003400E0
:10143000200020009E0F10000D003C001E007800D0
:101440000040EA0061416000C0B520009040780093
:10145000614061004401DD00F0CEB30080C0600057
:1014600082C07000C0B5200001487800020037003B
:101470000000EB00100798001E0090000000E00044
:1014800026003A000000EB00F0678800B10320005E
:101490006048200036A30200000000008001EB003D
:1014A000420020001100200010002000E022020075
:1014B000000000000040E90080407800A0B4200057
:1014C00001487800F1042000B093200036A3020008
:1014D000000000008001EB0022002000110020002D
:1014E00010002000E0220200000000000040EA009E
:1014F00061416000C0B5200090407800614061000B
:101500004401DD00F0CEB30080C0600082C07000F6
:10151000C0B5200001487800010037008DFF0700AA
:10152000CB02A900CB22A900C922A800C902A900A8
:10153000A0B420009040780020C0B3006C85020069
:10154000000000000080FA00000006000400FA001D
:10155000000F78001E007800100798001E00900011
:10156000E10F50000C0032001E009000E10F50000F
:10157000040039001E009000E20F50000700320006
:101580000800370081032000A0992000ACA20200CF
:1015900000000000070037001000070025000700CA
:1015A0000400370041022000C020200036A30200C2
:1015B000000000000080FA00000006000200FA00AF
:1015C000000F7800B1002000C009210036A30200FE
:1015D000000000000080FA00000006000000FA0091
:1015E000F1032000209D200036A30200000000002F
:1015F0000040EB00FC87020000000000F00F20001C
:101600003AA002000000000010C0B300FC870200F6
:101610000000000010C0B300B2870200000000000C
:101620000040EB00FC870200000000000080FA0090
:10163000000006000A00FA00881F7800D10220008E
:1016400010A12000ACA20200000000000000EB008E
:10165000000F7800100037001E0478002087020079
:1016600000000000804078006300470001747800AB
:101670009E00780063004700614078000080FB0016
:101680009E7802000000000000C2B300007A020051
:10169000000000001E0FE800300020009E0F100028
:1016A000EDFF360060A92800D075020000000000A0
:1016B000A1002000E0A32000ACA202000000000076
:1016C00063004700104078000080FB004400DE000B
:1016D0000080FB00400798004E009000E90F50008A
:1016E000130032004E009000E90F500004003C004F
:1016F0004E009000E80F5000080032001B00370039
:101700004E009000EA0F50000E0032004E00900094
:10171000EF0F50001000320014003700610020006D
:1017200080A42000ACA202000000000013003700DB
:1017300061002000E0A42000ACA202000000000034
:101740000E0037006100200040A52000ACA202007E
:10175000000000000900370031002000A0A5200093
:10176000ACA202000000000004003700710020005D
:10177000D0A52000ACA202000000000060A9280053
:10178000D075020000000000B100200040A620003B
:10179000ACA202000000000063004700104090006F
:1017A0000080FB004700DE000004E00005003A0076
:1017B00061002000F0A62000ACA2020000000000A2
:1017C00004003700F100200050A72000ACA2020066
:1017D0000000000060A92800D07502000000000091
:1017E000C100200040A82000ACA2020000000000C0
:1017F00063004700104090008080FB0080F72F00BE
:10180000008060004380DE00204798002E4090005A
:101810000004E00005003A00D100200000A92000EB
:10182000ACA20200000000001E0037002E40900015
:10183000EF4F500005003A0031002000A0A5200025
:10184000ACA20200000000001600370000042000D7
:10185000000F7800E30047000040EB00804878006C
:10186000080037001E00780000004000000F7800DC
:1018700063004700104078008040E80063004700A4
:101880000148780063004700904078002E409000A7
:1018900080CF5000F3FF39001E007800DE77020091
:1018A0000000000060A92800D075020000000000C0
:1018B00091012000D0A92000ACA20200000000008D
:1018C000630047009040900070C0B30000C060000B
:1018D0002047980010002000000F7800E300470028
:1018E0000040EB0080487800080037001E007800B8
:1018F00000004000000F78006300470010407800AF
:101900008040E8006300470001487800630047001A
:10191000904078002E40900080CF5000F3FF3900B7
:101920001E0078003C7802000000000060A928003A
:10193000D0750200000000004F0478000080FA001B
:10194000000006000000FA00E0A82800A4750200CC
:10195000000000000080FA00000006000A00FA0003
:1019600070408000300798001000200040928800EE
:10197000F4FF070000003700EE79020000000000CD
:10198000104798001E4090000080FB004007980020
:10199000CE009000E38F5000200032004E009000F7
:1019A000E30F50000A003C00CE009000E18F500091
:1019B0005B0032004E009000E10F50005E003C00E2
:1019C000CE0090000100E000E7003200DB003700AD
:1019D0004E009000E60F50000E003200CE00900046
:1019E000E68F500004003C004E009000E50F5000D0
:1019F00095003200D1003700CE009000E78F5000F4
:101A0000640032004E009000E80F50005400320095
:101A1000CA003700CBFF0700D7FF3700BE00900099
:101A200030C0B300804878003E0090008000E8009D
:101A300080C0B3008048780021E3A800C0C0B30094
:101A4000B09E020000000000200798003E009000B9
:101A50008080E8002E0090004800DE00804878007A
:101A60003E009000E30040002E0090008048780087
:101A7000B0C0B300B09E0200000000002007980034
:101A80003E009000E40040002E0090004800DE0080
:101A9000804878003E009000E50040002E00900055
:101AA00080487800A0C0B300B09E02000000000093
:101AB000200798003E009000E60040002E009000B5
:101AC0004800DE00804878003E009000E7004000BB
:101AD0002E0090008048780090C0B300B09E0200B5
:101AE00000000000200798003E009000E800400041
:101AF0002E0090004800DE00804878003E009000F4
:101B0000E90040002E0090008048780021E3A90001
:101B1000A10020003E009000BF00070096FF3700A4
:101B2000EE79020000000000104798001E4090006F
:101B30008F00070090FF3700EE79020000000000E0
:101B400010479800EE79020000000000004F780076
:101B50009E4078001E409000C100070086FF3700BD
:101B6000EE7902000000000010479800EE790200B4
:101B700000000000004F78001E4090000080FB0035
:101B8000C800DD001E80FB000080700040928800CD
:101B900079FF3700EE79020000000000104798003E
:101BA0001E4090000080FB00200798001E4090001F
:101BB000E14F500004003A0030C0B3001E7A02002A
:101BC000000000000300370020C2B3001E7A0200AC
:101BD00000000000EE7902000000000010479800AD
:101BE000EE79020000000000004F78009E40900057
:101BF000A0CAB30080CF500003003A0050C5B30024
:101C00009E4F1000050032000000EB0020079800F6
:101C100020C2B3001E7A020000000000BE00900047
:101C200070C0B300804878003E0090008000E8005B
:101C30002E00900080487800210020003E00900097
:101C4000750007004CFF3700EE790200000000002D
:101C500010479800EE79020000000000004F780065
:101C60008560A9001E4090000080FB00C800DD00D8
:101C70001E80FB0000807000100798009E009000FE
:101C800000002200808F5000020036000000220079
:101C9000100798001E009000670040004300DE001F
:101CA00020079800BE00900050C0B3008048780024
:101CB0003E0090000000E8009E409000014878003F
:101CC0003E0090000080E8001E48780031002000AF
:101CD0003E009000500007007040800000408800E7
:101CE0002E00900000004000104088000000EB0033
:101CF0002040880071408000408320000080400028
:101D0000304088000000EB00404088000000EB00FD
:101D1000504088009560A8004092800031408000CB
:101D200004408000800178001E01900004007800CB
:101D30001EA60200000000000FFF3700BE0090004A
:101D40000040EB00804878003E0090008000E800F2
:101D50000040EB0080487800110020003E00900019
:101D60002D00070004FF37000080FA000000060085
:101D70000200FA00004F7800CAC2A900CB22A900D5
:101D8000CB02A900CB42A900CA02A90020C0B3001F
:101D90009E4F100006003A00CAC2A800CB02A8005D
:101DA000CB22A800CB42A800CA02A8000500370039
:101DB000CAC2A900CB02A900CB22A900CB42A9002C
:101DC000CA02A90010C0B3009E4F100003003200E9
:101DD00020C0B3009E4F100007003A00C8C2A900FF
:101DE000C922A900C902A900C942A900C802A900C4
:101DF000C8E2A80006003700C8C2A800C922A8008F
:101E0000C902A800C942A800C802A800C8E2A800E8
:101E10000080FA00000006000600FA001007980093
:101E2000210798000000EB00000F78000700370042
:101E30009E0078001E009000008040001040780056
:101E4000007A0200000000001E0FE8002E00900043
:101E50009E0F1000F6FF39000080FA000000060017
:101E60000400FA00004F7800114798001E80FB0024
